:020000041004E6
:100000000000012011660410355F0410375F0410F2
:1000100000000000000000000000000000000000E0
:10002000000000000000000000000000395F041024
:1000300000000000000000003B5F04103D5F041062
:10004000756604107566041075660410755F0410FB
:100050008D5F0410756604107566041075660410D3
:10006000455F041075660410F95F0410756604108E
:1000700075660410A55F041000000000B55F041051
:1000800075660410495F0410E95F04100000000069
:10009000E15F04100000000000000000D15F0410C8
:1000A000D95F0410F15F04100000000000000000A0
:1000B0000000000000000000000000000000000040
:1000C00010B5904216D98AB2030C090C0C4659435C
:1000D00080B25343444350431B191A041B0C10189D
:1000E000594180225203002312184B41520DD8026D
:1000F000104310BD4843802252031218520D10467F
:1001000010BDC0468B0707D0013A22D30B780131CE
:10011000037001308B07F7D1830730D0DB4219D051
:100120000138043A08D308C943701B0A43801B0CEA
:1001300003710430043AF6D2D20707D30B88437018
:1001400001D08A78C2701B0A8370704701D00B7887
:1001500043707047043A06D308C903801B0C4380E0
:100160000430043AF8D2D20705D30B88038005D0B7
:100170008B788370704701D00B780370704770B430
:10018000103A03D378C978C0103AFBD2530701D391
:1001900018C918C001D508C908C0D20704D30B88F4
:1001A000038002300231002A01D50B78037070BC45
:1001B0007047C046EFF31482EFF30981154880F3CE
:1001C0001488BFF36F8FF0B543464C4655465E46E4
:1001D0006746F8B4104CEFF30883636006B4BFF3CE
:1001E0004F8F30BFC046C0460B4C646884F308880C
:1001F00082B003BCF8BC9846A146AA46B346BC46AA
:10020000F0BC04BC80F3098881F31488BFF36F8FBE
:100210001047C04600000000040000200023C25C1C
:100220000133002AFBD1581E7047000002B471460A
:1002300049084900095C49008E4402BC7047C04629
:1002400003B47146490840004900095E49008E44E4
:1002500003BC704703B47146490840004900095A7D
:1002600049008E4403BC7047002243088B4274D37C
:1002700003098B425FD3030A8B4244D3030B8B42A7
:1002800028D3030C8B420DD3FF22090212BA030CB0
:100290008B4202D31212090265D0030B8B4219D391
:1002A00000E0090AC30B8B4201D3CB03C01A5241B1
:1002B000830B8B4201D38B03C01A5241430B8B42F9
:1002C00001D34B03C01A5241030B8B4201D30B03E2
:1002D000C01A5241C30A8B4201D3CB02C01A524109
:1002E000830A8B4201D38B02C01A5241430A8B42CC
:1002F00001D34B02C01A5241030A8B4201D30B02B5
:10030000C01A5241CDD2C3098B4201D3CB01C01ACE
:10031000524183098B4201D38B01C01A52414309D8
:100320008B4201D34B01C01A524103098B4201D3C6
:100330000B01C01A5241C3088B4201D3CB00C01A33
:10034000524183088B4201D38B00C01A52414308AB
:100350008B4201D34B00C01A5241411A00D20146D0
:10036000524110467047FFE701B5002000F0F0F859
:1003700002BDC0460029F7D076E7704703460B431D
:100380007FD4002243088B4274D303098B425FD38E
:10039000030A8B4244D3030B8B4228D3030C8B42BA
:1003A0000DD3FF22090212BA030C8B4202D31212A0
:1003B000090265D0030B8B4219D300E0090AC30B75
:1003C0008B4201D3CB03C01A5241830B8B4201D322
:1003D0008B03C01A5241430B8B4201D34B03C01A0B
:1003E0005241030B8B4201D30B03C01A5241C30A83
:1003F0008B4201D3CB02C01A5241830A8B4201D3F4
:100400008B02C01A5241430A8B4201D34B02C01ADD
:100410005241030A8B4201D30B02C01A5241CDD282
:10042000C3098B4201D3CB01C01A524183098B42CD
:1004300001D38B01C01A524143098B4201D34B01B6
:10044000C01A524103098B4201D30B01C01A524119
:10045000C3088B4201D3CB00C01A524183088B42A0
:1004600001D38B00C01A524143088B4201D34B0089
:10047000C01A5241411A00D20146524110467047FB
:100480005DE0CA0F00D04942031000D34042534000
:1004900000229C4603098B422DD3030A8B4212D3C0
:1004A000FC22890112BA030A8B420CD389019211F2
:1004B0008B4208D3890192118B4204D389013AD02F
:1004C000921100E08909C3098B4201D3CB01C01A04
:1004D000524183098B4201D38B01C01A5241430917
:1004E0008B4201D34B01C01A524103098B4201D305
:1004F0000B01C01A5241C3088B4201D3CB00C01A72
:10050000524183088B4201D38B00C01A5241D9D289
:1005100043088B4201D34B00C01A5241411A00D20A
:100520000146634652415B10104601D34042002B06
:1005300000D54942704763465B1000D3404201B585
:10054000002000F005F802BD0029F8D016E770473A
:100550007047C0469140030090409C46203A93402B
:10056000194352426346D3401943704784461000F2
:1005700062468C461900634600E0C0461FB501F094
:10058000B5FA002801D40021C8421FBD10B501F002
:10059000F7F94042013010BD10B501F0A7FA00286C
:1005A00001DB002010BD012010BDC04610B501F0D8
:1005B0009DFA002801DD002010BD012010BDC046BD
:1005C00010B501F023FA002801DC002010BD012045
:1005D00010BDC04610B501F019FA002801DA00205C
:1005E00010BD012010BDC0461C2101231B049842F0
:1005F00001D3000C10391B0A984201D3000A0839B4
:100600001B09984201D30009043902A2105C40186A
:100610007047C0460403020201010101000000000E
:1006200000000000002B11D1002A0FD1002900D1B9
:10063000002802D00021C943080007B4024802A1E3
:100640004018029003BDC04609FFFFFF03B468468F
:1006500001B5029800F034F8019B9E4602B00CBC34
:100660007047C046F0B5CE469946030C9C4613042D
:1006700047461B0C1D000E0061460404240C80B587
:100680000700100C4B436543414360432C0CC018DA
:1006900024188C46A34203D980235B029846C444A5
:1006A000494679435643230C2D042D0C8919634484
:1006B00024046019C918C0BCB946B046F0BDC04694
:1006C000F0B557464E464546DE46E0B504000D00FF
:1006D0009246994683B08B4230D82DD04946504639
:1006E00002F06AFA29000600200002F065FA331AC7
:1006F0009846203B34D49B4653465A469340424644
:100700001F00534693401E00AF423BD8AF4200D17A
:1007100079E05B46A41BBD41002B00DA76E00022A5
:1007200000230092019301235A4693400193012331
:1007300042469340009329E08242CFD90022002311
:10074000009201930C9B002B01D01C605D6000980F
:10075000019903B0F0BCBB46B246A946A046F0BD25
:1007600042469B4620239B1A5246DA4041461300DC
:100770004A468A40170042461F43534693401E0094
:10078000AF42C3D900220023009201934346002BBD
:10079000D8D0FB0772081A4346467B080EE0AB42EE
:1007A00001D1A2420CD8A41A9D41012024196D4107
:1007B0000021013E24184D41002E06D0AB42EED957
:1007C000013E24196D41002EF8D1009801995B4635
:1007D00000196941002B24DB2B005A464646D340C2
:1007E0002A001C00F2405B461500002B2ADB260085
:1007F0009E40330026004746BE403200801A994191
:10080000009001919EE7A342BCD882E74246202394
:1008100000219B1A0022009101920122DA400192EC
:1008200085E7424620239B1A2A0046469A40230029
:10083000F340464613432A001C00F2405B46150075
:10084000002BD4DA202342462F009B1B9740260022
:10085000DE403B003343CDE7F0B546464F46D64633
:100860004502C0B5C30F470098460E1C6D0A3F0EE7
:100870005BD0FF2F21D08023ED00DB041D4300233C
:1008800099469A467F3F74027300640A1B0EF60F66
:10089000002B20D0FF2B43D080220020E400D20484
:1008A00014437F3B4246FF1A4B4672400F2B00D940
:1008B0009DE071499B00CB589F46002D5AD10823DB
:1008C0009946063B74029A467300FF27640A1B0E82
:1008D000F60F002BDED1002C3BD1012342464946C6
:1008E000724019430E2918D86448890041588F4630
:1008F0005346022B00D1B8E0032B6ED042462C00A9
:10090000012B40D100200024C0052043D207104312
:10091000E0BCBA46B146A846F0BDFF200024F3E78C
:10092000002C20D10223FF3FD8E7002D05D104235E
:100930009946033B00279A46A5E72800FFF754FE97
:100940007627431F9D4000237F4299469A463F1ACF
:1009500099E72000FFF748FE431F9C4076235B4247
:100960001B1A00209EE703234A461A4391460320A0
:10097000FC3397E70C239946093BFF279A4682E709
:1009800003282CD0320038007F30002847DD630771
:1009900004D00F232340042B00D00434230103D5BB
:1009A0003800374B80301C40FE28B6DCA401640AB6
:1009B000C0B2A9E780240022FF20E403A4E780233B
:1009C000DB031D4201D01C420BD08024E4032C43E6
:1009D00064024246FF20640A96E746462C008023C4
:1009E000DB031C4364023200FF20640A8CE76D01C4
:1009F000600185422DD21B230024013F01262900DE
:100A000064006D00002901DB854201D32D1A3443B7
:100A1000013B002BF3D16B1E9D412C43B3E7012317
:100A20001B1A1B2B00DD6DE721009E37D940BC400F
:100A30000B00611E8C412343590704D00F2119403C
:100A4000042900D00433590113D49B0100205C0A0F
:100A50005AE71A2301242D1AD0E7981E4342584121
:100A6000404232000024C0B24EE74246FF2000243C
:100A70004AE70120002447E7E4B8061024B906102D
:100A8000FFFFFFF710B5041E0DD0FFF7ADFD9E234D
:100A90001B1A962B0CDC082834D0083884406402DA
:100AA000640AD8B201E000200024C005204310BD34
:100AB000992B13DC421F9440144A224061071CD03A
:100AC0000F212140042918D00432D408520115D531
:100AD0009F236402181A640AC0B2E6E702002100EC
:100AE0001B3291400A00511E8A410521091ACC404F
:100AF0001443064A22406107E2D1D4086402640A22
:100B0000D8B2D2E76402640A8E30CEE7FFFFFFFB63
:100B1000F0B54F464646D646C0B50D0382B00092AA
:100B200001934E00C300CC0F690A450F9C46009A02
:100B3000019B0D435F001903D80F009B490A5B0F0F
:100B40001943009B760D7F0DDA00F31B844258D0C9
:100B5000002B13DD002F00D088E00800104300D1E7
:100B600059E1581E012B00D1C2E2B14FBB4200D166
:100B700041E1382800DD6AE2030064E1002B00D186
:100B8000B1E0BB1B002E00D0E1E164462C4300D154
:100B900076E25C1E012B00D1E8E2A54EB34200D103
:100BA000B7E2382C00DC6BE3541EA2429241524261
:100BB0008D1AA0461E0004002A0268D443461F1D59
:100BC00047459B415B42ED182B0200D49DE3984AB8
:100BD0000136964200D1EBE0964A73052A405B0D40
:100BE0005107FF0852020F43120B1B051343E40782
:100BF00023433800190002B0E0BCBA46B146A8460B
:100C0000F0BD002B00DCD7E0002F00D09AE00800F8
:100C1000104300D1FFE0581E012B00D148E2844F61
:100C2000BB4200D1E7E0382800DCB8E280221204A1
:100C3000154200D149E31E000023150098467C4B65
:100C400001369E4200D1B3E07A4B01211D4043465C
:100C50005A081940EF070A4317436D087B07B3D0C2
:100C60000F233B40042BAFD0B846A7E7704886421D
:100C700000D1C0E0382B00DCE2E001235B4263449A
:100C80009C45804140422D1A98462B0296D501235F
:100C90005B429846684D2800FFF7A6FC0300083B1E
:100CA00020214046CA1AD040020040469D4098404C
:100CB0002A438046B34200DA72E1981B4346013072
:100CC000091A45468B40C5405E1EB34117008F4050
:100CD0002B431F43C2403B00150000261343BDD1E8
:100CE0000027002281E7554F731C3B4200D01BE1D7
:100CF00063460F002B431743002E00D0C4E1002BA6
:100D000000D145E2002F00D107E163469B1A9846C7
:100D1000C445B6416B1A76429B1B8026360433428B
:100D200000D1CBE26346D31A9A4292411F00491B7D
:100D300052428A1A9C46174300D0EDE20400002379
:100D4000002252E73A48864255D0382B00DD48E170
:100D50008020000401431F2B00DDE3E12027F81A67
:100D6000824608005746B840814610004F46D8409A
:100D7000074338005746BA40D940571EBA416D184C
:100D8000104360448046E045804140422D182B02CC
:100D900000D554E743465B0700D1B9E20F23424632
:100DA0001340042B00D009E733004246D20834E058
:100DB00033000022002718E7002B00D18FE0BB1B77
:100DC000002E00D033E16046284300D140E2581E97
:100DD000012B00D10AE2164EB34200D185E2382839
:100DE00000DC87E280252D04294200D19CE21E0010
:100DF0000023984623E763466E07D8080643ED08AC
:100E000037002F4311D0802212032A4312033700E8
:100E1000074B120BE9E66246D2086E071643044AF6
:100E2000ED089342ECD03700D6E0014B0022DCE61F
:100E3000FF070000FFFF7FFFFFFF7F00FE070000AE
:100E40008020000401431F2B00DDB1E02027F81AA9
:100E5000824608005746B840814610004F46D840A9
:100E6000074338005746BA40D940571EBA416D1A59
:100E7000104363461B1A9C458041984640422D1AF8
:100E80002B0287D56D026D0A002D00D003E7404686
:100E9000FFF7AAFB030018331F2B00DC00E74246D4
:100EA000083882409E4200DD91E09B1B581C1F28A1
:100EB00000DCF8E117001F3BDF40202805D040236D
:100EC0001B1A9A40531E9A411743002F3CD000260C
:100ED0007B0700D0C4E63500B846330065E7CB4851
:100EE000731C034200D085E063462B43002E00D0E4
:100EF00092E10F001743002B00D1D8E1002F0CD056
:100F00006244624580416D1840422D182B0200D585
:100F1000F2E1170094462F4316D063466F07D808B6
:100F200007430023ED0857E063469B1A9846C445E3
:100F3000BF416B1A7F42DB1B1F0200D5AEE0474664
:100F40001D001F43A0D10024002300224DE6B04C19
:100F5000A74200D1DDE0382B00DD85E080242404A9
:100F600025431F2B00DDECE02026F41AA1462C00BF
:100F70004E46B4406646DE403443A04666464C4684
:100F8000A640DD40741EA6414446491B3443131B52
:100F90009A4292415242984604003E008D1A6FE7F1
:100FA000F61A03009B4D15405B0700D0F6E6FBE602
:100FB00018000F002038C740202B03D04020C31A50
:100FC00099400A43531E9A411000384351E7914912
:100FD000F31A0A405707D5082A035B05120B5B0D6D
:100FE00003E680231B041D4200D1BBE01D0000234B
:100FF000984624E68648834200D1DAE66244624598
:101000008041691840420918C807520810438046B9
:101010004D08520705D00F221E000240042A00D0BE
:10102000CCE542466F07D20817430D09D4E778484C
:10103000874200D1D5E0382B00DCB2E080252D04BA
:10104000294200D14CE100233E009846F7E50122F9
:10105000524262449445804140422D1A90461E00FF
:101060002A0200D513E6A9E5531E9A429241524244
:101070008D1A984604003E002B0200D507E69DE538
:1010800004000D00D208C8E6002B00D0E3E0002FDA
:101090003FD1802200245E4B1203A6E56346D31A9B
:1010A0009A4292414D1B524298460400AD1AEBE61B
:1010B00062441600664580416A18404212181302C5
:1010C00000D49DE0534973080A40D10719435708DB
:1010D0005B0700D1FEE00F230B40042B00D1F9E0A9
:1010E0000B1D98468845AD416D420223ED195CE623
:1010F00063469B1A9C4580416D1A40422D1A9846C2
:101100002B020DD443466F07DB081F43ED08012374
:1011100062E74E07D20804001643CD0870E60400CB
:101120000126AFE618000F002038C740202B03D05F
:101130004020C31A99400A43531E9A411000384375
:101140001FE61C002E00203CE640202B05D040244A
:10115000E31A9D4063462B439C466446631E9C41B4
:10116000344314E701236344984627E56346D31AC2
:101170009A4292414D1B5242AD1A98462B02CED450
:1011800043466F07DB081F4304000123ED0823E7F4
:10119000002F00D1D7E604000D009446BDE6030001
:1011A000D9E58020000405431F2B6BDC2020C01AEA
:1011B000804628004646B0406646DE400643B146BB
:1011C00060464646B040DD40461EB0414E46491995
:1011D0003043804690449045924152423E0055181B
:1011E000D5E54E07D2081643CD0809E663469E189A
:1011F00096429241691852428A18130200D561E75B
:101200005707F60801233743D508E5E6FE07000037
:10121000FF070000FFFF7FFF002BE2D06346DE08E0
:101220006B071E430B00ED08134300D1E8E5802354
:101230001B031D4206D0C808184203D10500D6087A
:1012400049070E43730FF600F6085B071E43D7E508
:101250000D00D208E1E56346DE086B071E43ED088A
:10126000002F00D1CCE580231B031D42EAD0CF081C
:101270001F42E7D1D608490704003D000E43E1E7CD
:1012800023006EE618002E002038C640202B05D023
:101290004020C31A9D4063462B439C466046431E34
:1012A0009841304395E720210023091A0EE50023D9
:1012B000002F00D1BAE50D00904676E547461F4362
:1012C00000D140E61D00C44627E601226244904654
:1012D0001E0073E4C9087F0702230F4315097BE64C
:1012E000531C98460D003E0068E4D6084B071E4389
:1012F000CD0885E5030057E7114BD2082B405F0767
:1013000017435A02120B01236FE43300B8464CE531
:101310004346DA08330080E532420AD0084B040025
:101320001A40674601235BE4013290460D001E001F
:1013300044E4DB0857071F4304000023D5084BE6AD
:10134000FFFF7FFFF0B5DE46454657464E46E0B507
:1013500087B0009201930B031B0B9B46CA0F4B00F7
:10136000040080465B0D029200D1BFE08F4A934299
:1013700038D05946420FC9000A438021090411435D
:10138000C20090468A4A894692469A440023002425
:101390000393009E019F3B031B0B7A0030009B468A
:1013A000520DFD0F002A00D17FE0804B9A426ED093
:1013B0005946730FC9000B438021090419438B461A
:1013C0007B49F3008C46514662448A1A92460021BA
:1013D000029E6E40F6B20F2C00D9F9E0754AA400C7
:1013E000125997465A460243914600D0B6E09A46B3
:1013F0000223904608240393CBE72E00002100230C
:10140000002288461B051343F60733434046190064
:1014100007B0F0BCBB46B246A946A046F0BDCB46DD
:101420004346029D0399022900D1FAE1032900D124
:10143000A1E00129E1D0604A524490464446002C84
:1014400000DC00E25A0704D00F221A40042A00D020
:101450007FE22E00DA085B46DB0106D55946574B82
:10146000802419408B46E4005444554B9C4209DCCF
:101470005B465B07134398465B4664055A02120BB2
:10148000630DBFE7002100228846484BBAE75B4660
:10149000009A13434B4A9446E244002B59D102224E
:1014A000144300220221934692E75B46009A1343BD
:1014B00049D05B46002B00D1A4E15846FFF794F8D1
:1014C000030002000B3B1D27009EFB1A110058462B
:1014D000DE4008398840330003439B46009B8B4025
:1014E000394952448A460021924471E75B460343DE
:1014F000994621D05B46002B00D171E15846FFF799
:1015000073F80B235B429C460200844466461D230D
:101510009B1B260011005846DE40083988403300E6
:101520000343994623008B409846284B00249B1A7E
:101530009A46002303932CE7002398469A460133EA
:101540000424039325E7012214430022012193463A
:101550003EE7032303211C43330039E79A46032364
:10156000D9460C24039314E70023802298460026D2
:101570000E4B120346E78022594612030A43120318
:1015800098462E00094B120B3CE780224946120375
:10159000114202D059461142F0D080224B4612032C
:1015A0001A431203029E014B120B2BE7FF070000A8
:1015B00001FCFFFF60B90610FF030000FFFFFFFE04
:1015C000FE07000001F8FFFFF30300000DFCFFFF22
:1015D000CB4500D2FAE000D1F5E001225242944618
:1015E0000022444648469046E2445A461F0E1202E4
:1015F0001B020293130C994617433B041B0C4946EC
:101600000093FEF7B7FE009A0B044243210C05003D
:1016100019438A4207D9C919013D8F4203D88A422A
:1016200001D9851EC919881A4946FEF7A3FE009AFA
:10163000240442430904240C03000C43A24204D9AD
:10164000E419013BA74200D8F7E00299A01A2D0443
:101650000C0C09041D43090C2A0C2B04AB460D008D
:101660001B0C5D43059163435143049462435B1833
:101670002C0CE318994203D9802149028C4662441C
:10168000190C2D041B042D0C8A185D19904200D2F0
:1016900087E000D182E043465D1BA8459B41801A4C
:1016A0005B42C01AB14B534498461C00874200D19C
:1016B0000CE14946FEF75EFE0200009B03905A4390
:1016C0000B04290C19438A420AD90300C919013BAA
:1016D00003938F4204D88A4202D9831E0393C91907
:1016E000881A4946FEF746FE0A00120494462A0468
:1016F00065460099120C414303002A43914207D9E1
:10170000D2190138974203D8914201D9981ED219B3
:10171000039B521A1B0403430598190C05008C46C1
:101720001904090C4D4389466146009565464843B6
:1017300004994D43AC464D464D432918009D2D0C50
:10174000A9464944884203D9802040028146CC44BE
:10175000009D080C2D0409042D0C60444D19824293
:101760000FD30BD001221343814A92456CDB1A1D23
:101770009A429B415B42D2089B446CE6002D00D10B
:1017800093E0591EBA188C46BA4200D285E08242D4
:1017900000D2C7E000D1D5E00B00E3E7A84500D3B5
:1017A00079E75B46591E029B9C46E0441C00984525
:1017B0009B415B42DB19C018874238D2824278D8FD
:1017C00075D08B4667E7434500D906E74A46D407FC
:1017D00050084246520814434246D207904604E756
:1017E000FEF702FF15239C46844402006346203224
:1017F0001C2B00DC8AE6230008388340994600232E
:10180000984692E6FEF7F0FE030002001533203200
:101810001C2B00DC57E600990838814000238B46DA
:101820005EE600212E0000228846524BEAE5874200
:10183000C7D14445C2D98B462DE7A24200D804E760
:10184000831EE41901E72E0001224146521A382A6C
:1018500000DDD3E51F2A3FDC47481C0050445946B1
:1018600083408140D440581E834121430B43594655
:10187000D1400A00590709D00F211940042905D089
:10188000191D99429B415B42D2180B00110268D589
:101890000021012300228846B4E50B00824200D0DB
:1018A00060E7029A954200D05CE73500C6E5454501
:1018B00087D902235B429C46029BE3449C46E0445A
:1018C00098459B415B42DB19C018E4E6002B36DDEE
:1018D000012300229B44BEE51F2140464942091ACC
:1018E0005846C8400100202A04D05846234A524492
:1018F000904003435A1E934107200B4301000022EE
:101900001940184209D00F21194004291FD0181D71
:1019100098428941030049424907DB080B43984636
:1019200000236FE50299023B49008C4602998C45E1
:1019300089414942C919521861460291AEE7012313
:101940005B4281E70299A942ECD36346A9E70021F3
:10195000E3E71A1D9A429B415B422E00D2089B444A
:1019600079E551075202120BD7E7C046FF0300008A
:1019700002FCFFFFFF0700001E0400003E04000001
:10198000F0B55746DE464E464546E0B50D0004002C
:10199000E80F83460903D80F090B82461A488C4684
:1019A0001F0369005E00490D3F0B760D81421AD07E
:1019B000864211D00120B1420FD1BC450DD1A242C7
:1019C0000BD1D3451ED0002907D1614611430A002F
:1019D000531E9A41100000E00120F0BCBB46B24605
:1019E000A946A046F0BD01208E42F6D1614639439A
:1019F0000F0017432743F0D15B465246981A431E07
:101A00009841EAE70020E8E7FF070000F0B55746F5
:101A10004E464546DE46E0B50D000E034900490D31
:101A20008A46DF0FE90FBC4683B02F4F0400804683
:101A30000191580019039146360B090B400DBA4528
:101A40001DD0B8420DD05746002F2AD1344300286C
:101A500024D10A4336D0002C41D1634658000138C6
:101A600015E0114338D15346002B01D12643F4D061
:101A7000019B634507D1019B5800013807E02643CD
:101A80002AD1504521D00120019B5F42384303B049
:101A9000F0BCBB46B246A946A046F0BD002CDCD047
:101AA000E6E70028EFD0019B6345ECD18245EADCF4
:101AB000E1DB8E42E7D8DED1C845E4D80020C84536
:101AC000E5D2D8E7002CE2D0DDE7114304D1019B39
:101AD0006345D8D10020DAE702204042D7E7019BD6
:101AE0006345E6D0CFE7C046FF070000F0B5574694
:101AF0004E464546DE46E0B50D000E034900490D51
:101B00008A46DF0FE90FBC4683B02E4F04008046A3
:101B10000191580019039146360B090B400DBA4547
:101B20001ED0B8420DD05746002F27D1344300288D
:101B300033D10A4334D0002C40D1634658000138D9
:101B400015E0114312D15346002B01D12643F4D0A6
:101B5000019B63451DD00120019B5F42384306E095
:101B6000264303D15045F6D111431CD0022003B0C7
:101B7000F0BCBB46B246A946A046F0BD0028EAD05C
:101B8000019B6345E7D18245E5DC02DB8E42E2D86A
:101B90000ED0019B58000138E9E7002CCDD0D7E7E3
:101BA000002CE4D0D7E7019B00206345DFD0D2E7CB
:101BB000C845D0D80020C845D9D2EAE7019B634583
:101BC000E4D0C8E7FF070000F0B557464E4645464B
:101BD000DE46E0B51F000B031B0B16009846CA0F2C
:101BE0004B000400924685B05B0D00D1C2E1CC4AA7
:101BF000934200D128E14146420FC9000A438021A7
:101C000009041143C2009146C64A884693469B4444
:101C10000023002501933C037A00FB0F3000240BC6
:101C2000520D009300D185E1BD4B9A4200D160E195
:101C3000BC4B9C46624493440A2D00DD14E1730FB3
:101C4000E4001C4380231B042343F0005246009908
:101C500000264A409246022D11DD0122AA40A6210B
:101C60001400C9000C400A4200D0FDE09021890018
:101C70000A4200D0D4E18821114200D0EFE0494669
:101C80004A460904140C090C020C0F00150000044C
:101C9000000C654347430195B9462F000D0006002F
:101CA0005543AC464D4666432D0CB4446544AE42A4
:101CB00005D93E0080277F02BC46664401964F4608
:101CC0003F043F0C2E0C2D04ED1902951D0C1B0436
:101CD0001B0C00951D001F0065434F43AC46009D43
:101CE00069436C433D0CA946614449448C4503D982
:101CF00080256D02AC4664443F040D0C3F0C090482
:101D0000C919AC467518039545462E04360C2F0CA0
:101D1000350045437843804638006444AC462D0C7A
:101D2000A9465043724342444A44904503D9802512
:101D30006D02A8464044150CA84665462D042D0C9E
:101D4000AC4635005D4312046244AC467B43009DC3
:101D5000404498462B006E4365467B4346442D0C19
:101D6000AD191F000093A84504D980235B02984653
:101D700047440097039B019E98462B04464498468F
:101D800063468E4289411B041B0C4344B6184942EA
:101D90001B195F1896429241BC46524280469146BA
:101DA0008C458941A3429B41E044C14449425B4286
:101DB000914592410B43804589412D0C4942524245
:101DC0000A435B199B18009A029994464A46634459
:101DD0005B02D20D1A43904672020A43511E8A4199
:101DE000F60D16434A4652021643B146DB0154D45F
:101DF0004D4A5A44002A00DC18E133005B0715D035
:101E00000F215B463140042910D04946081D484542
:101E100089418146494288444146C90106D5414627
:101E2000424A114080228846D2009A18404B9A427A
:101E300000DD2BE141464B464C07DB081C435205B5
:101E40004B021B0B520D1AE042460243914600D052
:101E5000E0E09B460223904608250193DBE6009ACA
:101E60009846924681460196019B022B00D10DE1D6
:101E7000032B35D0012B1BD1002200230024120597
:101E80001A435346DB071A432000110005B0F0BC8B
:101E9000BB46B246A946A046F0BD012273083240B7
:101EA00013434246D2071343994643465B0898467C
:101EB00080225B46D2005A440133002A00DCB6E09F
:101EC00049464907A8D00F214846014004299CD122
:101ED000A2E70F2D00D1FDE0009BA0469A46B14637
:101EE000802342461B0313431B034C460C4A1B0B27
:101EF000C5E70B4933008C462343E344002B77D1DD
:101F0000022129430A29AFDC5046009C60408246EA
:101F1000002D00D10EE10D00002002269DE6C046F6
:101F2000FF07000001FCFFFFFF030000FFFFFFFEB3
:101F3000FE070000230033434BD0002C00D1BBE050
:101F40002000FEF751FB030002000B3B1D20C31ACB
:101F50003000D84011000300300008398C40884020
:101F6000234359468A1A78498B4693440A2D00DC4C
:101F70006CE679E743460343994623D04346002B5A
:101F800000D187E04046FEF72FFB0B235B429C46C7
:101F90000200844411004046083988401D238046D1
:101FA00060461B1A2000D840030040460343984671
:101FB00023008B409946644B00259B1A9B460023C7
:101FC000019328E6002398469B460133042501939C
:101FD00021E6012215430A2D00DD45E7524600990E
:101FE0004A409246022D00DC46E70020012634E6F6
:101FF00003231D430A2D00DD6BE75346009A882119
:1020000053400122AA409A4603262300114200D1E0
:1020100035E624E79B46032381460C250193FAE528
:1020200000239A468023494A1B0328E75B46012187
:10203000891A382900DD1FE71F295ADD1F20404279
:10204000821A4046D040202908D0414A9446424650
:1020500063449A4013004A461A4391464A46072170
:10206000531E9A410C00024300231440114209D030
:1020700008311140042960D0111D9142A4410A0089
:1020800064426407D20814430022F8E600230024C7
:102090002E4AF4E6FEF7A8FA15239C468444020073
:1020A000634620321C2B00DC74E700239946230092
:1020B0000838834098467EE7FEF796FA0300020050
:1020C000153320321C2B00DC40E7330008388340F6
:1020D000002046E7802342461B031A4200D1FFE658
:1020E0001C4200D0FCE6009A234392463400174A73
:1020F000C5E6184A404694464A4663449840CA405A
:1021000010434A469A40531E9A4143460243CB40ED
:10211000510709D00F211140042905D0111D91420A
:10212000924152429B180A00190208D5012200234D
:102130000024A4E600230024A1E60024A2E75C0713
:102140005B021B0B9EE7C0460DFCFFFFFF07000074
:102150003E0400001E040000F0B54E464546DE4633
:102160005746E0B583B0009001910D034E000199F0
:10217000760DCC0F690A009D6D0F0D4300990092FA
:102180000193C8001903019BCB4A5B005B0D994684
:10219000019B8346DB0F98464B0A0099490F194370
:1021A000009BDB009C469A46914500D173E00123D9
:1021B00047465F404B46B846F31ABC4216D0002B48
:1021C00000DC9AE24F46002F00D082E067460F43C2
:1021D00000D13AE15F1E012B00D1A4E2934200D16D
:1021E0002EE1382F00DD43E23B003EE1002B00DC16
:1021F000D7E24F46002F00D0F8E067460F4300D1EA
:1022000023E15F1E012B00D157E2934200D117E179
:10221000382F00DC04E380221204154200D1AAE327
:102220001E0015000027A44B01369E4200D103E199
:102230000122A24B3A401D4079081143EA070A43A4
:102240006D08530709D00F231340042B05D0170046
:102250003A1DBA42BF417F42ED192B0200D477E309
:10226000954901368E4200D1E6E0944973050D4050
:102270005B0D6907D2086D020A432D0B1B052B432A
:10228000E40723431000190003B0F0BCBB46B2467C
:10229000A946A046F0BD8A4BF21863460B434CD0CA
:1022A000444550D0002A6CD0002E00D17DE1634619
:1022B00044464F07DA081743C8083A00024300D1E2
:1022C000CDE080252D0305432D033A007A4B2D0BDD
:1022D000D4E7964200D1B3E0382B00DCC2E0471EC1
:1022E000B842804140422D1A2B02B1D50127754DCD
:1022F0007F422800FEF778F90838202339001A1A9F
:102300008540D14087402943B04200DA45E1801B37
:1023100001301B1A3D009F40C5407A1E97410A00BC
:102320009A402F433A43C14013000D0000260B434F
:1023300000D086E700220025A0E7474601235F4042
:10234000B8464445AED1002A00D1EFE0002E00D0BF
:1023500088E14B462A00024300D1A0E25A1E012B1D
:1023600000D1B7E2544EB34200D17BE1382A00DC01
:1023700012E380252D04294200D112E31E0000271C
:1023800051E7514A731C134200D0F4E062462B001F
:102390000A430343002E00D074E1002B00D123E256
:1023A000002A00D1E0E06346C71AB8429241802675
:1023B0006B1A52429B1A3604334200D1C1E2634683
:1023C000181A844592414D1B5242AD1A0124020055
:1023D00043462A431C40002A00D1DBE0354200D1AD
:1023E000E9E2364B02001D40012342E7964227D026
:1023F000382B00DD11E18022120411431F2B00DD78
:10240000A1E120220F00D21A914697406246DA409D
:102410001743B84662464F46BA40D940571EBA41A4
:1024200047466D1817433F188742804140422D1898
:102430002B0200D5F7E634E03300002500221DE72B
:10244000C0086F070743E80837E7C7086A0717435C
:10245000194AE808934200D12FE73A00D8E0164B1A
:1024600000250BE78022120411431F2B00DDB7E08B
:1024700020220F00D21A914697406246DA40174355
:10248000B84662464F46BA40D940571EBA41474601
:102490006D1A1743C71BB842804140422D1A2B02C8
:1024A00016D47B0700D179E20F233B40042B00D0E8
:1024B000CEE63300FF08C9E7FF070000FFFF7FFFFC
:1024C00001F8FFFFFFFF7F00FE07000044460126E2
:1024D0006D026D0A002D00D00BE73800FEF784F87E
:1024E000030018301F2800DC07E73900083B99403B
:1024F000864200DD87E0831B581C1F2800DC14E2A5
:102500000A001F3BDA40202805D040231B1A9940BF
:102510004B1E99410A43002A3CD00026530700D0A5
:1025200091E6170035003300FF088FE7CA4A731C95
:1025300013427AD12B000343002E00D092E1624671
:102540000A43002B00D1F4E1002A0DD06346C718DE
:10255000874280416D1840422D182B0200D512E2AF
:102560003A00BB462A4315D05B466A07DF083A4368
:102570000023E8084CE06346C71AB84292416B1A40
:1025800052429B1A1A0200D587E03A001D001A43F6
:10259000A0D100240023002570E6B04D361A0D406E
:1025A0007B0700D080E7330084E74B462A000243D4
:1025B0007ED05A1E012B00D11FE1A94CA34200D1AD
:1025C00098E1382A00DC9CE16246571EBC459241E6
:1025D00052428D1A44461E002A0200D586E637E68E
:1025E0001A000F00203AD740B846202B05D04022D1
:1025F000D31A994063460B439A4657467B1E9F4128
:1026000043461F4346E7954A331A11404A07C80814
:1026100005035B052D0B5B0D30E680231B041D427B
:1026200000D1FBE01D000027FDE58D4A934200D15B
:1026300003E76246821882428041691840420818C6
:10264000C707520817434508520700D4AEE10F22CE
:102650001E003A40042A00D0FAE5FF086A073A4310
:102660000009D5E763464F07DA081743C80824E690
:10267000471EB842804140422D1A1E002A0200D552
:1026800034E6E5E5002B00D00DE1002A00D069E139
:1026900080250024724B2D03F0E563461F1ABC45CC
:1026A0009241012443464D1B5242AD1A1C4011E792
:1026B000624644460D00D708C8E66346C6188642FF
:1026C00080416918404209180B0200D40CE1634BA9
:1026D00070081940CB0703434A08400700D43BE188
:1026E0000F201840042800D136E11F1D9F42AD4144
:1026F0006D420223AD18FF08A8E6002B00D140E68A
:102700004B469B1B002E00D150E7382B2EDD634635
:102710005F1EBC45924152428D1A44464E462B02E2
:1027200000D5E3E594E56346C71AB84280416D1AC7
:1027300040422D1A2B0200D5C9E66A07FF08012383
:102740003A43E80864E71A000F00203AD740B84639
:10275000202B05D04022D31A994063460B439A465A
:1027600057467B1E9F4143461F435CE680223C0048
:10277000120415431F2B26DC20222F00D21A06003C
:1027800090409740DE40421E9041DD403743074372
:10279000491B6346DF1BBC45924152424E468D1A8F
:1027A0007DE6002B00D1C1E64B469B1B002E00D1DD
:1027B000D0E5382B36DD80252D04294200D1DDE01F
:1027C0004E4600272FE51A002E00203AD640202B37
:1027D00005D04022D31A9D402F000743BB465F46D9
:1027E0007B1E9F413743D4E7002A00D1D1E6012464
:1027F00043460D00E3461C40B6E663461F1ABC453F
:1028000092414D1B5242AD1A2B0200D55EE66A077B
:10281000FF08444601233A43E808F9E6471C17E558
:102820003B00EBE58022120415431F2B6CDC2022B9
:102830002F00D21A060090409740DE40421E904181
:10284000DD40374307434919674467459241524287
:102850004E465518ECE5C046FE070000FFFF7FFF1F
:10286000FF070000002B00D1FCE6C7086B071F43E1
:102870006346E8080B4300D11FE580231B03184281
:1028800007D0CA081A4204D163461000DF0849077E
:102890000F437B0FFF00FF085B071F430DE56246F8
:1028A0000D00D708D2E5C7086B071F43E808002AC8
:1028B00000D102E580231B031842EAD0CA081A425D
:1028C000E7D163460124DF084346490710000F4360
:1028D0001C40DEE760446045924169185242891805
:1028E00006000B0200D5F2E64A07F6080123324340
:1028F000C8088DE66346DF084B0744461F43C808F7
:10290000DBE44446130035E71A002E00203AD64097
:10291000202B05D04022D31A9D402F000743BB46F1
:102920005F467B1E9F4137438EE7202300271B1AFB
:10293000F5E40023002A00D192E567460D00FF0868
:1029400084E53A001A4300D123E61D00BB460BE69E
:1029500017003300FF0879E5DB0852071A4308091E
:10296000022355E663460124DA0843464F0717431E
:10297000C8081C40A1E41E00471C69E467460D001E
:102980004E46013764E40F4BFF081D406A076D0295
:1029900001233A432D0B71E4130046E73300FF088F
:1029A00054E567460D001E00013751E46A07FF0831
:1029B0003A4300092CE6C0086A0702430023E808EE
:1029C00026E6C046FFFF7FFFF0B5C6461E03360B66
:1029D000B0460D4E0C034D005F0000B5240B6D0D8D
:1029E0007F0DB5420BD0084900208F4204D14646E6
:1029F00016433000431E984180BCB846F0BD0443E6
:102A00000120002CF8D1EEE7FF0700000B000200C8
:102A100070B5164D0C0382B049000020009201935E
:102A2000240B490DDE0FA94204DD1148814203DD6C
:102A3000104BF01802B070BD8020400320430E4CB4
:102A4000641A1F2C08DD0D4B5B1AD8400300584256
:102A5000002EEFD11800EDE7094B009A9C460300C9
:102A600061448B40E2401343F1E7C046FE0300009F
:102A70001D040000FFFFFF7F33040000130400006B
:102A8000EDFBFFFF70B5002816D0C317C5185D40D9
:102A9000C40F2800FDF7A8FD104B1B1A5B055B0D4A
:102AA0000A2814DC02002E00153296400B22121A5E
:102AB000D5402D032D0B03E0002400230025002624
:102AC0001B052B43E40723433000190070BD0B386E
:102AD00085402D0300262D0BF2E7C0461E040000A2
:102AE00010B5041E10D0FDF77FFD0E4B1B1A5B05C1
:102AF0005B0D0A280FDC0B222100121AD140153081
:102B00000A038440120B01E0002300221B0513433B
:102B10002000190010BD22000B388240120300244F
:102B2000120BF3E71E04000070B542024300C40F0D
:102B3000FE201B0E591C550A08420CD0E0218900CA
:102B40008C466D07120B63441B051343E4072343B4
:102B50002800190070BD002B14D1002D1BD02800B7
:102B6000FDF742FD0A281CDC0B232A001B1ADA4061
:102B7000030015339D400E4B12031B1A5B05120B0D
:102B80005B0DE1E7002D09D0130B802212031A43DD
:102B90006D07084BD8E700230022D5E70022054B3C
:102BA000D2E703002A000B3B9A400025E3E7C0462A
:102BB00089030000FF07000010B5002903D1FDF7CD
:102BC00013FD203002E00800FDF70EFD10BDC046E9
:102BD000F0B58023A1B06946374D5B0002000B8041
:102BE0002800012101F02CFA01F062FA280001F01E
:102BF000ADF9040001F05CFA002C02D0012021B0F4
:102C0000F0BD21000A2201A826F0E2FC48226B4612
:102C100001279B1804AE2900347001A81F7000F032
:102C200054FC01F045FA2A000221300001F0C8F8F6
:102C300001F03EFA2A003900042000F0F8FC0400FC
:102C400001F036FA002C1BD11C4B4E2205931223A7
:102C50006B44DC871A4B2900B3876B469B181F70A7
:102C60006B4601A81F81019700F0C5FB01F020FA17
:102C70002A000221300000F065FF040001F018FA7C
:102C8000200001F015FA002CB8D12A000221684674
:102C900000F05CFC070001F00BFA002FAED12A0017
:102CA00001213000347001F08BF801F001FA054881
:102CB00026F08EFB2000A2E7800100200602010022
:102CC00006020000A0B906107FB5254DB821286086
:102CD000244826F00DFB64230322B821286804F061
:102CE00031FE002806D0204826F072FB0124200087
:102CF00004B070BD1D4826F06BFB05266A461C4BD0
:102D0000B821938100960223286803AA04F0FEF9F3
:102D1000041E08D02100174826F0EAFA21001648C0
:102D200026F0E6FAE3E76A46144BB8219381009651
:102D30000223286803AA04F0E9F9041EEED16A46CA
:102D40000F4BB821938100960223286803AA04F050
:102D5000DDF9041EE2D10B4826F03AFBC7E7C04676
:102D6000F00100203FBA061075BA06109BBA061093
:102D7000101C0000CABA061027BB06101150000034
:102D800012040000FFBA0610F0B50125052785B032
:102D9000124E02970195009004002B002822B821C2
:102DA000306804F05DFC002815D163190093029788
:102DB00001952B002922B821306804F051FC00282D
:102DC00009D102340297019500942B002A22B821E0
:102DD000306804F045FC05B0F0BDC046F0010020AD
:102DE000F7B5134E3368002B0DD0124C124D2378DB
:102DF000012B0AD103F080FC2B68C31A0220642B3C
:102E000002D9032323700120FEBD0127277003F0A0
:102E100073FC28600325094B0195009328223B0091
:102E2000B821306804F0FAFC0028EDD02570EAE7FC
:102E3000F0010020EC010020E8010020ED0100205D
:102E40000C4B020019780220012905D019780329BA
:102E500003D100221A700120704719780229FAD193
:102E600005490878107048785070002089781870EB
:102E70009170F1E7EC010020ED010020054B1B688B
:102E8000834205D1044B1A78012A01D101321A700C
:102E90007047C046F0010020EC010020054B1B6884
:102EA000834205D1044B1A78012A01D102321A70EB
:102EB0007047C046F0010020EC01002010B5002052
:102EC0000DF0DAFE08F068FB002801D002F070F97E
:102ED00008F0FCF908F0D2FA09F074FB00200DF0BC
:102EE000CCFE002010BD012010B540420DF00CFFBB
:102EF00010BD704770470000802337B51B01994211
:102F000020D16A460023941D01AD21002800D38002
:102F10002B8002F0CDFD2A880B4B110A1A702288F3
:102F200059700A4B110A2020597001211A700DF0B6
:102F3000A7FE0748FFF728FF002803D101214030F2
:102F40000DF09EFE37BDC046F9010020F7010020BC
:102F5000F401002010B5002812D004788C4204D26D
:102F6000017001211C7A214319720178914201D824
:102F7000002010BD02700222197A0A431A72F7E784
:102F800001204042F5E700280AD0836B002B07D0D0
:102F9000C36B002B04D0006C434258414042704741
:102FA0000120FBE7F0B50500A1B018000E001700E6
:102FB0001C00FFF7E8FF00282ED1002E2CD0637AEA
:102FC000002B01D180331D43A36BE27A9C466946F6
:102FD00028006368D2196546A8472200A0724732CC
:102FE00012780220236C6168012A01D1E12040009F
:102FF00098470A2000232056984208D002204042D9
:1030000008E01900E27A69448A5CF25401339AB20A
:10301000BA42F6D321B0F0BD0120F0E713B56A46FD
:10302000D41D0300012221001B20FFF7BBFF002855
:1030300007D12378DB065B0F5A1E022A01D8043819
:10304000C01A16BD73B5040008000E00FFF79BFF01
:10305000002817D101AD288033000222290040301A
:10306000FFF7A0FF00280CD12B786A78D909A1704E
:103070005906490F61700F210B4023700323134041
:10308000E37076BD01204042FBE773B50400080001
:103090000E00FFF778FF00281ED101AD2880330015
:1030A000022229004230FFF77DFF002813D16A7801
:1030B0002B780125D909A1709911294061719906D0
:1030C000890F61700F210B402370D3102B40E370E8
:1030D00007231A40227176BD01204042FBE70023FE
:1030E000F7B501AE04000D00338002220B004B2027
:1030F0003100FFF757FF002817D132787378520854
:10310000E2710122032799111140A1709910DE0983
:1031100039403B406670E1702371002E05D12100DB
:103120002B0008314D30FFF73DFFFEBDF7B507001E
:1031300018000D0016001C00FFF725FF00284AD1DB
:10314000002D48D0637A002B01D17F331F4023002C
:1031500047331B78012B2ED1731901930095019BE6
:10316000009A9A4216D0009B781BC018E36B01228C
:103170001E0000996368C0B2B047A072E120236CC2
:10318000616840009847009B013300930A23E3568F
:10319000002BE4D07C2F08D12978012308002200DD
:1031A00018404732194214D013700A2020560028C4
:1031B00013D0022010E0E36B32009C4629006368C4
:1031C00038006646B047236CA072616802209847B9
:1031D000E0E71070E9E701204042FEBD73B504004E
:1031E000160008001D0001A9002C12D0C3061B0FF9
:1031F00040090B7048702B0002225B20FFF796FFFE
:10320000002805D12B00320021005E30FFF78EFF31
:1032100076BD01204042FBE773B56B46DC1D002301
:1032200005000E00237001220B0059202100FFF73A
:10323000B9FE002809D101222378210093431D43C0
:10324000593033002570FFF771FF76BDF0B50D00E2
:10325000002185B004002B00012203AF461C023080
:103260003980FFF777FE011E03D00120404205B0F0
:10327000F0BDA3780093012B34D12B000322300042
:10328000FFF768FE061EF0D1E31C01930C222B0011
:1032900001212000FFF75EFE0028E6D103222B006B
:1032A0003100A018FFF756FE0028DED170220F2152
:1032B000637840301B011340009AD20113432278F7
:1032C0000A40134303223B70E378390013407B70BC
:1032D000013A2B00FFF72AFF0028C8D12800FFF78A
:1032E0009DFEC4E72B000722C9E773B50D0000213E
:1032F00004002B00012201AE02303180FFF72AFECC
:10330000011E02D00120404276BD2B000322601C2A
:10331000FFF720FE011EF5D12B000122601DFFF7F3
:1033200019FE0028EED106212B000D222000FFF708
:1033300011FE011EE6D12B000122E01CFFF70AFE60
:10334000011EDFD12B000422201DFFF703FE002801
:10335000D8D1402330216279423092011A406378FB
:103360001B010B401A43A3782139DB011A43237850
:103370000B401A4332700822E3780839DB0013400F
:1033800022790A401343737002222B003100FFF7A9
:10339000CDFE0028B8D12800FFF740FEB4E7F7B50E
:1033A0006B46DD1D0023060008000C002B70FFF7A4
:1033B000EAFD00281AD12300012229007C30FFF702
:1033C000F1FD002811D101272B783E40BB431E435D
:1033D0003A00230029007C302E70FFF7A7FE00285A
:1033E00007D12B7847343B402370FEBD012040427B
:1033F000FBE70D20FBE7F7B50E0001AD040003224B
:103400000021280026F0E4F83000FFF7BCFD00287A
:1034100056D1002C54D027787B1E022B53D8330072
:10342000032229005330FFF7BDFD00282BD10221D4
:103430003B008B43012B27D00221A3796A785B00E4
:103440008A430B401343E279491892000A408B43A8
:103450001343227A0431D2000A408B431343627A29
:10346000083112018B430A4013436B7001216378CA
:10347000AA780B408A431343AB7003223300290020
:103480005320FFF753FEFEBDA3782A785B008A43E2
:103490000B4004211343E2788B4392000A4013430C
:1034A00022794918D2000A408B43134362790831CC
:1034B00012018B430A4013432B70012FD6D0BBE778
:1034C00001204042DFE70C20FBE7F7B504000800CD
:1034D0000F00FFF758FD002835D1002C33D001AE86
:1034E0003080B0703B000322310053302578FFF765
:1034F00059FD002826D102222F007378B178974316
:10350000012F0CD1327856103E40A67096103E40E6
:10351000E670D61012113E403A4026716271023DAB
:10352000012D0CD801225D101540A5719D1015408C
:10353000E571DD101B1115401340257263720123E4
:1035400019406170FEBD01204042FBE7F7B5050060
:10355000100017000C00FFF716FD021E4ED1002DC3
:103560004CD029190600040002202B0084460125B6
:103570008B422BD1002A44D16B46DD1D2A703B00C3
:1035800029007D200132FFF70DFD002835D1E3072A
:1035900003D504232A7813432B7002231C4202D044
:1035A0002A7813432B70630703D501232A7813432A
:1035B0002B70F3071FD508232A7813432B703B0089
:1035C000012229007D20FFF7B1FD16E018780228BE
:1035D0000DD003D8002807D12C4303E0202808D0C1
:1035E000082252420133C3E760460443FAE704204D
:1035F000FBE72E43F6E73443E1D1FEBD0120404214
:10360000FBE70820FBE770B5040008000D00FFF79A
:10361000BAFC002808D1002C06D02B000122210082
:103620000330FFF7BFFC70BD01204042FBE7F7B558
:103630006B46DE1D002304000D00170033703100BF
:10364000130058200122FFF7ADFC002818D1032DEC
:103650001BD82301DBB21A0031780A43022D08D0AF
:10366000032D0ED022000A43012D02D00A0023436D
:103670009A4332703B00012231005820FFF756FD7B
:10368000FEBD0C4323431A00F3E70C204042F7E74A
:1036900070B5050008000C00FFF775FC00280CD180
:1036A000002D0AD0236C6168054898472300012249
:1036B00029002120FFF776FC70BD01204042FBE786
:1036C000204E00000023F0B585B002AA0500D3719A
:1036D000FFF759FC002800D083E02B004A331B88F9
:1036E0000193002B00D17CE0EE89F30702D5013E67
:1036F000B6B2EE81012E01D80226EE81290000200B
:10370000FFF74DFE041E1CD12900FFF785FD041EA6
:1037100017D131000198FCF72DFECEB28BB2002EEE
:1037200012D168692B0031008019EA89FFF756FD34
:10373000EB890400F618019BB6B2B34232D90028D7
:10374000EFD0200005B0F0BD2700DEB2019B9E1B2C
:10375000B6B2BE420DD9002CF3D168692B003900F6
:10376000C019EA89FFF73AFDEB890400FF18BFB2E0
:10377000EFE7002CE5D10223EF89EB81019BB342F7
:103780000FD9002C01D0EF81DBE768692B003100F5
:103790008019EA89FFF722FDEB890400F618B6B21A
:1037A000ECE7EF81002CCCD129000120FFF734FD9C
:1037B000041EC6D129000120FFF7F1FD041EC0D16F
:1037C00002ABD81D2900FFF763FF0F2202ABDB79A4
:1037D000040013402B740028B3D1012BB1D009246D
:1037E00000E001246442ACE737B5B6236A46937122
:1037F00000230500D371FFF7C6FB00282AD16946D4
:1038000001222B0006317E30FFF790FC0400FA20E5
:103810002B6C6968C00098472B00012247331A704F
:10382000002C07D16B7A002B06D02800FFF74AFF47
:10383000041E0AD020003EBD694620002B0007313F
:10384000FFF7B0FB041EF5D1EFE7002200232A6347
:103850006B63EFE701246442ECE7000037B56B4689
:10386000DD1D002304002B70FFF78DFB002829D1FC
:103870002300012247331A70607A002808D0230001
:10388000012229000020FFF78DFB002807D03EBD54
:1038900023002900FFF786FB0028F8D1EFE72B78FB
:1038A00022789A420AD1102323730F3BE376064B0A
:1038B000A085A3622000FFF797FFE8E703202370AD
:1038C0004042E4E70120FBE700010200F0B585B0CB
:1038D000029102ABD91D029B14000870002B40D04E
:1038E000002A3ED0127EC3B29A423DD92300012263
:1038F0002F20FFF71BFC002824D1E3890F2B29D8A8
:10390000DA0701D5013BE381002630271025019617
:10391000029B0199E28959182300954214D338007B
:10392000FFF740FBA37B019ADF199A18D2B20192EC
:10393000FFB29E191023F6B29D1BEDB2002801D1F3
:10394000002DE5D105B0F0BD2A003800FFF72AFBB5
:10395000AE19EFE72300102202993020FFF722FB77
:10396000F0E701204042EDE70A20FBE7F0B585B023
:103970000F00102204000021684625F029FE0322D2
:103980006D4600239446BE7EDAB2B24202D30820CE
:1039900040420FE061465943786A01334218415C66
:1039A0000929F1D19678507829003A00FFF78EFF67
:1039B000002801D005B0F0BDAB5D01211A000A401E
:1039C00022705A100A4062709A109B060A405B0FE0
:1039D000A270E370EEE7F0B505008BB010000F00A9
:1039E0001600FFF7D0FA041E00D070E0002D00D1C1
:1039F0006DE0330047331B783F010193EB190393CC
:103A0000039B9D4202D120000BB0F0BD2B78032B0D
:103A100007D9019B012B04D131000020FFF7BFFC27
:103A20000400002C4AD12B78092B49D0292B02D035
:103A300008246442E7E71022210006A825F0C8FD0B
:103A4000330048331B889B061AD4B37E03279C4659
:103A50002300DAB29445EBD939005943706A013337
:103A60004218415C2929F4D1937806AF029350782B
:103A700039003200FFF72AFF002810D00400C2E707
:103A800004ABDF1D0122330039001E20FFF78AFA44
:103A90000028F3D13B785A0607D5803B05E0029B0E
:103AA000FA5C7F2313405206F7D4AB80019B012BB5
:103AB00004D131000198FFF772FC040010359FE734
:103AC0003100281DFFF752FF0028EFD0D6E7012470
:103AD000AFE7030030B548331B88040085B09B076F
:103AE00012D5FFF750FA002811D16D462923220084
:103AF000012168462B70FFF76EFF002802D1AB88CA
:103B00000634E38705B030BD08204042FAE70120C3
:103B1000FBE7F8B50C00032100238C46577ED9B291
:103B20008F4201D800200BE065465D43166A0133E1
:103B30007119755DA542F2D1032225F0F2FD012035
:103B4000F8BD0000F0B506008BB010000C001500A9
:103B5000FFF719FA002800D02EE1002E00D12BE14A
:103B60002B0047331B78019338236343F3180393E7
:103B7000039B9E4205D1019B012B00D116E100243D
:103B800013E0019B012B0AD03078092800D9DCE032
:103B9000FCF74CFB0E1419DBDBDBDBDBDBC729009E
:103BA0000020FFF7FCFB041EEED020000BB0F0BDA0
:103BB0002900301DFFF74AFB04009EE02900301D5C
:103BC000FFF793FBF8E730002B000B2201210930AF
:103BD000FFF7C0F9002800D0EEE006AF2B0001226D
:103BE00039006B30FFF7DEF9041EDED12021337976
:103BF0003A785B018A430B4013433B7001222B0050
:103C000039006B20FFF792FA041ECED104AB187175
:103C100038802B00022239004B30FFF7C3F9041E15
:103C2000C3D101223B7840211340F27A153452006F
:103C300013437F223B707B7813407279D201134388
:103C4000B2798B4392010A401343F27934399200DE
:103C50000A408B431343327A09398B430A4013439A
:103C60007B700427290005A8FFF7CDFC04AB1B7966
:103C70003B400343DBB2002B49D12B0006A90222B3
:103C80004B20FFF753FA0400FA202B6C6968800080
:103C90009847002C00D088E77379002B32D131008F
:103CA0002B00EC760C3101224D20FFF73FFA040087
:103CB000FA202B6C696880009847002C00D074E7CC
:103CC00006AF2B00012239004420FFF76BF9041ED8
:103CD00000D06AE70F21B37A727A1B010A401343BE
:103CE00039003B7001222B004420FFF71FFA04002B
:103CF000FA202B6C6968800098473836002C00D178
:103D000036E752E70123EB76F3792B77D8E7013CCE
:103D10002B6C69682948E4B29847002CA2D10F2483
:103D200014E006AF10220021380025F051FC0023DA
:103D300005AC2A002380A37009212000FFF7E9FECB
:103D4000A27863780292002802D1082464422CE70A
:103D50002A0039001800FFF7B9FD041E00D024E73F
:103D6000029BB1885B0858003A5A4905D20A490DAE
:103D7000D2020A433A52581C40003A5AF188D20AF9
:103D80004905490DD2020A4302333A525B00FA5AFE
:103D90003189D20A4905490DD2020A43FA52390043
:103DA0002B0010223020FFF7C1F905E72900019808
:103DB000FFF7F5FA0400F8E60124C7E71027000032
:103DC000F0B5040089B010000E001500FFF7DBF815
:103DD000002800D0A8E0002C00D1A5E02B0047333C
:103DE0001B78009338237343E3180193019BA3428C
:103DF00004D1009B012B64D0002017E02378032B13
:103E00000BD8022B62D02078092857D8FCF70EFA7D
:103E10001017615656565656561C009B012BF2D170
:103E200029000020FFF7BBFA0028ECD009B0F0BD54
:103E30002900201DFFF706F9002873D0F6E72900B6
:103E4000201DFFF722F9F7E704AF10220021380008
:103E500025F0BEFB002303AE30002A000921338089
:103E6000B370FFF756FE7378B678002826D02A0084
:103E700039001800FFF72AFD0028D7D1731CDBB2E8
:103E8000FA5CBB5D120213435B055B0DA380F31C60
:103E9000DBB2FA5CB31CDBB2FB5C120213435B05C2
:103EA0005B0DE380731DDBB20436FA5CF6B2BB5DDA
:103EB000120213435B055B0D238133E0082040426F
:103EC000B4E729000098FFF76AFAAFE7009B012BDF
:103ED000A6D02800FFF757F8002825D104AE2B0004
:103EE000012231006B30FFF75DF800289ED10127D9
:103EF000337829005B113B402371201DFFF7EFF859
:103F0000002800D092E72B003A0031004430FFF740
:103F100049F8002800D089E733781A09A2720F22E5
:103F200013406372383461E70120C8E700280AD0E3
:103F3000836B002B07D0C36B002B04D0006C434273
:103F40005841404270470120FBE7000010B50400D3
:103F5000FFF7ECFF002823D124232370124BA36426
:103F6000637A5A425341E3726369002B01D10F4BCC
:103F700063612000FFF772FC002810D10C4B08226F
:103F800023620C4B200063620B4B23830723A37631
:103F90000A4BE365230060331A70FFF79AFD10BDEA
:103FA00001204042FBE7C0460300002061320710B9
:103FB0002E32071019320710081100003C1400209F
:103FC00030B504000D001978642385B092B20293D5
:103FD0000192490022000095633B034803F040FB37
:103FE00040B205B030BDC0468004002030B50400AA
:103FF0000D001978642385B092B2029301924900B2
:1040000022000095633B034803F050FA40B205B02C
:1040100030BDC0468004002007B5FA2189008842DF
:1040200004D3FCF721F902F073FB07BD8000019077
:10403000019B5A1E0192002BF7D0C046F8E7000002
:10404000F8B5041E24D0144F144E154D012910D17B
:10405000144A68238263144A3B70C2632022C281DF
:1040600000224172066442616A702B704560002034
:10407000F8BD002902D10D4825F0AAF93A780023AD
:104080002A702E226B7065602664E2816361EEE720
:1040900001204042ECE7C046FD0100201940041019
:1040A000FB010020C13F0410ED3F041058BB061077
:1040B0000100223010B5242800D977E0FCF7B6F8CB
:1040C00073706D766A76766764615E5B5855524FA1
:1040D0004C49284643402B763D3A253734312E2231
:1040E0001F1B171318000121314825F001F910BDDD
:1040F00002213048F9E701212F484942F5E7022122
:104100002E48FAE703212E48F7E708212D48F4E767
:1041100010212D48F1E70C212C48EEE704212C4812
:10412000EBE705212B48E8E706212B48E5E70721C7
:104130002A48E2E709212A48DFE70A212948DCE783
:104140000D212948D9E70E212848D6E70F21284814
:10415000D3E711212748D0E712212748CDE71321C3
:104160002648CAE714212648C7E715212548C4E791
:1041700016212548C1E717212448BEE71821244805
:10418000BBE719212348B8E71A212348B5E71B21CB
:104190002248B2E71E212248AFE720212148ACE7A0
:1041A00021212148A9E722212048A6E720489CE7B1
:1041B00067BB061083BB0610A6BB061037BC0610F3
:1041C000C4BC061021BD061099BD061007BE06101E
:1041D00086BE06104EBF06100EC00610CAC00610DE
:1041E000A1C106101AC2061096C2061007C3061017
:1041F00080C30610F2C3061077C40610E4C406108C
:104200004EC50610A1C50610F7C5061038C6061023
:10421000B7C6061032C7061096C70610FFC70610AD
:1042200050C80610CBC806103AC90610C7C90610F8
:1042300031CA0610F0B51D0089B0284B039206AABA
:10424000138000231C001E009070D17015715371F3
:10425000D118897801337618F6B2A419E4B2042B88
:10426000F6D1002D0CD0039B002B09D01900E818C3
:104270000B780131F618F6B23419E4B28842F7D15E
:10428000FA23174F9B00009384210623386802F01D
:104290003DFF002802D0012009B0F0BD002D0ED155
:1042A000FA2305AA9B001670547000938421022300
:1042B000386802F02BFF431E9841C0B2ECE7039B25
:1042C000002BEDD0FA239B00009384212B00039A4E
:1042D000386802F01BFF0028E2D0DCE7B56200007E
:1042E0007C04002010B50E4825F072F88021902043
:1042F00000228900C00502F0AEFC642002F008FA3A
:104300008021902001228900C00502F0A4FCFA203F
:10431000400002F0FDF9034825F05AF8002010BDD6
:1043200053CA06107CCA0610FA2330B59B0087B02A
:1043300002930223040005AD084801930095FD2275
:1043400084210068013B03F08BF9002804D12B88FD
:104350005BBA238007B030BD0120FBE77C0400205E
:1043600007B501236A4653800023938006331080EB
:1043700008211800FFF75EFF0EBD00001FB5C02327
:104380009B000193064B6A46029300238A21137314
:104390000620093301AAFFF74DFF05B000BDC04656
:1043A00002007210F0B516260024FA2787B06E447A
:1043B0003480BF003000FFF7B7FF00281FD13388DB
:1043C000002B1CD01D1C802B00D980250E4B0F48C4
:1043D000ADB20093029701950123FF22842100686A
:1043E00003F03EF900280AD180232C19A4B21B0146
:1043F0009C42DFD32100064824F07AFF01E0002C24
:10440000F8D107B0F0BDC046320300207C04002084
:10441000A0CA061010B5264C2060264824F0D8FF0C
:10442000802101228900244802F015FC234824F051
:10443000CFFFFFF757FFFA230322842120689B0058
:1044400003F080FA002813D0FA20400002F060F94F
:10445000FA230322842120689B0003F073FA0028CA
:1044600006D04221164824F043FF0124200010BD4D
:104470004221144824F03CFFFFF780FF00280ED0B3
:10448000114824F0A5FFFFF78DFFFA208000FFF709
:1044900067FF041E05D00D4824F09AFFE5E70C489D
:1044A000EFE70C4824F094FF0B4824F091FFDDE780
:1044B0007C040020D7CA06100000104803CB061069
:1044C00023CB06105CCB06108FCB0610F6CB061064
:1044D000C3CB06101CCC06103FCC0610134B70B596
:1044E0001B68002B12D0124C124E2378002B0FD0D9
:1044F0002378022B0CD802F0FFF8FA2233689200DE
:10450000C31A0220934202D904232370012070BDF4
:104510000125257002F0F0F8002330601A00072111
:104520002800FFF787FE0028F1D0EDE77C0400208B
:10453000B8030020B4030020F0B58B4C87B023787B
:10454000DDB2012B33D102F0D7F8884B1E68861BF1
:10455000C72E03D80225280007B0F0BD1627002378
:104560006F4438003B80FFF7DFFE00281AD13A88FD
:10457000632A17D902232370131CC02A00D9C02331
:104580007B499AB20B807B4B7B4801920093FF22C0
:1045900001238421006803F041F90028DAD00423C4
:1045A0002370D8E7FA239B009E42D3D9F7E72378FC
:1045B000DDB2022BCFD02378042B03D1002323704C
:1045C0000125C8E72378032BFAD1694E00213388EF
:1045D000492B02D933884A3B99B20023654DEA5CE6
:1045E000B52A00D09DE05A1CAA5C622A00D098E04F
:1045F0009A1CAF5CDA1CAA5CD2B2012F00D090E00A
:10460000072A00D08DE006335B195A791979120216
:104610000A4302849979C21CD177D979021DD177D6
:10462000197A421DD177597A821DD177997AC21DA4
:10463000D177D97A0132D1771A7D00250270DA7DDF
:1046400042705A7E197E12020A43997E0904114370
:10465000DA7E12060A4382605A7F197F12020A43E9
:10466000997F09041143DA7F12060A4342605A1DFA
:10467000D17F9A1DD27F12020A43D91DC97F090436
:1046800011431A000832D27F257012060A43C26015
:104690001A00283211780132127812020A431900E6
:1046A0002A310978090411431A002B3212781206B4
:1046B0000A4302611A002C32117801321278120278
:1046C0000A4319002E310978090411431A002F32C8
:1046D000127812060A4342611A003C321178013204
:1046E000127812020A4319003E3109780904114375
:1046F0001A003F32127812060A43190082611A002A
:104700004131097840321278090211431A004232CD
:10471000127843331B7812040A431B061343C36108
:1047200019E701339BB2994200D358E7134B1F8816
:104730000137BFB21F80012F07D01E213800FBF7C1
:1047400019FE89B2002900D038E731882B786A78C1
:10475000AE78ED7889B20092DBB23A00029501960C
:10476000074824F0C5FD29E7B8030020B403002062
:10477000B2030020B90300207C0400203003002095
:1047800063CC0610054B1B68834205D1044B1A7895
:10479000022A01D101321A707047C0467C04002001
:1047A000B8030020054B1B68834205D1044B1A78DF
:1047B000022A01D102321A707047C0467C040020E0
:1047C000B8030020F0B589B01422002103A824F01A
:1047D000FFFE082180279020604BBF001A6DC005A6
:1047E0000A431A651A6D00240A400292029A1A6D51
:1047F00004390A431A651B6D01220B4001933900ED
:10480000019B02F028FA902000221021C00502F03E
:1048100022FA01223900524802F01DFA90200125A7
:10482000022603AB1900C00506960397049505946C
:1048300002F076F99020102303AA1100C00503931B
:1048400004950594069402F06BF903AA11004448FC
:10485000069603970495059402F062F980231B01E4
:1048600003939020802303AA11005B02C0050493E8
:104870000594822602F054F98023902003AAF603BF
:104880005B011100C00503930496059402F048F9FA
:1048900003AA1100324804960395059402F040F9EA
:1048A0001023039303AB19002D480496059402F0DE
:1048B00037F92023039303AB190029480496059484
:1048C00002F02EF94023039303AB19002448049609
:1048D000059402F025F98023039303AB19002048C7
:1048E0000496059402F01CF980235B00039303AB4C
:1048F00019001B480496059402F012F90421902037
:10490000052302260391C00503A907930496059584
:10491000069402F005F984212000890003F0A2FF2B
:1049200084212000890003F0B1FF3900280003F042
:1049300099FF3900280003F0A9FF0421200003F0AB
:1049400077FF0CF09BF9220029000F2001F0F2FE06
:104950000F2001F019FF09B0F0BDC046000040482B
:1049600000001048054B82B01A6D02431A651B6D9A
:1049700018400190019B02B07047C04600004048BB
:10498000822310B5124CDB052360124B01226360B9
:1049900000232000A360E26023616361A361E361FF
:1049A000236202F055FB002801D000F001FC002139
:1049B000200003F097FE002801D000F0F9FB002151
:1049C000200003F0B5FE002801D000F0F1FB10BD7F
:1049D000D40400205B3D300010B5134B134C012272
:1049E0002360134B200063600023E260A360236117
:1049F0006361A361E361236202F02AFB002801D016
:104A000000F0D6FB0021200003F06CFE002801D04E
:104A100000F0CEFB0021200003F08AFE002801D028
:104A200000F0C6FB10BDC04600100041800400200D
:104A30009129700070B5050088B01422002103A8E8
:104A400024F0C6FD82222B68D205934268D104204F
:104A5000FFF788FF902000260324122303A9C00536
:104A60000493039406940596079602F059F82100E2
:104A7000300003F0F7FE2100300003F007FF802133
:104A8000594B89039A6D01200A439A659B6D0B402F
:104A90000193019BFFF766FF544C554B20002360A8
:104AA000092363600733A3607033236180239B0174
:104AB000E6606661A661E661236201F08BFEB042AA
:104AC00001D000F075FB4B4BAC63A5624A4C8022D1
:104AD0002360082363600023A360E3606361A36134
:104AE000E361C02320009B012261236201F072FE7A
:104AF000002801D000F05CFB002201211120EC63B2
:104B0000A56201F017FE112001F03EFE00220320F5
:104B1000110001F00FFE032001F036FE08B070BD59
:104B2000364A9342FAD10420FFF71CFFC024122317
:104B300090200026E401049303A90F3BC0050693CF
:104B400003940596079601F0EBFF2100300003F077
:104B500089FE2100300003F099FE8021224B0904D8
:104B60009A6D01200A439A659B6D0B400293029B4C
:104B7000FFF7F8FE224C234B200023600B236360D9
:104B80000533A3607033236180239B01E660666177
:104B9000A661E661236201F01DFEB04201D000F083
:104BA00007FB194BAC63A562184C802223600A23D3
:104BB00063600023A360E3606361A361E361C023DA
:104BC00020009B012261236201F004FE002801D035
:104BD00000F0EEFA002204201100EC63A56201F05F
:104BE000A9FD042098E7C04600004048E4020020E8
:104BF000080070481C007048980200200010004116
:104C00004C02002030007048440070480002002030
:104C100010B5154B154C5A78197812020A4312B286
:104C20002280DA78997812020A4312B262805A79A5
:104C3000197912020A4312B2A280DA799979120222
:104C40000A4312B2E2805A7A197A12020A4312B265
:104C500022819A7ADB7A1B0213431BB2638101F033
:104C60004BFD606110BDC0463705002044050020A3
:104C700010B50C4A0C4C537811781B020B435BBAED
:104C8000A381D37891781B020B435BBAE3815379FC
:104C900011791B020B435BBA238201F02DFD606189
:104CA00010BDC046310500204405002010B5002489
:104CB0000E4824F08DFB0E4B21001C700D4B18226A
:104CC0000D481C6024F084FC21000C220B4824F0C9
:104CD0007FFC210006220A4824F07AFC0122094BBD
:104CE00009481A7024F074FB200010BDBFCC0610D8
:104CF000300500202C050020440500203705002049
:104D00003105002028050020E9CC0610012310B54C
:104D1000002806D072B61822034924F002FD62B6BC
:104D20000023180010BDC046440500201FB51E4BCF
:104D30001B78002B20D001F0DFFC1C4A1368C31A3B
:104D4000632B19D91A4C10602378012B15D0032B33
:104D500024D0002B25D10C2264330293154BD02193
:104D6000009315480123019202F07AFC002803D138
:104D7000FFF74EFF012323701FBD642202925E3AAB
:104D800001920E4AF02100920B48122202F068FCB8
:104D9000002806D1FFF76CFF0223ECE7084824F057
:104DA00017FB0023E7E7C046280500202C0500205C
:104DB0003005002037050020800400203105002048
:104DC0000CCD061070B5114D11486A78297824F081
:104DD0008FFA90200F4C2B78002223706B781021D3
:104DE000C005637001F037FF3223022221000A4818
:104DF00005F08EFA002802D1084824F0E9FA902044
:104E000001221021C00501F026FF70BDA50500207C
:104E100031CD061054140020300600203ACD061083
:104E200070B5144824F0D4FA012500246E000A233A
:104E300001221148B1B202F085FD002806D13200EE
:104E400029000E4824F054FA0134E4B201357F2DD4
:104E5000ECD1002C09D10A4824F0BAFA094824F010
:104E6000B7FA094824F0B4FA70BD2100074824F0CD
:104E70003FFAF6E75ECD0610800400207BCD0610D9
:104E8000AFCD0610CFCD06100BCE0610F5CD061017
:104E9000F0B5844B87B01D780593002D00D0A9E0B4
:104EA000814824F095FA814824F092FA804C200041
:104EB00000F0B0FD002800D09EE07E4824F088FA83
:104EC000012128000BF046F8012108000BF042F800
:104ED0000126794824F07CFAC82001F019FC8022D0
:104EE00023681202DA61754824F072FA3223032231
:104EF000B821200002F026FD002800D189E03223ED
:104F00000322BA21200002F01DFD002800D187E015
:104F10006B4824F05DFA6B4824F05AFA0027FFF73B
:104F20007FFF2000FDF7D0FE002800D07AE0664821
:104F300024F04EFA012102200BF00CF80123634803
:104F4000039324F045FAC82001F0E2FB200001F0B1
:104F5000ABFA5F4F002800D07FE05E4824F038FABB
:104F60000121032039700AF0F5FF5B48FFF752FA80
:104F7000002800D083E0594824F02AFA01210420B7
:104F80000AF0E8FF01235648049324F021FA642034
:104F900001F0BEFB2000FDF71BFE002800D077E0EB
:104FA000504824F015FA01234F48029324F010FAD8
:104FB000642001F0ADFB200001F06CF9002800D066
:104FC0006BE04A4824F004FA01250123059A02996E
:104FD000137047482A0024F08BF9464824F0F8F96A
:104FE000049B320001933B78310000934248039BBD
:104FF00024F07EF907B0F0BD404824F0E9F929001B
:1050000028000AF0A7FF290001200AF0A3FF2E00C4
:105010005FE75C213A484A0024F06AF9012780E7FB
:105020005D21F7E7002F0FD1364824F0D1F936483B
:1050300024F0CEF9FA20400001F06AFB2000FDF7D1
:1050400043FE002800D172E7304824F0C1F9002166
:1050500002200AF07FFF002371E72D4824F0B8F901
:10506000FA20400001F054FB200001F01DFA002856
:1050700000D172E7274824F0ABF9002171E72648F8
:1050800024F0A6F9002104200AF064FF00237AE747
:10509000224824F09DF9002386E7214824F098F95E
:1050A00093E7C0468405002028CE061043CE0610A4
:1050B0008004002087CE0610D0CE0610F6CE061053
:1050C00018CF061060CF0610D6CF061091D006106C
:1050D00099050020B8D00610D404002058D106103D
:1050E000A8D10610CDD1061021D2061055D2061037
:1050F000AAD20610D3D20610F3D206109DCE061007
:1051000097CF0610EBCF061027D006105FD0061001
:10511000E2D006101CD1061074D10610F0D1061092
:1051200079D2061010B500F02DFD10BD10B50400A9
:10513000FDF7A4FE200001F04BFA2000FFF722FB50
:1051400010BD10B5040000F02DFD2000FDF7A6FEF7
:10515000200001F04DFA2000FFF724FB10BD0000F5
:105160007FB50F4B02689A4218D1FFF7DFFD684602
:10517000FFF7CCFD002811D106226946094824F02A
:10518000D0FA06226B460848991824F0CAFA06227B
:1051900003A9064824F0C5FA0BF036F907B000BDA4
:1051A00000200040B6050020B0050020AA05002020
:1051B00010B5024824F00CF972B6FEE72BD30610A6
:1051C00000B589B01022002104A824F001FA0021C2
:1051D0000822684624F0FCF90523029380235B0231
:1051E0000393042302A8069304F05AFC011E01D085
:1051F000FFF7DEFF202300906846019304F092FD44
:105200000028F5D109B000BD7FB51022002101A80A
:1052100024F0DEF902230093802368465B010593A6
:1052200004F026FE002801D0FFF7C2FF07B000BD42
:10523000F0B59FB001F048FAFFF7C2FF0823984C81
:105240008026226D0A2513432365964B96481A68DB
:10525000964F920092081A6080221968D2050A437C
:1052600000211A6036025A6932435A610991099A3B
:10527000824241DD5A693A405A610A910A9A824251
:105280003EDD013D002DEED1FFF7BEFF8022636DB4
:10529000520013436365636D13400B930B9BFFF741
:1052A00091FAFFF76DFBFFF797FB00F0B7FC00F0FA
:1052B0003BFD00F08FFD01F071F800F065FD00F09E
:1052C00081FC00F0C7FD0122636D794813436365DB
:1052D000636D856013400C930C9B764B05610360F6
:1052E000754B43606323C3601D33836105F0F9F898
:1052F000002809D0FFF75CFF099A01320992B6E74E
:105300000A9A01320A92B9E72A0005210A2001F01F
:1053100011FA0A2001F038FA0A24684D64230122A8
:105320006749280005F0A9FB013C642001F0F0F971
:10533000002CF2D1192263490DA824F0F2F9FA23C6
:1053400018229B000DA9280005F097FB5E4824F069
:105350003FF804F087FD5D4B0100180023F0C8FF03
:105360005B4824F035F8642001F0D2F9FFF790FD96
:105370002100584A10200BF077FD574824F028F8F8
:105380002000FDF79BFD554824F022F8544824F0F6
:105390001FF8FFF78BFC002825D1524824F018F89D
:1053A000514824F015F8514824F012F8504824F0E0
:1053B0000FF8FDF798FD09F043FB041E15D14D4B86
:1053C000186001224C4B52421A8000224B4B1A604B
:1053D000944200D01AE10122494B52421A80002225
:1053E000484B1A6064E14848DBE7070045373B78E3
:1053F000002B00D1E7E0060049363378002B43D17B
:10540000424D2B68002B00D096E0414F380023F02E
:10541000DFFF404823F0DCFF3178002905D023006E
:1054200050331A783C4823F063FF380023F0D0FF54
:10543000A67CE37B227C617C0396267B3748029620
:10544000667B0196A47B009423F052FF09F0E6FAF4
:10545000334B02003349984200D03349334823F09C
:1054600047FF334823F0B4FF0022110010000BF077
:10547000C0FD304B0100180023F03AFF01F03CF969
:1054800000280AD0286094E701F036F9E36CC01ACE
:10549000FA23DB0098428CD3B2E701232B6088E724
:1054A00000004048000010484FC30000FF7FFFFF8E
:1054B000BC05002000200040FF7C00009C0600206E
:1054C000A1D3061079DA0610A3D30610C1D30610B3
:1054D000D8D30610C54D041005D4061025D40610E7
:1054E00042D4061060D406108AD40610F6D40610F2
:1054F00018D506107C0500204E14002078050020E9
:105500004C14002074050020C9D40610800500202A
:10551000BA0C071041D5061075D506108CD50610AB
:10552000FFFF0000D50E07104ED30610BED50610A3
:10553000E9D5061031D6061001F0DEF82B68C01A46
:10554000632800D835E70026C8483E702E6023F057
:105550003FFF082302930193FA239B0050220093FC
:1055600028213300012005F0E4FDC14A0500B042C6
:1055700000D1C04A2900C04823F0BAFE002D65D1F1
:10558000BE4823F025FF220001200C32A17C05F04B
:10559000DEFDBB4A051E00D1BA4A2900BA4823F0F5
:1055A000A7FEBA48002D06D02900B94823F0A0FE76
:1055B0000C2D4ED1B74823F00BFFB74823F008FF5E
:1055C000B64823F005FF260047363378B44D002B4C
:1055D00065D02B68002B4BD101F08EF82860B148C4
:1055E00023F0F6FE6379002B00D1EAE6E379002B85
:1055F00000D0E6E6AC4B62881988AC4D914253D09E
:105600001A8001F079F800284BD028606379002BCC
:1056100000D1E0E6E379002B4AD0637A002B47D033
:10562000A67A002E44D1A24B62881988A14D9142DE
:1056300000D18AE11A8001F05FF8002800D181E1F1
:10564000286035E0FF2008F0C7FCB9E79A4823F04E
:10565000BFFE0023E3722379002BF3D0012008F072
:10566000BBFC964823F0B4FE012006F0E7FEA7E756
:1056700001F042F82B68C01A6328B3D90023904880
:1056800033702B6023F0A4FE608809F001FE011E38
:1056900001D18C48A4E78C4823F02AFEA2E72B60B6
:1056A000A0E701232B60B1E72B68002B00D02FE18E
:1056B00001F022F8854A864B0592FA2206931B6870
:1056C0000400844FC31A9200934219D3FA23DB00DB
:1056D000984215D9069B1860059B1B78002B06D1B4
:1056E00000F000FA002802D10122059B1A703B78D5
:1056F000002B05D1FEF7F2FE002801D101233B70FB
:10570000754E3378002B10D1FA22744D92002B681D
:10571000E31A934209D3724B9C4206D9FDF760FB12
:10572000002802D101232C6033703B78002B44D039
:105730006C4A1368E31A632B3FD914AE002114603E
:105740003000282223F044FF3000FEF7F5FE0790DA
:10575000002800D01DE1FA21159B634D1A122B7011
:105760006A701A141B0EEB70169BAA701A122B711A
:105770006A711A141B0EEB71179BAA711A122B7205
:105780006A721A141B0EEB721A9BAA721A122B73EE
:105790006A731A141B0E1B98AA73EB738900FAF72D
:1057A000EDFD3378287400B200126874AB7473781E
:1057B000EB740AF0A9F8079B3B70059B1B78002B44
:1057C00021D0122704ABFF18002314AE310038009B
:1057D00033803B8000F0B2F9051E00D0DFE039884D
:1057E000424B32881980424B080A1A80414B58704C
:1057F0001970414B110A5970202001211A700BF0C9
:105800003FFA059B1D70344E3378002B0AD03B487D
:10581000FDF716FB051E00D0D2E0012140200BF061
:105820002FFA3570364D2B78002B14D1354B1B7861
:10583000002B00D1D8E0FA22334E92003368E31AED
:10584000934200D2D0E000F063FE002800D0C7E011
:10585000012334602B702D4800F090FE041E00D010
:10586000C5E00AF0B1FA2C70BEE0C0466CD6061056
:1058700059D3061055D3061096D60610D1D6061069
:105880006AD306105DD3061013D7061045D706104D
:105890009FD70610C9D706106CD706107ED8061001
:1058A0007C05002010D906104E1400207805002039
:1058B0004C140020740500204FD8061012D8061092
:1058C0002CD9061051D9061079D906106E05002082
:1058D000700500206D0500206C0500206805002083
:1058E000980800006405002085050020521400205F
:1058F00050140020F9010020F7010020F4010020DD
:1059000060050020990500205C0500209A05002014
:10591000267A002E00D0CBE600F0EEFE2B68C01AEF
:10592000FA235B00984200D270E633482E6023F0E1
:105930004FFD608805F053FC304B0100180023F048
:10594000D7FC63E601232B60B2E62B68002B00D165
:10595000AEE600F0D1FE2B68C01AFA235B00984235
:1059600000D2A5E6F43BFF3BA37225482E6023F04E
:105970002FFD022360880093DB181A00310005F028
:1059800068FC204A011E00D11F4A204823F0B0FCC9
:105990008EE6079B012B00D00FE700230CE70128C0
:1059A00003D10023059A13702DE7022800D02AE7BF
:1059B000FA22069B52001B68E31A9342F1D822E7B1
:1059C000012802D1002333702CE7022800D029E7F8
:1059D000FA220F4B52001B68E31A9342F2D821E7D8
:1059E0002B78002B00D036E709F02EF8E1E4012CEB
:1059F000FAD100232B70F7E7A9D90610E9D90610D0
:105A000019DA061088D3061075D3061054DA06107A
:105A10006805002030B5050085B0A8211E4823F098
:105A200067FC1E4C3220256000F072FE0A253023F0
:105A30006A4613730095A8212F3B03AA206801F042
:105A400065FB280000F064FE6A46154BA82193818F
:105A50000023937300952068033303AA01F056FBDB
:105A6000002806D00F4823F0B3FC0124200005B025
:105A700030BD6A460C4BA8219381E63BFF3B9373F4
:105A800000952068BE3B03AA01F040FB041EE9D14B
:105A9000064823F09DFCE9E792DA0610F0050020A5
:105AA000A6030000AFDA0610A6020000C5DA061051
:105AB0007FB5642304000A48009302AD0E002A005B
:105AC000A82100685F3B01F0C5FB012806D000203B
:105AD0002B885BBA33806B885BBA238004B070BDBF
:105AE000F005002070B5114D2B68002B0DD0104C27
:105AF000104E2378012B0AD100F0FEFD3368C31A43
:105B00000220642B02D903232370012070BD0123DE
:105B1000237000F0F1FD05233060A821064A2868B3
:105B200001F026FC0028F1D0EDE7C046F00500208A
:105B3000E8050020E4050020E905002030B50F4B02
:105B400004001A780220012A05D01A78032A03D10A
:105B500000221A70012030BD1A78022AFAD10848B2
:105B60000278457812022A430A808278C1780020A0
:105B700012020A4322801870EDE7C046E8050020B3
:105B8000E9050020054B1B68834205D1044B1A78B8
:105B9000012A01D101321A707047C046F005002079
:105BA000E8050020054B1B68834205D1044B1A7899
:105BB000012A01D102321A707047C046F005002058
:105BC000E80500200548064B10B5036002F0D4FD3F
:105BD000002801D0FFF7ECFA10BDC046F405002004
:105BE0000000304807B50B4B02689A4211D1802162
:105BF000094B49021A6D0D200A431A651B6D0022DC
:105C00000B4001930121019B00F094FD0D2000F059
:105C1000BBFD07BD0000304800004048002307B529
:105C2000012200930B4B196E11420CD1196C1143D8
:105C30001964196C91431964196E114319661B6E2E
:105C400013400193019BC023DB056846009302F0DB
:105C500059FE07BD0000404870B58EB00400142204
:105C6000002103A823F0B4FC1822002108A823F087
:105C7000AFFCC0232268DB059A4251D101240423E2
:105C800008A808940C9304F0F3F8002801D0FFF75B
:105C90008FFA0421234B90201A6E022522431A66A4
:105CA0001A6E032622400292029A1A6D00240A43B9
:105CB0001A651B6DC0050B400193019B802303A94E
:105CC000DB000393049505940696079500F028FFE2
:105CD000802390205B0003A9C005039304950594DD
:105CE0000696079500F01CFFA0212000C90002F0D5
:105CF000B9FDA0212000C90002F0C8FD0AF0BEFFD6
:105D000022002100122000F015FD122000F03CFDC1
:105D100019202200210000F00DFD192000F034FDB3
:105D20000EB070BD000040481FB50822002102A837
:105D300023F04EFC0122114B196E11420CD1196C4B
:105D400011431964196C91431964196E1143196652
:105D50001B6E13400193019B094A13690F2BFCD959
:105D6000A0236A465B001381403BFF3B9372054BC7
:105D700002A8039303F040FB05B000BD00004048BB
:105D800000180060102700000548064B10B503609E
:105D900004F0AAF8002801D0FFF70AFA10BDC046A7
:105DA0000006002000006048084B026882B09A425A
:105DB00009D18021064BC9021A6D0A431A651B6D71
:105DC0000B400193019B02B07047C0460000604841
:105DD0000000404809480A4B7F2210B503600023A9
:105DE000826080324360C2600361436104F0EEF878
:105DF000002801D0FFF7DCF910BDC04614060020D2
:105E00000040004010B5040088B01822002102A80C
:105E100023F0DEFB0D4B22689A4215D1202302931A
:105E2000802302A85B02059304F022F8002801D029
:105E3000FFF7BEF98021064B49015A6D0A435A65A6
:105E40005B6D0B400193019B08B010BD004000400A
:105E500000004048E0221148114B10B50360822336
:105E6000D200C26080225B00436000239200826106
:105E7000E13AFF3A836003614361C26103624362B6
:105E80008362193A03630833C262436304F0C8F9BA
:105E9000002801D0FFF78CF910BDC0463006002065
:105EA0000030004110B5040088B01422002103A87E
:105EB00023F08EFB154B22689A4224D18021144B8B
:105EC00049019A6D90200A439A659A6DE0240A4030
:105ED00004210292029A1A6DC0050A431A651B6DCD
:105EE00003940B400193019B022303A90493013BFC
:105EF000079300F015FE2100002002F0B3FC210002
:105F0000002002F0C3FC08B010BDC04600300041C4
:105F1000000040488021064B49005A6D82B00A4378
:105F20005A655B6D0B400193019B02B07047C04600
:105F300000004048FEE7FEE77047704710B500F0EC
:105F4000CFFB10BD7047000010B5064800F0E3FC21
:105F5000054800F0E0FC054800F0DDFC044800F0D6
:105F6000DAFC10BDE4020020980200204C02002060
:105F70000002002010B5044C200001F06DFD20004F
:105F800002F07CF910BDC046D404002010B5044CCA
:105F9000200001F061FD200002F070F910BDC04644
:105FA0008004002010B5024802F007FC10BDC04676
:105FB000F40500208021902010B50901C00500F0F3
:105FC00050FE802190204901C00500F04AFE10BD1E
:105FD00010B503F02FFD10BD10B503F031FD10BD5D
:105FE00010B503F033FD10BD10B502F003FE10BD77
:105FF00010B502F00FFE10BD10B5024804F0D8FA3B
:1060000010BDC046BC0500200120704710B523F02C
:1060100063FB162303600120404210BD10B523F03E
:106020005BFB16230360FEE770B50E00140000252D
:10603000A54201DB200070BD00E000BF70550135B6
:10604000F6E770B50E0014000025A54201DB200024
:1060500070BD705D00F01AFA0135F6E7012040428C
:10606000704780239B0100204B60704701207047E0
:10607000002070470B490C4A0300521A0B4910B517
:106080000868002801D10A480860C318934206D95D
:1060900023F022FB0C2303600120404210BD0B6063
:1060A000FCE7C0460020000000000120940600200C
:1060B0003C5E0020074B9A689B681B065B0F9207AB
:1060C00006D5054A013BDA401300044A13607047C5
:1060D000034AF8E7000040480048E801B8140020EF
:1060E0000090D003F8B5444B444A1968444C454BE2
:1060F000002911D11969002902D1996B00290BD00F
:1061000001239360FAF770F8BFF34F8F3E4BE360C3
:10611000BFF34F8FC046FDE73C49A160A168116104
:10612000202259680A435A60402259680A435A603B
:10613000802259680A435A60042259691142FCD0EE
:106140003021DA6932488A4310390A43DA61DA6960
:106150000240DA618022D86952000243DA612D4B95
:106160001A682D4B9A422DD01E222C4B1868904352
:106170000E3A02431A600122186802431A60284A44
:106180002848D4680440F02040052043D060802097
:10619000D46800042043D0601868234A104080224D
:1061A000920002431A601A681143196019681F4A65
:1061B0001140C02252010A431A6080221968D2009D
:1061C0000A431A60C02000220326FF258000170022
:1061D0002C003740FF00BC40154993089B005B181A
:1061E00019580132A143C024BC4021431950202A30
:1061F000EDD162B6F8BDC0469400404804000020CE
:1062000000ED00E0000050480400FA050000041012
:10621000FFFBFFFFF81E0010CCECBCFC94005048C4
:1062200000004048FFFFFFC03FFCFFFFFFC7FFFF2C
:1062300000E100E01FB50A4B02001C6801231800B2
:10624000002C0AD0002A08D06421009202910D226D
:10625000200001938C3101F003FA04B010BDC04658
:10626000980600200A4B30B517251C68012387B01B
:106270006D44020029701800002C07D06421200012
:106280000291019300958C3101F010F907B030BDF7
:106290009806002037B56B46DD1D0023324C2B706D
:1062A0002060324823F094F864230322F021206810
:1062B00001F048FB002806D078212D4823F018F87B
:1062C000012420003EBD78212A4823F011F828003F
:1062D000FFF7B0FF041E03D0274823F079F8EFE75B
:1062E0002978264823F004F80A2000F011FA21004A
:1062F0002000FFF7B7FF002801D02148EDE7052077
:1063000000F006FA12210120FFF7ACFF002801D0AF
:106310001C48E2E7052000F0FBF970210220FFF79E
:10632000A1FF041E1848D8D1052000F0F1F9210082
:106330000320FFF797FF002801D01448CDE7052080
:1063400000F0E6F901210720FFF78CFF041E10483A
:10635000C3D10A2000F0DCF90E4823F039F82821D7
:106360000D4822F0C5FFACE798060020DCDA0610E5
:1063700010DB06104DDB061084DB0610ADDB0610CB
:10638000D1DB061001DC061031DC061061DC0610E2
:1063900091DC0610BADC0610E1DC061010B5184BD3
:1063A000184C0C22236096239B016360002320007D
:1063B000A360E36023616261A361E36123626362BE
:1063C000A36204F02FFC002801D0FEF7F1FE0021AB
:1063D000200004F0ADFC002801D0FEF7E9FE00210A
:1063E000200004F0C5FC002801D0FEF7E1FE2000EB
:1063F00004F080FC002801D0FEF7DAFE10BDC04694
:10640000004000419C06002030B5040089B01422F1
:10641000002103A823F0DCF8194B22689A422CD102
:1064200080210824174BC9009A6DC0250A439A653C
:106430009A6D2D020A400292029A1A6D1248224366
:106440001A651B6D03A923400193019B022304934A
:1064500005330793039500F063FB2900012002F048
:1064600001FA2900012002F011FA20000022012186
:1064700000F060F9200000F087F909B030BDC04697
:10648000004000410000404800001048012307B5CB
:106490005B4201900122034801A904F0EEFA019841
:1064A0000EBDC0469C06002010B5002805D111483D
:1064B00022F08EFF0124200010BD0F4C66222060C8
:1064C00033210E4822F014FF20680A23012266219E
:1064D00001F038FA041E04D02100094822F008FF18
:1064E000E9E7084822F074FF0122074B1A70074BB6
:1064F0001C60E0E72BDD06107C0700204FDD061056
:1065000094DD0610CDDD061078070020740700200A
:10651000154BF7B51B78002B11D0144D2B68002BB1
:106520000DD0134C134F2378012B0AD100F0E4F85F
:106530003B68C31A0220642B02D903232370012075
:10654000FEBD0126267000F0D7F8082338600193BD
:10655000094B0022009366213300286801F05EF9A0
:106560000028EDD0E9E7C046780700207C0700202E
:1065700068070020640700206907002070B5041E2A
:1065800009D0104D02202B78012B05D02B78032B3E
:1065900003D100232B70012070BD2B78022BFAD180
:1065A00008222000084923F0BCF8084A002013689C
:1065B00028700133136023721B0A63720123A372D4
:1065C000EAE7C0466807002069070020740700203A
:1065D000054B1B68834205D1044B1A78012A01D16F
:1065E00001321A707047C0467C07002068070020FF
:1065F000054B1B68834205D1044B1A78012A01D14F
:1066000002321A707047C0467C07002068070020DD
:1066100010488546FFF766FD002103E00E4B5B58EE
:10662000435004310D480E4B42189A42F6D30D4A9E
:1066300002E00023136004320B4B9A42F9D30B4A59
:1066400002E0002313600432094B9A42F9D3FEF7AB
:10665000EFFDFEE700000120945B07103C140020D2
:10666000E41900207C0100203C140020C000002020
:106670007C010020FEE7000070B5114E0500337864
:10668000002B01D1012070BD03F0ECFB0400FA20C7
:1066900031788000F9F7E8FD01002000F9F7E4FD0A
:1066A00000F07EF8041EEDD1032DEBD8020001208E
:1066B0002900404200F03EF8024B20001D60E2E756
:1066C000BC140020C014002010B50320FFF7D4FF35
:1066D000041E03D1FFF71EFC200010BD0124FBE7C0
:1066E000034A044B11681B785B1813607047C0465F
:1066F00080070020BC140020014B18687047C0467A
:1067000080070020014B18687047C046C014002065
:1067100070B50400FFF7F0FF0500631C02D0044BC6
:106720001B78E418FFF7E8FF401BA042FAD370BDC6
:10673000BC14002010B5FF2403220B0021000240EE
:10674000D20091409B012340C943934000280ADBBB
:10675000C0240B4A800880008018A40002590A4017
:106760001343035110BD0F2210400838054A80081A
:1067700080008018C26911401943C161F2E7C04628
:1067800000E100E000ED00E0002805DB1F231840D9
:106790001E3B8340014A13607047C04600E100E0A1
:1067A0008022431E5204012093420DD2C021074A89
:1067B00007485360036A09061B021B0A0B43036266
:1067C00000200723906013607047C04610E000E08F
:1067D00000ED00E0F8B504000120002C32D025685F
:1067E000194B1421E818F9F73FFD184B800023647A
:1067F0000223A21D6064D3772E68154BA1681E404A
:10680000E36827690B433B4367693B43A7693B4305
:10681000E7693B43276A3B4333432B609123DB0506
:10682000C0188023A064DB01994201D1002363607A
:106830001F2163680B40036000200123E0630534DF
:10684000D377E077F8BDC046F8FF8FB700007048F7
:106850000F80FFFFF7B5441D0193E57F012D35D073
:106860000125871DE577FD7F0026AC466346EDB226
:10687000012B2AD10224FC770468C66326683B33C7
:10688000AE432660466C076C1E40B540019B7D60A0
:1068900063608368102B0ED1A260E160036B002B54
:1068A0000CD00E23226813432360012300202268AA
:1068B00013432360FEBDA160E260EFE7042223687A
:1068C0009343236022680A23EDE7E6770220F1E78D
:1068D00070B5841DE37F022B03D00423C363012022
:1068E00070BD0E2103683C251A688A431A60012294
:1068F000196891431960436C016C2B4015009D4051
:106900004D60E2770022431DDA77836B934200D01B
:1069100098470020E4E7F8B53C260427426C016C58
:1069200032403E0096400D6803681C6835420DD029
:106930003C420BD01A68920602D41A68BA431A6015
:10694000036B4E60002B19D0984717E002273E00DA
:106950009640354213D03C4211D01A68920606D4B4
:106960000A241A68A2431A600122831DDA770022E2
:10697000431D4E60DA77C36A9342E5D1F8BD08261D
:10698000370097403D42F9D03442F7D00E251C68BD
:10699000AC431C6001231C009440821D4C60C36307
:1069A000D3770022431DDA77436BE5E70630C07FDB
:1069B000C0B270470F22094B10B51C6980032243F7
:1069C000000C1A6198610A681A644A685A648A68F5
:1069D0009A64CA68DA64CC221A6010BD00100040C4
:1069E00070B50400FFF788FE012605000E4A136902
:1069F00033420FD00C21136900200B408B4208D189
:106A00000A489468416821434160012011690B43A1
:106A1000136170BD631CEAD0FFF76EFE401BA042FD
:106A2000E4D30320F5E7C0460010004084070020AF
:106A3000F8B5154D07002B780C0016000220012B2D
:106A40001CD00123FA202B70002380006B60FFF71D
:106A5000C7FF002810D1002F11D10F220B4BA40328
:106A60001969240C0A431A6133229C611E641A605E
:106A7000FA208000FFF7B4FF00232B70F8BD31002F
:106A80002000FFF797FFF3E7840700200010004085
:106A90000F22054B40061969000C0A431A611122A6
:106AA00098611A607047C04600100040F8B51A4E51
:106AB000040033780F000220012B13D00123337020
:106AC000002373602368FF2B0DD10F22134BFA2094
:106AD000196980000A431A6122221A60FFF780FFB9
:106AE00000233370F8BD01235B420B606568636867
:106AF000A2689B18AB4201D80020F1E72800FFF7FD
:106B0000C7FFFA208000FFF76BFF002801D03D602F
:106B1000E6E70135EBE7C04684070020001000409F
:106B20000023F7B50A681400DC4000D1F7BD012648
:106B30009E40324200D180E003245D00AC4003223D
:106B4000E4434F6800943A40541E012C31D88568C4
:106B5000009C2540AC46CC685D00AC4065462C43AB
:106B6000846045683C09B543012634409C402C4371
:106B70004460C568009C5E0025408C68B4402C438E
:106B8000C460022A17D107250F261D40AD00AE4074
:106B9000B446DC08A40004190194246A2600644663
:106BA000A643B4460E696446AE402643019C266265
:106BB00001E0032ADDD10468009D25402C005D0022
:106BC000AA4022430260C0229202174235D080229E
:106BD000D20217420AD0802501229026ED059A4064
:106BE000EC68F605B0422AD12243EA60FA020AD5DF
:106BF000802501229026ED059A402C69F605B042C9
:106C000020D122432A617A020AD5802501229026CA
:106C1000ED059A406C69F605B04216D122436A61CF
:106C2000FF030AD5802501229026ED059A40AC6924
:106C3000F605B0420CD12243AA61013372E7120477
:106C40009443D1E712049443DBE712049443E5E74D
:106C500012049443EFE7002A01D0816170478162FA
:106C6000FCE79022802310B5D205DB05904206D1C7
:106C7000DA69114207D0D961FCF73EF903E0DC691B
:106C80000A04224200D110BDDA61F5E703689A696F
:106C9000920701D500229A6201229969114202D11C
:106CA00099690A439A61704730B5039C0068234391
:106CB000120489051A43890D054B45680A43640D82
:106CC000234352009D4352082A43426030BDC046D0
:106CD000FF63FF0310B5426B1A4C0BB2A2421ED0E9
:106CE000194CA2421BD0194CA24218D0B822F2244F
:106CF000DB171A40CB07DB17234013438A0706D55F
:106D0000F422134301680A6813430B6010BD102975
:106D100001D19022F5E72029F4D10B43F2E7B82204
:106D2000F224DB171A40CB07DB17234013438A07F3
:106D3000E6D41029EDD0202901D16022E1E74029D5
:106D4000EBD0DFE7098104109D840410AD7F0410AF
:106D5000002310B5CA0708D5030041331A78282349
:106D60001A40CA33282A00D1B03B8A0708D502004E
:106D70002824413212782240A2420BD144221343EC
:106D800009B2002901DAB822134301680A689A435C
:106D90000A6010BDF422F2E7F7B505681700AA698A
:106DA000102316000400019100201E401A420DD04D
:106DB0000600EB61009025682022AB69134260D188
:106DC000002E30D004260120009B1E438022AB6998
:106DD0005200134202D00120EA6106438022D20011
:106DE000134203D0082101200E43EA618022920061
:106DF00013424BD00223EA611E432000FFF746FFF7
:106E00006B68244A012013406B60636C202233437B
:106E10006364230041331A7022000023423240345D
:106E20001370237034E0019B0133C5D0FFF764FC7D
:106E3000019BC01B984201D8002BBCD122002368C3
:106E40004232586811789A69C9B212040BD580226F
:106E5000D201104207D1202905D059680A435A604F
:106E6000FFF74AFC0700202523689B692B42A2D12B
:106E7000FFF742FCC01B1928F6D9202301260093F6
:106E800099E7002E9ED12023EB619BE70028B4D127
:106E9000FEBDC04600E800FEF8B504000D00160077
:106EA000022723689B693B4201D0002021E0320089
:106EB00029002000FFF770FF002819D16B1CF0D0CB
:106EC000FFF71AFC801BA84201D8002DE9D12368E6
:106ED000996902230A001A401942E2D12021636C09
:106EE0000B43636423004034413319705A7022709D
:106EF0000120F8BDF8B504000D0017001E0023683E
:106F00009B692B405B1B5A425341BB4201D000207E
:106F100026E031002000069AFFF73EFF00281ED130
:106F2000731CECD0FFF7E8FB069BC01AB04201D8F7
:106F3000002EE4D123689B692B405B1B5A425341CE
:106F4000BB42DCD12022636C1343636423004133D2
:106F50001A70220000234232403413702370012043
:106F6000F8BDF8B504000E001700202523689B69C2
:106F70002B4201D000201DE03A0031002000FFF735
:106F80000BFF002815D1FFF7B7FBC01BB04201D89B
:106F9000002EEBD123689B691A002A402B42E5D1D1
:106FA000636C2B4363642300403441331D705A707B
:106FB00022700120F8BD0000F7B504000025042769
:106FC00020260091019223689B693B4201D1002D4C
:106FD00001D02800FEBD019A20000099FFF7DCFED9
:106FE000236805009A69324214D0002811D19A69A9
:106FF0001022996911421AD0DA616764DE615A6819
:1070000012490A405A60230041331E705870013BF8
:1070100018700125FFF770FB019BC01A009B984276
:1070200001D8002BCFD1002D03D00125CBE7606420
:10703000F0E723689B693B42C5D1636C33436364CB
:10704000230041331E70013B1D70EEE700E800FE97
:1070500070B504000120002C4ED0250041352B785E
:10706000DAB2002B05D12300403320001A70FDF75F
:10707000E1FC242301212B702368E0681A68A668CC
:107080008A431A601D4962680A401A619A681C495D
:107090000A409A60012807D18022120232439A6086
:1070A0005A681848024009E08422120232439A606A
:1070B0000228F5D180225868120102435A605868AC
:1070C000114A02435A60DA6800200A40DA606169B6
:1070D00022690A43A16909020A43DA60216AE26966
:1070E0000A431A60012219680A431A602023606467
:1070F0002B7020634234207070BDC046FFFFFFF04C
:10710000FF7FFFFFFFF7FFFF00800002F0B50600E2
:1071100085B0029203934136337804000F000220B9
:10712000202B14D1230040331A78012A0FD00122DA
:107130001A70FFF7E1FA802105000090192301225F
:1071400020000902FFF7D6FE002802D0012005B07A
:10715000F0BD212333702300102242331A70029BAA
:1071600060646362039B39496385638D6063FF2BB1
:1071700030D98023EF3222855B04029E2068367866
:10718000013A8662029892B201306062608D228577
:10719000013880B201326085D2B2009139002000FE
:1071A000FFF782FD638D2A0020000A99002B1DD174
:1071B000FFF7D7FE0028C9D120212368244DD961CB
:1071C0005A682A405A60230040344133197058707D
:1071D0002070BCE7628D92B22285002A02D0802303
:1071E0009B04CAE7009180239B04D7E7FFF754FE76
:1071F0000028ABD1636A2268197801339162636217
:10720000638D228D013B9BB26385013A638D92B2FF
:107210002285002BC6D0002AC4D1802120000A9BE1
:107220000095FFF767FE002800D08FE7638DFF2BE6
:1072300005D9FF22802322855B040090AEE7628D92
:1072400092B22285D2B20090CDE7C04600200080E5
:1072500000E800FEF0B5060085B0029203934136C7
:10726000337804000F000220202B14D12300403378
:107270001A78012A0FD001221A70FFF73DFA8021F7
:10728000050000901923012220000902FFF732FEB9
:10729000002802D0012005B0F0BD22233370260063
:1072A000123B42363370029B60646362039B6063EF
:1072B0006385628D2C4BFF2A20D9FF222285009303
:1072C00080235B0439002000FFF7EEFC638D2A0069
:1072D00020000A99002B19D1FFF743FE0028D9D1CD
:1072E00020212368214DD9615A682A405A60230021
:1072F00040344133197030702070CCE7628D92B207
:107300002285D2B2009380239B04DBE7FFF754FE73
:107310000028BFD123685A6A636A1A70636A228D93
:1073200001336362638D013A013B9BB26385638DD8
:1073300092B22285002BC9D0002AC7D1802120001B
:107340000A9B0095FFF7D6FD0028A3D1638DFF2B84
:1073500003D9FF2222850090B2E7628D92B2228586
:10736000D2B20090CFE7C0460024008000E800FEC3
:107370009C460300F0B587B00491413319780400AE
:107380000220202952D1216880258F692D023E00DC
:107390002E402F424AD1250040352F78012F45D06D
:1073A00001382870270021301870102342373B70B5
:1073B000634666646385374B6262E362364B6363A0
:1073C000638DFF2B34D9FF26802326855B04E06B79
:1073D0000393002834D00025304B0563C362304B43
:1073E0008563436324313300FFF734FA23004033CD
:1073F00006000593A84230D1258D2A4BEAB2200021
:1074000004990093039BFFF74FFC638D10215B1BD6
:107410009BB26385059B20001E70FFF75BFC8023F9
:1074200022681B0211680B431360002007B0F0BDF7
:10743000668DB6B22685002E1BD080239B04C6E73E
:107440002300202241331A7080233870626C40344C
:107450001343636020700120E8E7230020224133BA
:107460001A7010233D70626C13436364059B1D709A
:10747000F1E70D4B200063630A4B049900938023CE
:1074800032009B04FFF710FC022120002E70FFF752
:1074900021FCCAE70000FFFF0981041029820410C3
:1074A00011820410002400806D7E0410F0B50700E6
:1074B00087B003930CAB029204CB41371B88049234
:1074C00005933B7804000E000220202B08D1002AEF
:1074D00002D0059B002B05D180239B006364012013
:1074E00007B0F0BD230040331A780220012AF7D0FC
:1074F00001221A70FFF700F980210500009019237E
:10750000012220000902FFF7F5FC0028E7D1212322
:107510003B7027001F3342373B70049B60646362FB
:10752000059B606363856B461A7B4B4B3100009370
:10753000802320005B04FFF7B7FB2A0020000E9990
:10754000FFF7AAFC002829D1039A2368012A16D143
:107550006A46127A9A620022802120000E9B0095D2
:10756000FFF7C8FC002819D1638DFF2B1AD88023A0
:10757000628D9B0492B22285D2B2009017E0029AEB
:107580002000120A9A620E992A00FFF785FC002853
:1075900004D16B4622681B7A9362DCE700234034F7
:1075A00023709CE7FF22802322855B04009031003A
:1075B0002000FFF779FB2A0020000E99FFF76CFCF2
:1075C000002800D08BE7636A226819780133916242
:1075D0006362638D228D013B9BB26385013A638DAB
:1075E00092B22285002B16D0002A14D180212000CF
:1075F0000E9B0095FFF77EFC002800D06FE7638D9F
:10760000FF2B21D9FF22802322855B0400903100CB
:107610002000FFF749FB638D002BCCD12A0020000E
:107620000E99FFF79EFC002800D058E72021236820
:107630000A4DD9615A682A405A60230040344133C8
:107640001970387020704BE78023628D9B0492B2D2
:107650002285D2B20090DAE70020008000E800FE28
:10766000F0B5060087B003930CAB029204CB413611
:107670001B8804920593337804000F000220202B0E
:1076800008D1002A02D0059B002B05D180239B0046
:107690006364012007B0F0BD230040331A78022054
:1076A000012AF7D001221A70FFF726F8802119234A
:1076B00000900500012220000902FFF71BFC031EB9
:1076C000E7D12222327026001E3242363270049AEE
:1076D00060646262059A4E4962856A466063127B05
:1076E000200000913900FFF7DFFA2A0020000E99F0
:1076F000FFF7D2FB00282AD1039A2368012A17D169
:107700006A46127A9A620022402120000E9B009560
:10771000FFF7F0FB00281AD1628D3E4BFF2A1AD8E2
:10772000628D92B2228500938023D2B29B0417E02F
:10773000029A2000120A9A620E992A00FFF7ACFB07
:10774000002804D16B4622681B7A9362DBE7002392
:10775000403423709DE7FF222285009380235B0441
:1077600039002000FFF7A0FA0022042120000E9B20
:107770000095FFF7BFFB002800D08AE723685A6A0C
:10778000636A1A70636A228D01336362638D013A02
:10779000013B9BB26385638D92B22285002B16D08C
:1077A000002A14D1802120000E9B0095FFF7A2FB38
:1077B000002800D06DE7638DFF2B21D9FF228023A5
:1077C00022855B04009039002000FFF76DFA638D7D
:1077D000002BC9D12A0020000E99FFF7C2FB002818
:1077E00000D056E7202123680B4DD9615A682A4002
:1077F0005A6023004034413319703070207049E7DB
:107800008023628D9B0492B22285D2B20090DAE787
:10781000002000800024008000E800FEF0B587B062
:10782000049304000CAB039141309446017804CBDF
:1078300002251B88202907D1002A01D0002B06D160
:1078400080239B0063640125280007B0F0BD2168F8
:1078500080268F6936023D00354005950225374266
:10786000F2D1260040363778012FEDD0013D35703A
:107870002700213505704020423738700598626234
:10788000606463852A4BE3622A4B6363039BE36472
:10789000FF23608D984201D8638D9BB26046049DA2
:1078A0002385C0B2012D26D1886201204042206587
:1078B000E06B002823D000261F4D0663C5621F4DD4
:1078C000866345632431FEF7C5FF2300403305007E
:1078D0000593B0421FD16B461A7C194B0399009354
:1078E00003002000FFF7E0F9059B012120001D7037
:1078F000FFF7F0F9A8E765462D0A8D62D7E7230068
:10790000202241331A7080233870626C4034134354
:107910006360207097E72300202241331A70102300
:107920003E70626C13436364059B1E708BE7C04618
:107930000000FFFFAD7F04102982041011820410A3
:1079400000200080F0B507001D00002389B00592DB
:10795000079341373B7804000220202B67D123682E
:107960009E69802332001B021A401E425FD1230011
:1079700040331E78012E5AD001381870242389050F
:107980003B708B0D62640393E368012B32D1304B63
:10799000039A134322685360FEF7AEFE0600226886
:1079A000936992699B06D206DB0FD20F134323D053
:1079B000102123689A691140049110210A4238D19C
:1079C0002B002000049A00964918FFF793FA00282C
:1079D00025D0636C042B04D120222368DA61049B38
:1079E0006364079B059A01330793079B079B9342A8
:1079F000CAD30AE0174BCBE76B1CD0D0FEF77CFE56
:107A0000801BA84201D8002DC9D120233B70626C95
:107A100040341343636000230120237007E02023D8
:107A20002268D3612200403441321370207009B0C3
:107A3000F0BD10222021DA6120002B0000220096E8
:107A4000FFF758FA0028CCD120222368DA61C8E772
:107A50000020000200280002036810B599691A6826
:107A6000436B002B00D0984710BD7047030070B5E2
:107A700000252022060042331D70013B19780400C6
:107A800040361A7021290AD1112345630363203936
:107A9000FFF75EF920003570FFF7E7FF70BD122396
:107AA000456303630221FFF753F920003570FDF7AA
:107AB00039FBF3E7704770470100036810B5040015
:107AC00000201A6842310870510418D51A68184904
:107AD0000A401A60230041331A78292A14D1013A46
:107AE0001A702123200023630121FFF731F92300BD
:107AF0000022403320001A70FFF7DCFF10BD120493
:107B0000E8D51A680B49E3E71A782A2AF6D1023A2F
:107B10001A702223200023630221FFF719F92300A2
:107B20000022403320001A70FFF7C5FFE6E7C04689
:107B3000FFBFFFFFFF7FFFFF70470300F7B528225D
:107B400041331B7804000168134093423CD1FE2767
:107B50008D698E698B68CA68ED030192C268360C24
:107B6000ED0F3E40022A25D19B059A0D5B0F734015
:107B7000180006263040334210D1A36C0133A364B1
:107B8000A36C022B09D19B19A064CB612300403365
:107B9000187029002000FFF7CFFFF7BD80212000DB
:107BA0000902FFF7D5F82300002240331A70019A2A
:107BB0003A40EEE780210902FFF7CAF823000022CD
:107BC00040331A703200E4E70823CB6100234034CD
:107BD0002370E2E770470000184B10B5C362002322
:107BE000020003630400202041321070537004220D
:107BF0006363114212D02368596A636A1970636A19
:107C000001336362238D002B08D0013B2385638DF4
:107C1000013B9BB26385636C1A4362642000084990
:107C2000FFF796F8102223682000DA612300002273
:107C300040331A70FFF7CEFF10BDC0460000FFFFB3
:107C400003800000704770470100020010B5413109
:107C50000C7800234032602C06D1403C0C7003634A
:107C60001370FFF7F0FF10BD03631370FDF769FA9F
:107C7000F9E7000070B505000022040041354230EC
:107C80002B7802703A48283BE0626285626C0A43B6
:107C90006264022B2BD803212000FFF759F8282318
:107CA0002B70344BA06B6363236B002840D01A0009
:107CB0001021113A8A433BD123681A68520403D534
:107CC0001A682D490A401A60FEF770FE01282BD071
:107CD000A06B2A4B00228363230040331A70FEF707
:107CE000F7FD002823D0A06B836B98471FE020008E
:107CF0002349FFF72DF82000FEF7C8FF2B78602BF3
:107D000010D020222A702368996911420AD09969FB
:107D1000103A114204D0DA61616C0C3A0A43626491
:107D20002022DA610023BDE72000FFF78DFF70BD40
:107D3000E06B0028F8D01022123B9343F4D1236863
:107D40001A68120403D51A680E490A401A60FEF731
:107D50002DFE0128E8D0E06B084B0022836323004E
:107D600040331A70FEF7B4FD0028E0D0E06BBBE7AB
:107D70000000FFFFA9850410FFBFFFFFC5860410A8
:107D800003800000FF7FFFFFF7B520230500066892
:107D90004135F3612B7804000F00212B2BD10121F9
:107DA000FEF7D6FF1123236373682E4A13407360D6
:107DB000002363632C4BE36210231F4204D0F36162
:107DC000626C0C3B134363642B78602B05D17F07F7
:107DD00003D5736ADBB20193019B2000FEF756FFC7
:107DE000636C2A78602A01D0002B0CD02000616CD3
:107DF000FFF740FFF7BD2B78222BD5D10221FEF7EC
:107E0000A7FF1223CFE72A78212A13D1013A2A703B
:107E100022002100236342321078403113700B702E
:107E2000402803D12000FFF70DFFE3E72000FFF714
:107E30001CFEDFE72A78222ADCD1023A2A702200CF
:107E40002100236342321078403113700B704028B8
:107E500003D12000FDF76AF9CCE72000FDF762F9B5
:107E6000C8E7C04600E800FE0000FFFFF0B50700CD
:107E700040373B7804000D001600022085B0012B2E
:107E80001AD001233B700F33194217D01A4215D074
:107E900022682000D361626C0C3B13436364FEF7DD
:107EA000F5FE20231D4205D01E4203D029002000EC
:107EB000FFF76AFF0020387005B0F0BD04231D42B3
:107EC00011D01E420FD09D4323685A6A636A1A700C
:107ED000636A01336362238D013B2385638D013B1C
:107EE0009BB26385DDE76B06DA0F002B0CDB022308
:107EF0001D4209D01E4207D0638D002BD1D0636A8A
:107F0000226819789162E4E72B0635D57306C8D547
:107F1000628D2368002A23D0208D002820D1596843
:107F2000638D8905890DFF2B08D9FF2280232285C7
:107F30005B0400902000FEF7B7FEB2E7628DE36AB3
:107F400092B20393184B22859C46039BD2B26345A1
:107F500002D0E36A0090EDE7802300909B04E9E7FC
:107F60005B689B0103D42000FFF780FD99E7402167
:107F70002000FFF77FFE94E7002A00D191E7730607
:107F800000D48EE7638D002BF1D123685A689201EB
:107F900000D586E7E16A044A9142E4D1802259681B
:107FA000D2010A435A607CE70000FFFFF7B50600E4
:107FB0004036337804000220012B15D001233370A2
:107FC0000F33194211D01A420FD022682000D3611A
:107FD000626C0C3B134320216364FEF77BFE2000A0
:107FE000FEF754FE00203070FEBD0223194208D077
:107FF0001A4206D02368226D9A6201235B422365F0
:10800000F0E740250B063BD52A4239D0012120005C
:10801000FEF79EFE10212000FEF75CFE638D002B14
:1080200029D0638DFF2B1BD90023BF35E16C25853B
:10803000009380232A0089B25B042000FEF734FEFF
:10804000638D5B1B9BB26385230041331A782368E1
:108050001968222A47D1802212020A431A60C1E716
:108060000023658DE16CADB2258500938023EAB2D3
:1080700089B29B04E1E729002000FFF7FBFDB1E78F
:10808000294233D02A4231D0270001212000FEF7B7
:108090005FFE413710212000FEF71CFE3B78223B9B
:1080A0005A425341174A9B029B18628DFF2A10D9EE
:1080B000FF25E16C2585009380232A0089B25B04AB
:1080C0002000FEF7F1FD638D5B1B9BB263853A7860
:1080D000BDE7658DE16CADB2258500938023EAB2E2
:1080E00089B29B04ECE78022D201B6E72023194233
:1080F00000D177E71A4200D174E72000FFF744FE71
:1081000070E7C04600200080F7B5070040373B7895
:1081100004000220012B15D001233B700F331942BC
:1081200011D01A420FD022682000D361626C0C3B40
:10813000134320216364FEF7CDFD2000FEF7A6FD6A
:1081400000203870FEBD4023080641D51A423FD0BA
:10815000266832689A433260638D002B2CD0716898
:10816000638D8905890DFF2B17D9FF258023258570
:108170005B040020EAB200902000FEF795FD638DBD
:108180005B1B9BB26385413423783268222B10D16C
:1081900080231B0213433360D2E7658D1B4BE26AD9
:1081A000ADB225859A4201D0E36AE2E780239B04C1
:1081B000DFE78023DB01EDE773689B0103D4200038
:1081C000FFF754FCBCE740212000FFF753FDB7E761
:1081D000194212D01A4210D0638D002BF3D12268BD
:1081E00053689B01ACD4E16A084B9942E7D18023E4
:1081F0005168DB010B435360A2E7202319429FD053
:108200001A429DD02000FFF7BFFD99E70000FFFF55
:108210008023806A10B502681B0251680B435360CB
:108220001021FFF727FD10BD10B5846A124A21689E
:108230000B6813400B60638D002B04D120212000BC
:10824000FEF748FD14E0238D626A608DD218FF238B
:108250006262984201D8638D9BB2E06B2385243122
:10826000FEF7F8FA002804D010212000FFF702FDE5
:1082700010BD4021E3E7C046FF7FFFFF70B58025BA
:1082800003686D0099691A68294206D0140604D55E
:108290000124466C34434464DD618025ED002942AD
:1082A00006D0140604D50824466C34434464DD61CA
:1082B0008024A400214206D0120604D50222416C7B
:1082C0000A434264DC610B23416C194201D0FFF781
:1082D000D1FC70BDF7B5056806002B6841360093E8
:1082E000C36A04000193202330780F002138EB612A
:1082F00009280CD8F7F79AFF05680B0B0B0B0B6ED0
:10830000056820005D49FEF723FD212323638022B9
:108310006B68120213436B606B68594A200013406C
:108320006B60FEF7B3FC009B5B0459D52B68554A84
:1083300013402B60A36B002B03D01B685B689BB2C0
:10834000638504231F420FD06A6A9F43636A1A70D1
:10835000636A01336362238D002B05D0013B2385C3
:10836000638D013B9BB26385638D002B03D0042397
:10837000626C1343636410231F4211D0009A1A42A7
:108380000ED0628D002A49D13378282B33D1802337
:10839000019A9B049A422ED139002000FFF71CFC61
:1083A0002300002242331A70656C6263954244D008
:1083B0002000616CFFF75EFC3378282B03D1390075
:1083C0002000FFF709FCF7BD20002F49FEF7C0FC95
:1083D00022239BE720002D49FEF7BAFC002395E7F6
:1083E0008022009B12021342ABD02B68284A134014
:1083F0002B60E36B9FE731781022236829290BD18A
:1084000024490198884207D02000DA61FEF73EFC3B
:108410002000FFF751FBC3E7DA61C1E72268D361AF
:108420000423626C13436364019A1B4B1A42B7D155
:108430002000616CFFF71EFCB2E72700E36A154AD3
:10844000403793420CD02000FFF736FB2023114A1F
:108450002000E262337025633D70FFF7BBFBB2E79B
:10846000202332782000337025633D70222A02D108
:10847000FFF721FBA7E7FFF71DFBA4E70180000042
:1084800000E800FEFFBFFFFF028000000380000045
:10849000FF7FFFFF0000FFFFFFFFFFFEF8B50500B5
:1084A00040352E780400C36A0220012E0BD001381B
:1084B00028701F30014207D0024205D02000FFF78C
:1084C00009FF00202870F8BD102631425ED03242EC
:1084D0005CD080273F0250043A401700C00F07438A
:1084E00051D0E66B002E1DD0002A03D032685268AE
:1084F000564272412600A76B4136002F05D0002856
:1085000003D038684068002801D0012A1CD1327895
:10851000282A09D180229204934205D12000FFF736
:108520005BFBCEE73200E5E7102130782268D161AD
:108530002928C6D11A488342C3D02000FEF7A6FBE3
:108540002000FFF7B9FABCE710212268D1610422AC
:10855000616C0A4362643078124AC0B21342B0D1EF
:108560002138092808D8F7F761FE050C0707070727
:108570000707050C212323632000616CFFF77AFBBA
:108580009FE72223F7E72368DE619AE70823194271
:1085900097D01A4200D194E72000FFF7CEFA90E777
:1085A0000000FFFFFFFFFFFE70B5050040352E788D
:1085B0000400C36A0220012E0BD0013828701F303E
:1085C000014207D0024205D02000FFF783FE0020C1
:1085D000287070BD102001422FD002422DD0628D34
:1085E000002A1CD1220041321078282807D180208F
:1085F0008004834203D12000FFF7EEFAE7E7102161
:1086000010782268D1612928E1D12C488342DED03C
:108610002000FEF73BFB2000FFF74EFAD7E7226869
:10862000D0610422616C0A436264254A1342CED1B0
:108630002000616CFFF71EFBC9E70420014219D03E
:10864000024217D0628D002A0DD02268516A626AF8
:108650001170626A01326262228D013A2285628D56
:10866000013A92B26285628D002AB0D1134A9342D8
:10867000ADD0D0E70820014205D0024203D020004F
:10868000FFF75BFAA3E702200142A0D002429ED08E
:10869000628D002A0DD0636A2268197801339162D5
:1086A0006362638D013B9BB26385238D013B238510
:1086B0008DE7034A134200D089E7ACE70000FFFFD3
:1086C000FFFFFFFE806A10B5836B002B01D00022F4
:1086D0009A63C36B002B01D000229A63FFF7B4FAB0
:1086E00010BD0000F0B504004134227803000F00F3
:1086F0000220D6B2202A18D11D0040352A78012A3E
:1087000013D0242222701B68233A1968074891432A
:10871000196019680140002019601968394319600F
:1087200019680A431A6026702870F0BDFFEFFFFF3A
:108730000200F0B5413214780300E5B20220202C8B
:1087400017D11C0040342678012E12D02230107030
:108750001B6823381E68074F86431E601E68090287
:108760003E403143196019680843186000201570B5
:108770002070F0BDFFF0FFFF10B504000120002CB9
:108780001AD02379002B02D12000FDF72BFA022307
:1087900080212371236800201A680A431A601A682E
:1087A0008A431A605A6873390A435A605A688A437E
:1087B0005A600123A060237110BD0822036870B5C0
:1087C0009E6804005D6816420BD0154209D0012155
:1087D00080680143A1605968114359605968914309
:1087E0005960042216420BD0154209D00221A0681C
:1087F0000143A16059681143596059689143596018
:10880000A368002B02D0200002F0C8FD01231E4205
:108810000CD01D420AD022682000516819435160D3
:10882000516899435160237102F0AEFE70BD0000A3
:10883000002803D001280AD001207047084B1A6A8B
:108840000A431A625A6A8A435A620020F5E7044BC7
:108850009A6A0A439A62DA6A8A43DA62F5E7C0469C
:1088600000005048002803D0012807D0012070479D
:10887000054A136A8B4313620020F8E7024A936AA1
:108880008B439362F8E7C04600005048002803D0AD
:10889000012807D001207047054A536A8B43536271
:1088A0000020F8E7024AD36A8B43D362F8E7C04658
:1088B00000005048A923114A9B00D1580433D358D3
:1088C000C9B21B061B0C0B43AB2189007F205158FA
:1088D000002B0DD00B290BD806224A43773A1E2BCA
:1088E00008D8A220FF305843054BC018800A8018D2
:1088F00040B2704706325B08F1E7C04600140060E2
:10890000A0460000F0B5A94B85B01A68A84B9A4262
:1089100000D044E10F22A74B1F681D681E6819682C
:108920001B683F0A2D0B360C1740154016401B0ED6
:10893000083A134003930123090D1140029101935A
:1089400000239D4C2371984201D0FDF785F9C02387
:108950000321DB05DA680F208A43DA60DA682D012B
:108960008A43DA60954B964A9C469B6A9E21134047
:1089700062469362934B89005A5882433243F026F1
:108980005A5004395A58B2432A435A505A588243CB
:108990003A435A50019A002A0DD02C395A580838B7
:1089A00082430298024338205A505A58824303980F
:1089B000C00002435A50FF2055258349C227CA6C84
:1089C0007F0082432A43CA6466228E6D8643324307
:1089D0008A65C426CA6E7600824315431D22CD6681
:1089E0009D5985432A439A515922DD5985432A438B
:1089F000DA51C622520016009D585B3A8543FF3A71
:108A00002A439A5101220D6F15430D6766686F4D19
:108A10002E408025ED0135436560FC2567686C4E6E
:108A2000AD0337403D439027656065683F052D02E3
:108A30002D0A2F43E8256760A768ED0337403D43C3
:108A4000E027A560A568BF052D022D0A2F437625D6
:108A5000A760A76887433D43A560A7685B4D2F408B
:108A6000E825AD013D43A560E568C2272E4080257D
:108A70006D033543E560E568564E7F002E40C02506
:108A80006D053543E5600525266986433543256137
:108A9000E5681A268543EB382843E060E5684B48D3
:108AA0000540A020C0002843E060042065692843F9
:108AB00060618020656900042843606180206569E9
:108AC000800528436061444D444805829E25AD00E1
:108AD0005D59C27485745D2505759D25AD005D5990
:108AE00045753F4DC5829225AD005D5942760576AC
:108AF00012258576CD6CC5763A4D85838D6DC2770E
:108B000085778518EE77CE6E851CEE77C426364DB8
:108B1000760045849E59451DEE772126851DEA770E
:108B2000C51DEE77314DDE5907000585C62508378E
:108B3000FE776D005E5905002A352E7005002B3535
:108B40002A7005001B272C352F700D6F01002D3169
:108B50000D700500002106002E352970244D0C36BD
:108B6000056045608660C1600168206821608021E1
:108B70001A616069C90501436161996A60461143E0
:108B80009962C023DB05596859606146496C1143FD
:108B90004164016C0A4302645B6805B0F0BD0023C8
:108BA0000826072537000193CAE6C046F81E0010C4
:108BB000CCECBCFCE81E0010C000002000180060D7
:108BC000FFFFFFBF00140060FC140060FF00FFFF08
:108BD000FFFF00FFFFFFFFC0015E00009C070020B9
:108BE00001520000011500000122000001230000D5
:108BF000AC07002070B5C024E405E56966686660CE
:108C000000F0DEFB2800304303F00CFC00F0C8FB52
:108C1000636870BD10B503F0E1F910BD30B5104ABE
:108C2000916893689942FBD10029F9D00D4CCBB2E1
:108C300063430D126C431B121B1910335B11C3608D
:108C40000160D168D3689942FBD10029F9D0064B65
:108C50008A11534380331B128360416030BDC0468C
:108C600000100060F6BC0800530700000A4B020029
:108C70005869002310B51900F7F7F4FC032200230C
:108C8000F7F7F0FC80220023D204801859414B01F1
:108C9000C00E184310BDC046D0070020F8B5EFF352
:108CA000108772B6154E164B164A18693300346F8A
:108CB000756F88331860B36FF169C01AF7F700FA5F
:108CC00000230200A4185D41330080335A68AA4291
:108CD00003D80CD11B68A34209D90120094AF169C4
:108CE0004042F7F7EDF900230200A4185D418036F9
:108CF0003460756087F31088F8BDC046D007002047
:108D00000018006035060000F8B51E4C1E4E1F4AC4
:108D1000A16907001B20B57BF7F7D2F9C0B27071CB
:108D2000B079EDB2C0B2FFF7A1FF23003D33187058
:108D3000307AED1001354019FFF798FF23003833E2
:108D40001870707A4019FFF791FF230039331870BB
:108D5000B07AC0B2FFF78AFF23003A331870F07A76
:108D6000C0B2FFF783FF23003B331870002F07D0FA
:108D70006823327A3C34521953431B0A1B33237045
:108D8000F8BDC046D0070020C00000202603000028
:108D9000F8B51D4C1D4B1E4D1869A36F1D4A286068
:108DA000216AC01AF7F78CF9226F636F060000275B
:108DB00092197B41267822676367BE4213D1A06F68
:108DC0002968091AA06881420DD20120114A216A3E
:108DD0004042F7F775F933000200206F616F1218F7
:108DE0004B4122676367210080310A604B6021009C
:108DF000883109686068A167002180185941E369DA
:108E0000A062E1622362F8BDD00700200018006074
:108E1000580800203506000003000020F0B5714A14
:108E2000714C127885B0824200D1A4E0EFF3108239
:108E3000039272B6012B01D1FFF730FFA26AE36AF9
:108E4000A06DE16D803426686768C8240025A402FF
:108E5000A4185D418D420ED801D184420BD8B924AB
:108E60000025640012196B419F4204D800D0B4E081
:108E7000964200D8B1E04C225242D31712184B410F
:108E8000009201930A22002392197B41019D564CC6
:108E90009D4205D800D09BE0009D954200D897E008
:108EA00022003C32157822002300643212786033AD
:108EB0001B78002A64D0002B5FD0230038331B7846
:108EC000861B4A4AA16930000093F7F7F9F823009E
:108ED00088331F68A36E0100C8335B19444A454DAF
:108EE0009E4255D907246B790326C31A00981B1A92
:108EF000D8195062906AA0439062C020C005C4682F
:108F0000B443C460C468B443C4608020946AC0059C
:108F1000204390628020946A8005204390626879A3
:108F2000009C0019344EC9193160802629791B181C
:108F300031432971F021A9750F31E975411D2A4C82
:108F40008B423CD2C0230320DB05D9688143D96022
:108F5000D9688143D960936A284902380B409362EB
:108F60002300012261331A70802362345B00238066
:108F7000039B83F3108805B0F0BD230039339EE7CF
:108F8000002B02D023003A3399E723003B3396E7C6
:108F90003D342378194E9C46C31A00981B1AC020F2
:108FA000DC19C0050461946A344094620324C668E5
:108FB000A643013C3443C46000986044B2E7104AC1
:108FC000E169F7F77DF823008C3318700020C7E7BC
:108FD0000023623401202370CAE70122094B0020DC
:108FE0001A70C5E732080020D007002026030000D1
:108FF00000180060C000002060080020FFFFFFBFD5
:1090000035060000740800200023F0B5040087B086
:10901000039002910B70002C00D18CE0257B002D79
:1090200000D18FE0EFF31083059372B6FFF736FEA1
:109030000020FFF7F1FE2668676830003900434BD7
:109040009C46434B1A685B68801A994100900191D5
:10905000019B002B05DC00D070E0009B002B00D1B1
:109060006CE061466346A031086800219B6D801961
:10907000794104936346DB6D994203D811D1049A78
:1090800090420ED9334831490078002809D09F42D8
:1090900006D802D1049B9E4202D801239D310B7059
:1090A00000252A4B2C4A99690098F7F709F82B4BB1
:1090B0001A69202800D22020083280188022D86225
:1090C000996A92051143996280211E6BC9050E436E
:1090D0001E63C0260327F605B446F6683E40022EFE
:1090E00022D06646F6683E40BE421DD0002D1BD001
:1090F0001B4D7C372E793E402E710026AE75EE75E5
:109100000F25A8435862986A083DA8439862986A58
:1091100001439962996A0A439A62124A0D4B117887
:1091200018781E7001431170059B83F31088029B11
:109130001B78002B08D1200007B0F0BD0123029A54
:109140001370F1E7246966E7039CF4E7D007002079
:10915000500800203108002026030000001800609D
:10916000C00000203208002073B56B460B4EDD1D99
:10917000290030680A4CFFF747FF2B783060012B3D
:109180000BD12300210099331B789A3109785A1C9E
:109190008A4200D0D3B29934237073BD6408002092
:1091A000D0070020F0B585B002A9CD1D0021012413
:1091B00029700192067B2100002E1ED11E490473E6
:1091C0000F681E4C390002604360002908D04A68CD
:1091D0009A4215D304D10A689446019A94450FD354
:1091E0000161002E0FD12900FFF70EFF23009433F9
:1091F00018602B78002B0CD12978080005B0F0BD41
:109200000E000969E1E730618742ECD0FFF7ACFF5F
:10921000F2E7EFF3108172B62300200099331B7838
:109220009A3000785A1C824200D0D3B2993423700D
:1092300081F31088E0E7C04664080020D0070020D2
:1092400010B50E4C217B00290AD12378002B05D0C4
:1092500001220B4B186902431A61996001232373A1
:10926000FFF71CFD00216420803422686368121817
:109270004B410448FFF796FF10BDC046D0070020C1
:109280000010006010080020C023DB0570B504004A
:109290005E69EFF3108572B6FFF700FD0B4B0C4AC9
:1092A000106851681A008832206061601068D969BE
:1092B000084A801BF6F704FF85F310880200206837
:1092C00061680023801A994170BDC046D007002014
:1092D0005008002035060000C023F7B50321002701
:1092E000DB05DA681F4E8A43DA60DA688A43DA609F
:1092F0001D4A1E49936A0B4093621D4B1F70330039
:1093000062331F80EFF31083019372B6B46DF56D75
:10931000FFF7C4FC330080331A685B68A41A9D41D0
:109320003B008C363278A41A9D41019B83F3108850
:10933000104B5B68DB05DB0D222B01D0FFF714FF20
:10934000002D02DC0BD1002C09D00120002D02DC05
:1093500002D10E2C00D900204000C0B2FEBD012079
:10936000FCE7C046D007002000180060FFFFFFBFE9
:109370003108002000ED00E0EFF3108072B6074BDB
:109380001A69C0230432DB051A610322D9689143AC
:10939000013A0A43DA6080F31088704700180060D1
:1093A000C0210322C905CB6810B51340022B05D09C
:1093B000CB681340934201D0FFF7D6FE10BD0000EA
:1093C000054A064B1178002901D0002111700022B6
:1093D00063331A707047C04631080020D007002060
:1093E00010B5034B034AD969F6F76AFE10BDC046B3
:1093F000D007002035060000F8B50123574D0600C0
:10940000EA6C1A43EA64AA6C1A43AA648021544A9B
:1094100009041160802149031160696C1943696472
:10942000296C0B432B6480235B04136002884D4C32
:109430004D49131CC72A00D8C82377689BB20B601C
:109440003B005A1E93412370002F02D1B378002BAA
:109450001BD00122454B19691142FCD017215960DC
:1094600019690A431A6100229A600132196911428E
:10947000FCD03F48FFF7D2FBE3692362002F0FD1F6
:10948000A020C005FFF7ACFF16E0C8235B032362F2
:10949000E361384BA361384B2361384B6361EFE7DD
:1094A00038030A21F6F7E0FE070060603448FFF752
:1094B00097FF874250D26068002360603088314A4D
:1094C000A1692373A066F6F7FBFD102800DA1020CF
:1094D00080235B01984200DB2B482300002200110F
:1094E0008C33A8601A702B692500A367230000261F
:1094F000002730338035A1691A706068214A2E60D8
:109500006F6026676767F6F7DBFD230022789C33E0
:109510001A702300002294331A602300012198332B
:109520001960230061331A70230062331A80174BCD
:10953000A665E765A060A3646265FFF7AFFB2868D6
:1095400069680023626812184B411148FFF72AFE30
:109550000120FFF7D9FBF8BD094893E70018006028
:1095600000E100E0D007002070080020001000603B
:10957000E0070020C2F528008D5B0000ECEB6501E0
:10958000FFEFFFFF26030000FF0F000041920410D1
:109590001008002010B5FFF781FB024B18685968CE
:1095A00010BDC0465008002070B5FFF7FBFD064D0A
:1095B00004002B78002B04D10448FFF741FE01235F
:1095C0002B70200070BDC0466808002010080020E5
:1095D00037B51B4A0300126800251100194C0029F9
:1095E00005D08B4226D118699A4201D0286110001B
:1095F0006946CD1D00212970197382421DD02900B2
:10960000FFF702FD2300943318602B78002B10D055
:10961000EFF3108172B62300200099331B789A3043
:1096200000785A1C824200D0D3B29934237081F35F
:10963000108837BD0D000969D1E794342260F8E73E
:1096400064080020D00700200023F0B593B006AADC
:10965000D3717A4B7A4C1B78019323009A331B7891
:109660000293029A019B934237D1237B002B00D1B6
:10967000C4E0744B1B69DB072DD500232373230043
:109680009C331A78002A00D081E023009B3319789C
:10969000002900D17BE01A702300A4331A78002A35
:1096A00005D000221A702300013262331A700120A3
:1096B000FFF7B2FB644D2800FFF78AFFFFF7EEFAD1
:1096C00021000023626880310868496812184B4104
:1096D0002800FFF767FD13B0F0BD230094331F6827
:1096E00000253E000395002E18D0337B002B03D1BC
:1096F000039601353669F6E732687368049205937C
:10970000FFF7CCFA04980599504B1A685B68801AE9
:109710009941002902DCEBD10528E9D9281E04D0A3
:10972000002338003700039A1361494B1F6000285B
:1097300024D1250006AB9435D91D2868FFF764FCB9
:1097400006ABDB792860012B10D1EFF3108172B6E4
:109750002300200099331B789A3000785A1C8242EB
:1097600000D0D3B2354A137081F310889A3423782D
:10977000019AD318029A9B1A23706AE70023037395
:1097800083680669002B00D098473000CFE7237824
:10979000002B2BD008AD2800FFF740FAAE68A06E72
:1097A00031002C4A80B2F6F78BFC102800DA10202A
:1097B00080235B01984200DB2748284B001198600A
:1097C000EFF3108772B62300012230331A706B68F2
:1097D000A6616361089B2361EB68E361FFF7D8FA38
:1097E00087F310880020FFF78FFA55E7EFF3108515
:1097F00072B6FFF7CDFA85F310884DE72378002B7A
:1098000000D168E7FFF74AFA226F636F2100FA245C
:1098100000256403A4185D4180314868A84205D83A
:1098200000D058E70B68A34200D854E7064C20004C
:10983000FFF7CEFE2000FFF703FD4CE7690800208C
:10984000D007002000100060100800205008002001
:109850006408002026030000FF0F000000180060CD
:10986000002313B50E4901930B700E4B019A0E485D
:10987000196B0E4A014019631100140099310978DF
:109880009A342478481CA04200D0C1B29932117099
:109890000121DA6C0A43DA64DB6C0B40019313BDDF
:1098A0006D08002000180060FFFFFFBFD0070020F8
:1098B00013B5002401200194019BFFF7ADFA084B7A
:1098C0001A78A24202D01C70FFF7CAFF0121054B93
:1098D0005A6C0A435A645B6C0B40019313BDC0463B
:1098E0006D0800200018006010B50400FFF7D6F9DD
:1098F000044A2000136851689C429B415B42C9188E
:1099000010BDC046500800204B1E9941F0B5434B96
:10991000434C85B01970531E9A41230060331A706E
:109920002300002261331A702300013262331A804F
:10993000EFF3108572B6FFF7D7FF230080331A6864
:109940005B6806000F00801A994100920193A6659A
:10995000E7650200002902D132498A4207D9002373
:109960006234237085F31088012005B0F0BD21001A
:1099700094310B689C46002B10D11800FFF74CFA6D
:10998000060085F3108898342378002B04D12648EC
:10999000FFF756FC012323703000E6E71A685B6886
:1099A00002920393039B019A9A4215D803D1029B1A
:1099B000009A9A4210D821000023A0310A68029828
:1099C000039912184B41BB4206D801D1B24203D8C9
:1099D00063461B7B002B16D10020FFF71DFA2300E6
:1099E00094331B68E26D596806009142C9D803D1CF
:1099F0001968A26D9142C4D81B7B002BC1D00122F3
:109A00000A4B1A70BDE77F210026094B1A790A40DC
:109A10001A719E75DE75FFF7A7FBB2E734080020C8
:109A2000D007002065FEFFFF100800206D08002011
:109A3000C000002010B5FFF713FF02F0EFFC10BDCF
:109A400010B502F0E7FCFFF733FF10BD002382B032
:109A50000193019BC0230122DB05596F0A435A671A
:109A60005B6F019302B07047024B18688003C00F10
:109A70007047C046000040480421044B9A688A435E
:109A80009A609A6802398A439A6070470000404899
:109A9000024B18684005C00F7047C04600004048A0
:109AA000F8B505000120002D00D194E02B68DB06FD
:109AB00066D42B68DB0723D5924B93491868934AE9
:109AC0000840802189010143196080211868014301
:109AD000196070211868884340390143196080215A
:109AE0006B6849028B4200D076E011680B4313602B
:109AF000FCF702FE0400FFF7B7FF002800D180E06A
:109B000004222B68134200D082E02B689B0700D40C
:109B1000CBE004227D4C23689343236023680C32FE
:109B200093432360202322681A42FCD1784A794863
:109B3000916A01409162D16A0140D162A168764A7E
:109B40001140802212020A436021A260E2688A4327
:109B50001343E360EB682268102B00D091E01343BD
:109B60002360FCF7C9FD2027060023683B4200D094
:109B70009BE0FCF7C1FD694B801B9842F5D929E0B9
:109B8000A96800290ED1FFF777FFFCF7B5FD0400A7
:109B9000FFF77EFF01288CD0FCF7AEFD001B642888
:109BA000F6D917E00222594B986802439A600422C2
:109BB000986802439A600429E7D1FCF79DFD0400F0
:109BC000FFF766FF012800D073E7FCF795FD001B47
:109BD0006428F5D90320F8BD11685148014011608F
:109BE000002B00D084E7FCF787FD0400FFF73CFF63
:109BF000002800D184E7FCF77FFD001B6428F5D91D
:109C0000E8E7FCF779FD001B642800D873E7E1E77B
:109C10002B693E4C002B23D02368934323600823F9
:109C200022681A42FCD1102223680827934323603C
:109C3000A268394B1A4080235B021343A3600423BC
:109C4000226813432360FCF757FD060023683B425C
:109C500000D05AE7FCF750FD801B0228F6D9B9E77F
:109C60002368082793432360FCF746FD060023681A
:109C70003B4200D149E7FCF73FFD801B0228F6D9A3
:109C8000A8E710218A432260002B00D069E7FCF787
:109C900033FD2027060023683B4206D0FCF72CFD4D
:109CA0001E4B801B9842F6D994E72B681B0701D402
:109CB000002090E7154C6B692268402B0FD11343AD
:109CC0002360FCF719FD4026050023683342EFD1DD
:109CD000FCF712FD114A401B9042F6D97AE7402565
:109CE000AA432260002BECD1FCF706FD0600236896
:109CF0002B42DDD0FCF700FD084A801B9042F6D9CC
:109D000068E7C04698004048FFC0FFFF0000404899
:109D100000005048FFCFFFFFFF7FFEFF88130000C9
:109D2000FFFFFEFFF0B504000D0085B0002802D152
:109D3000012005B0F0BD3022474E736893430B43BA
:109D400073600368022B21D1FFF796FEFFF7A0FE98
:109D50000028EDD0414A424913680B40E0211360CE
:109D600093688B4361680B4393603024736823408E
:109D7000AB425CD100230293029B052B68DDFCF70C
:109D800099F9FCF7BFFCFCF777FCD2E7002B23D155
:109D9000FFF77EFE0028CBD0FFF766FE0028C7D075
:109DA00080232E4F9B013A6813433B60FCF7A4FCD1
:109DB000019080223B68D201134207D1FCF79CFC42
:109DC000019BC01A0228F4D90320B2E7E022BB6845
:109DD000934362681343BB602368012BC5D1802382
:109DE0001E4F9B023A681A42FCD00223BA68134302
:109DF000BB6000230393039B052B14DD0423BA6887
:109E00001343BB60FFF744FE002800D090E7FFF744
:109E10002BFE002800D18BE7E022BB6893436268E9
:109E20001343BB60A1E7C046039B0133E2E77368BD
:109E3000A3432B437360FCF75FFC07007368234068
:109E4000AB4297D0FCF758FCC01B0228F6D9BBE701
:109E5000C046029B01338EE70010004000004048DE
:109E6000FFDFFFFF014B18687047C046B8140020A1
:109E7000036810B5DA0706D5062416490A6EA24310
:109E8000046922430A669A0706D51249124C8A6869
:109E90002240446922438A605A0706D50D490F4C77
:109EA0008A682240446822438A601B0706D5094A13
:109EB0000B4993680B4081680B439360C1688B0624
:109EC00005D5044A0748936803400B43936000207C
:109ED00010BDC04600004048FFEFFFFFFFFF7FFFBF
:109EE000FFFFBFFFFF7FFEFF10B504000120002C25
:109EF00019D0637ADAB2002B03D120002272FBF76B
:109F000053FF0223002008216372236818601A6837
:109F10008A4361680A4304211A601A688A431A60F6
:109F200001236372E06010BDF8B50B4A03680400BA
:109F3000DA60FCF7E1FBFA2705002026BF00236862
:109F4000DB68334201D00020F8BDFCF7D5FB401B95
:109F5000B842F4D90320F7E75D050100F7B54026C4
:109F600003680400DA68002532420ED18022D968E5
:109F7000FA270A43DA60FCF7BFFBBF0001902368B1
:109F8000DB68334201D1012D01D12800FEBDFCF771
:109F9000B3FB019BC01AB842F1D9042301256376B3
:109FA000EDE78021036810B5DA6804008A43DA60BF
:109FB0009B689B0601D5002010BDFFF7B5FF002868
:109FC000F9D0042301206376F6E7000010B5041EE3
:109FD00001D1012010BD437EDAB2002B02D10276FE
:109FE000FBF710FF022363762368DA68D20603D5F5
:109FF000012300206376EDE7CA225A62773A2000F7
:10A000005A62FFF7ABFF002816D123680D499A6802
:10A0100020690A409A606268996802436069024355
:10A020000A439A60E26820001A61A2681969120462
:10A030000A431A61FFF7B5FFFF2223685A6200281E
:10A04000D6D0C6E7BFFF8FFFF0B50E0085B0150074
:10A050000400FCF751FBAD192D1AFCF74DFB8027CE
:10A06000254B01901B685B011B0D6B43039322681A
:10A070009368180038403B4232D0731CF8D0FCF78C
:10A080003BFB019BC01AA8422CD3E02123685A68ED
:10A090008A435A6082226168520091420CD1802129
:10A0A000A26809028A4203D08021C9008A4203D1F2
:10A0B00040211A688A431A608021A26A89018A4273
:10A0C00006D119680D480140196019680A431A60E1
:10A0D000230001225D331A70002303205C342370B7
:10A0E00005B0F0BD039B002B03D0039B013B039302
:10A0F000BDE71D00BBE7C046B8140020FFDFFFFF2F
:10A10000F0B51D00002385B0170002AAD37004002B
:10A110000E00FCF7F1FAED192D1AFCF7EDFA2322E7
:10A120002368009001932A4B1B6853431B0D6B431C
:10A13000039302AB2168DA1C8B681800304033426D
:10A140003BD0C023DB009E4204D1019B1B7BDBB2D2
:10A15000137013787B1CEFD0FCF7CEFA009BC01A6B
:10A16000A8422CD3E02123685A688A435A6082228D
:10A170006168520091420CD18021A26809028A4292
:10A1800003D08021C9008A4203D140211A688A4342
:10A190001A608021A26A89018A4206D119680D4895
:10A1A0000140196019680A431A60230001225D33D7
:10A1B0001A70002303205C34237005B0F0BD039BAC
:10A1C000002B02D0039B013BB2E71D00B1E7C04664
:10A1D000B8140020FFDFFFFF70B513000D0016005C
:10A1E0000A00C02149010400FFF78AFF002805D0BA
:10A1F00020230320226E1343236670BD3200290002
:10A200002000FFF721FF0028F2D1C02133002A00EF
:10A210002000C900FFF774FF0028EED0E8E7000037
:10A22000F8B504000120002C67D0636A002B65D1CB
:10A23000822261685200914200D0E3610023250030
:10A24000A3625D352B78DAB2002B05D123005C3395
:10A2500020001A70FBF726FE022340222B70216893
:10A26000E6680B689343E0220B60D200002396421D
:10A2700048D9F02218001201964200D0A36282222F
:10A280008427636852001340A2683F023A400227C5
:10A2900013432269A5693A401343012267691740B5
:10A2A0003B438027BF002F403B43E76937321740CD
:10A2B0003B43276A4832174080223B43A76A9201FA
:10A2C00017403B43102708220B60636A2D0C3B406C
:10A2D000676B17403B43F0273F013E403343042662
:10A2E00035402B4303434B60CB69084803400020B3
:10A2F000CB61012320665D342370F8BD0023236108
:10A3000063619BE780204001B6E7C046FFF7FFFF8F
:10A31000F0B5040085B01E000D001700FCF7ECF945
:10A3200023005D33009001931B78D8B2012B00D03D
:10A33000B1E0002D00D17FE0002F00D17CE02300B0
:10A340005C331A78012A00D1A5E018700323019A22
:10A3500013700023A21D23662364A563A787E787E4
:10A3600002329387D3878022A1682365E3641202B7
:10A370002368914208D140211A688A431A608022DA
:10A380001968D2010A431A6040221968114202D1A9
:10A3900019680A431A60E021E0686268C9008842CF
:10A3A0004CD9002A01D0012F07D12A880235DA6062
:10A3B000E38FA563013B9BB2E38702250CE0226893
:10A3C00093682B4228D0A36B19880233D160A36312
:10A3D000E38F013B9BB2E387E38F002BEFD131008A
:10A3E0002000009AFFF7F8FE002851D1A368002B47
:10A3F00006D103932368DA6803929B680393039B57
:10A400000123019A1370230000225C331A70206E1E
:10A41000431E9841C0B20FE0FCF76EF9009BC01AD2
:10A42000B042D9D3731CD7D0230001225D331A70F8
:10A43000002303205C34237005B0F0BD002A01D056
:10A44000012F08D12A781A73A36B0133A363E38F1A
:10A45000013B9BB2E38702250DE023689A682A42FC
:10A460000DD0A26B12781A73A36B0133A363E38F31
:10A47000013B9BB2E387E38F002BEED1AFE7FCF704
:10A480003BF9009BC01AB042F5D3731CF3D0CBE765
:10A4900020232366AAE70220CEE700000E4A10B56B
:10A4A0000368904207D17024A3434C6823430B4CAC
:10A4B0002340CC6823438024A3434C692343036097
:10A4C0008B68C3620B688362904201D10B6903639E
:10A4D0000123436110BDC04600200040FFFCFFFF88
:10A4E000704770B504000120002C21D0A37FDAB2A0
:10A4F000002B03D120006277FFF7F2FF0223251D16
:10A500002068A3772900FFF7C9FF01230020E21884
:10A51000E377D377A21CD377E21CD377621DEB7766
:10A52000D377A21DD377E21DD377D218D377A37741
:10A5300070BD0000817F03000120CAB2814214D1A6
:10A54000022199771B68D9681143D96007498B426A
:10A5500007D1996806480140062905D0073881428D
:10A5600002D019680A431A6000207047002000409A
:10A57000070001000121036810B5DA688A43DA6038
:10A580001C6A074A144206D11C6A064A144202D1C8
:10A590001A688A431A6001238377002010BDC046E1
:10A5A0001111110044040000704770477047704754
:10A5B0000222036870B5DD681E69040016420DD0E2
:10A5C00015420BD0053A1A61043202779B699B074A
:10A5D00000D17CE0FFF7E9FF0023237704231E422C
:10A5E00012D01D4210D00522236852421A61073250
:10A5F00022779A69C0239B0020001A4200D16CE0A8
:10A60000FFF7D3FF0023237708231E420FD01D42FC
:10A610000DD00922236852421A610D322277DB697C
:10A6200020009B075FD0FFF7C0FF00232377102394
:10A630001E4211D01D420FD01122236852421A61CE
:10A6400019322277DA69C0239B0020001A4250D0C9
:10A65000FFF7ABFF0023237701231E4208D01D42E2
:10A6600006D002222368524220001A61FAF778FDD0
:10A6700080231E4208D01D4206D081222368524208
:10A6800020001A6100F03FF8F30507D52B0605D529
:10A6900023681B4A20001A6100F036F840231E424E
:10A6A00008D01D4206D041222368524220001A6180
:10A6B000FFF77DFF20231E4208D01D4206D0212235
:10A6C0002368524220001A6100F01CF870BDFFF7A9
:10A6D0006BFF2000FFF76AFF7EE7FFF765FF2000B2
:10A6E000FFF764FF8EE7FFF75FFF2000FFF75EFFD5
:10A6F0009BE7FFF759FF2000FFF758FFAAE7C04686
:10A70000FFFEFFFF704770477047704730B5EFF3AB
:10A710001084012282F310880168134D0B682B40CE
:10A720000B6084F31088EFF3108182F310880268C5
:10A730000E4C93682340936081F31088C36E012B05
:10A740000AD1EFF3108183F3108810240268136894
:10A75000A343136081F31088030020228C331A6016
:10A760000023C366436730BDDFFEFFFFFEFFFFEF40
:10A770007047704770477047704770477047704721
:10A7800003000C4A94331A600B4ABC305A600B4ADF
:10A790009A600B4ADA600B4A1A610B4A5A610B4AFB
:10A7A0009A610B4ADA610B4A1A620B4A5A620B4BE6
:10A7B0000360704771A7041073A7041075A70410F5
:10A7C00077A7041079A704107BA704107DA70410B5
:10A7D0007FA70410F1AC0410F3AC04100BA7041015
:10A7E000F0B5C36985B001690093836805680B43C0
:10A7F00041692A680B4300993D4F0B433D490400D2
:10A800000A4013432B606B683B4A1340C2681343F2
:10A810006B608269BD4201D0036A1A43AB68374955
:10A8200037480B400F211343AB60EB6A626A8B43DE
:10A830001343EB62334B5200D35A19000393F5F7DD
:10A8400013FD6668BD4225D103237343012783426C
:10A850003AD83303834237D30023039A0021284890
:10A86000F5F7E0FE03001A0E1802730800930023A8
:10A87000090211430193009A019B8018594132004B
:10A880000023F5F7CFFE204BC218204B9A421BD86D
:10A89000E86018E0802200997308120291421BD1EF
:10A8A0004000C0183100F5F7DFFC0300184A103BE8
:10A8B0000127934208D803000F22000793439BB25D
:10A8C000400F0343EB600027124B3800A3660023C0
:10A8D0006367A36705B0F0BD18183100F5F7C4FC35
:10A8E00003000B4A103B01279342EDD8D0E7C04646
:10A8F00000500041F369FFCFFFCFFFFFFFF4FF11CE
:10A900000024F4006252071000FDFFFFFFFC0F005F
:10A91000EFFF000001000100836A30B51A0706D579
:10A920000168284C4A682240846B22434A60DA0757
:10A9300006D50168244C4A682240C46A22434A6012
:10A940009A0706D50168214C4A682240046B2243CD
:10A950004A605A0706D501681D4C4A682240446B7C
:10A9600022434A60DA0606D501681A4C8A682240FA
:10A97000C46B22438A609A0606D50168164C8A6821
:10A980002240046C22438A605A0610D50168134D98
:10A990004A68446C2A4022434A608022520394420F
:10A9A00005D14A680E4C2240846C22434A601B0643
:10A9B00006D502680B4953680B40C16C0B435360CA
:10A9C00030BDC046FF7FFFFFFFFFFDFFFFFFFEFF23
:10A9D000FFFFFBFFFFEFFFFFFFDFFFFFFFFFEFFFCB
:10A9E000FFFF9FFFFFFFF7FFF7B504000D00170003
:10A9F00000932268D3692B405B1B59424B41BB42F9
:10AA000001D0002026E0089B0133F3D0FBF774FE51
:10AA1000009BC01A089B98422DD8002B2BD023688E
:10AA20001A685207E5D52A004021403A8A43E0D00F
:10AA3000DA69082611003140019132420BD0200022
:10AA40001E62FFF763FE230090331E600023012087
:10AA500084342370FEBD8022D96912011142C8D00E
:10AA60001A622000FFF752FE2300202290331A6062
:10AA7000019B843423700320ECE7F0B5070087B016
:10AA8000883705933B6804000D0016000220202B38
:10AA900002D1002902D1012007B0F0BD002AFAD06E
:10AAA0008023A2685B019A4204D12369002B01D163
:10AAB000CB07F0D42300002290331A6021233B609F
:10AAC000FBF71AFE230054331E8002331E800393CB
:10AAD0008023A268002604905B019A4204D1236976
:10AAE000B34201D12E001D00230056331B889AB2B9
:10AAF000002B0CD1059B200000934021049BFFF705
:10AB000073FF2023883423600028C5D00CE0059B08
:10AB10000022009380212000049BFFF765FF00289E
:10AB200004D02023883423600320B5E72268002D59
:10AB300010D133880236DB05DB0D936221223B689E
:10AB400013409342A7D1039B039A1B88013B9BB2FE
:10AB50001380C9E72B7801359362EFE7030073B5E3
:10AB60000026040090331E60FBF7C6FD2368050035
:10AB70001B681B071FD58021284B320000938903D7
:10AB800003002000FFF730FFB04214D0EFF3108134
:10AB9000012383F3108880202268136883431360A5
:10ABA00081F310882300202288331A6003200023B9
:10ABB0008434237076BD260023688C361B685B07BF
:10ABC00023D58021154B0022009320002B00C903C0
:10ABD000FFF70AFF002818D0EFF31080012282F35C
:10ABE000108821680E4D0B682B400B6080F3108895
:10ABF000EFF3108082F3108821688B6893438B6099
:10AC000080F3108820233360D0E723002022002027
:10AC100088331A603260E0662067C8E7FFFFFF01F3
:10AC2000DFFEFFFF70B5041E01D1012070BD0500DD
:10AC300088352B68002B0DD1020084321370FFF78A
:10AC40009FFD2200C0321368002B01D1124B13600C
:10AC500020009847242301222B6025682B6893430A
:10AC60002B60A36A002B02D02000FFF755FE2000C6
:10AC7000FFF7B6FD0128D8D06B68084A20001340C2
:10AC80002A226B60AB689343AB6001232A681343AD
:10AC90002B60FFF763FFC9E709640410FFB7FFFFEC
:10ACA000F7B50700436E04006A37002B04D101207A
:10ACB000388068342080F7BD03680B4E9A689B6823
:10ACC0000A4D5B0FF05CE95CC0000192F5F756FBA2
:10ACD000019B38801B015B0FF05CE95CC000F5F75D
:10ACE0004DFB80B2E5E7C046825207107A5207104A
:10ACF0007047704770B50400843422780300022046
:10AD0000012A11D01D002422012688352A601A68E4
:10AD100011681068B0431060044801400020586674
:10AD2000202311602B60207070BDC046FFFFFFDF45
:10AD3000F8B5050084350B0029780222012915D0C9
:10AD400006000121046888362232326027682268B2
:10AD50008A432260A168C900C9081943A160FFF7AE
:10AD60009FFF20230022276033602A701000F8BD67
:10AD7000F8B5050084350A0029780223012915D089
:10AD8000060001210468883622333360276823686F
:10AD90008B432360A168064B19401143A160FFF764
:10ADA0007FFF20232760336000232B701800F8BD3D
:10ADB000FFFFFFF1064A137E062B05D0990088504D
:10ADC000002001331376704701204042FBE7C04664
:10ADD00078080020037870B50400042B05D0822B7E
:10ADE0000ED0200001F0C4FD70BDC61C6378FF2B9F
:10ADF000F7D173789B08032BF3D10025280009E0D5
:10AE0000061DF3E7AA003000D35898470128EBD07D
:10AE10000135EDB2034B1A7EAA42F3D80028E0D0E8
:10AE2000E2E7C0467808002010B507F001FC10BD2D
:10AE300010B507F0A3FC10BD10B507F0F7FC10BD6E
:10AE400010B507F02DFD10BD10B507F04BFD10BD7E
:10AE500010B507F06DFD10BD10B507F08DFD10BDEC
:10AE600010B507F09DFD10BD10B507F04DFE10BDEB
:10AE700010B508F095F810BD10B506F00BFB10BD2D
:10AE800010B506F031FB10BD10B50BF00FFB10BD77
:10AE900010B50BF0F5FC10BD10B50BF004FD10BDA6
:10AEA00010B50BF030FD10BD10B50BF02EFD10BD30
:10AEB00010B506F049FB10BD10B506F009FF10BD36
:10AEC00010B506F035FF10BD10B506F04DFF10BDF2
:10AED00010B506F065FF10BD10B506F0A1FF10BD5E
:10AEE00010B506F0E3FF10BD10B507F00FF810BD68
:10AEF00010B507F029F810BD10B507F041F810BDE6
:10AF000010B515F0F7F810BD10B518F0E5FC10BD40
:10AF100010B518F089FC10BD10B518F09DFC10BDDF
:10AF200010B50BF05FFF10BD37B506AC07AD2D783F
:10AF30002478019500940CF05BFB37BD10B50DF043
:10AF40006BFF10BD10B50EF017FB10BD10B50EF065
:10AF5000E7FF10BD10B50FF02FF810BD10B50FF0C2
:10AF600011FB10BD10B50FF065FB10BD10B50FF053
:10AF7000A5FE10BD10B510F07FFA10BD10B510F091
:10AF8000CDFB10BD10B510F0BDFD10BD10B510F01B
:10AF90003DFE10BD10B511F055FF10BD10B511F0FC
:10AFA000A1FF10BD10B512F08FFA10BD10B512F050
:10AFB000D5FA10BD10B512F013FB10BD10B512F08C
:10AFC00049FA10BD10B512F04FFA10BD10B512F0CD
:10AFD00099FE10BD10B513F049FF10BD10B514F067
:10AFE000D9F810BD10B511F05BFE10BDF0B58DB0F5
:10AFF00012AC247809930A9413AC247818AB1B780C
:10B000000B9415AD14AC16AE17AF24782D783678A6
:10B010003F7806930B9B059701930A9B0496009338
:10B020000395099B029414F0E3FB0DB0F0BD10B53D
:10B0300016F0EDF910BD10B516F02CFA10BD10B5D4
:10B0400016F034FB10BD10B516F066FD10BD10B53E
:10B0500016F0D0FF10BD10B516F0ACFD10BD10B548
:10B0600016F0C0FD10BD10B516F0E4FD10BD10B512
:10B0700017F018F810BD10B517F034F810BD10B562
:10B0800017F052FA10BD10B517F08EFA10BD10B5BA
:10B0900017F06CFB10BD10B517F07EFD10BD10B59C
:10B0A00017F0B4FD10BD10B517F092FE10BD10B52D
:10B0B00017F0A6FE10BD10B517F0CAFE10BD10B5F2
:10B0C00017F0CAFE10BD10B517F0EEFF10BD10B599
:10B0D00017F0BFFF10BD10B517F084FF10BD10B5FD
:10B0E00018F0CCF810BD10B508F006FB10BD10B577
:10B0F00008F06EFB10BD10B508F0DEFB10BD10B5FA
:10B1000008F01AFF10BD10B50AF04EF810BD10B5CA
:10B110000AF004F910BD10B505F0BEFE10BD37B53C
:10B1200006AC07AD2D8824880195009405F0B8FE83
:10B130003EBD7FB508AC09AD0AAE24882D8836889F
:10B1400001950296009405F0BDFE04B070BD10B5E7
:10B1500005F0CBFE10BD10B505F0D0FE10BD10B54A
:10B1600005F0E2FE10BD10B505F047FF10BD7FB53C
:10B1700008AC09AD0AAE24782D7836780195029690
:10B18000009405F043FF04B070BD10B505F082FFD8
:10B1900010BD10B505F08AFF10BD10B505F08EFF8B
:10B1A00010BD10B505F08EFF10BD10B505F08EFF77
:10B1B00010BD10B505F08EFF10BD37B506AC248864
:10B1C000079D0094019505F089FF3EBD37B506AC9B
:10B1D0002488079D0094019505F08FFF3EBD10B5B2
:10B1E00005F094FF10BD10B505F094FF10BD13B528
:10B1F000049C009405F096FF16BD13B5049C0094C2
:10B2000005F09FFF16BD13B504AC2488009406F02A
:10B21000B3F816BDF0B589B007930EAC0FAD10AE04
:10B2200011AF12AB24882D8836883F781B7803979E
:10B2300004930296079B0195009406F0AAF809B0C2
:10B24000F0BD10B50BF01CF910BD10B50BF01CFBD8
:10B2500010BD13B504AC248800940BF019FB16BD87
:10B2600030B50C008DB011006B46103115780132ED
:10B27000DD73013B9142F9D1010004AB0C310A6846
:10B28000150A1A705D70150C120EDA709D700A00A6
:10B29000043304399042F2D1694608AA04A800F0A8
:10B2A0002DF8210008AB0C31DA78987812060004EA
:10B2B00002431878024358780433000202430A60BC
:10B2C0000A0004399442EFD10DB030BD01220A4B7F
:10B2D00082B0196E11420CD1196C11431964196CAA
:10B2E00091431964196E114319661B6E1340019343
:10B2F000019B002002B0704700004048F0B5642573
:10B300001F4E85B03378AC460133DBB23370C023B7
:10B3100002ACDB05073435780127EDB201950D68E5
:10B320009D624D68DD628D681D63CD685D63056853
:10B330009D634568DD6385681D64C5685D64654619
:10B3400025709D6D3D439D6501272578013DEDB23A
:10B350002570DD6D3D4202D02578002DF4D1257891
:10B360009D6C019F1560DD6C55601D6D95605D6D78
:10B37000D5603578BD42CED1002005B0F0BDC046C5
:10B38000940800200200202330B5013BD55CCC5C42
:10B39000281BA54201D1002BF7D130BD10B500F01C
:10B3A000CDFC00F0E7FC10BD70B5254D90B0060057
:10B3B00020220C00684629001EF0B3F92900202243
:10B3C000203108A81EF0ADF9012E1CD108A92000DB
:10B3D000FFF7D8FF1B4904220B78002804DB1A432F
:10B3E0000A70012010B070BD9343174A1549A41A82
:10B3F0000B70110013002031E25804C39942FBD1B5
:10B4000000200860EEE7022E0BD169462000FFF70E
:10B41000B9FF0C4901220B780028E0DA93430B4A6C
:10B42000E4E7032EDDD169462000FFF7ABFF0549B5
:10B4300002220B780028D2DA9343054AD6E7C046A9
:10B4400070B806109C0800206C0430489004304806
:10B45000B4043048421E03000120022A0AD82330D7
:10B460005843054BC0180023C25CCA540133202B3B
:10B47000FAD100207047C0464804304810B500F0AB
:10B4800043FC0822064B99680A439A600422996893
:10B490000A439A60012299680A439A6010BDC04627
:10B4A00000003048F8B506000D00170000F034FC2D
:10B4B000041E23D1124B310001201F60FFF774FFDF
:10B4C000012804D100F03AFC0324644214E029006E
:10B4D0000220FFF769FF0128F4D029000320203162
:10B4E000FFF762FF0128EDD00121064B1A680A43DD
:10B4F0001A601A688A431A602000F8BD0224E4E743
:10B500009808002000003048054B01201B78002BD4
:10B5100004D1044B1868431E9841C0B27047C0461E
:10B520009C0800200004304870B5FFF7EDFF124C76
:10B53000124D012809D100F001FC03230420210051
:10B5400023602B684042984770BD60220021200094
:10B550001EF03EF821000120FFF77CFF0849022081
:10B56000FFF778FF07490320FFF774FF00F0E6FBC1
:10B57000210000202B68E6E7A008002098080020A2
:10B58000C0080020E008002010B500F0D7FBFFF74E
:10B59000CBFF00F0EFFB10BD80210C4BC9021A6DF0
:10B5A00082B00A431A651B6D0B4004210193019B75
:10B5B000074B1A688A431A60012259681142FCD06D
:10B5C00058684007C00F02B07047C04600004048AE
:10B5D000000060480122044B59681142FCD09B686E
:10B5E000038000207047C046000060480122074BDE
:10B5F00059681142FCD09A680280012259681142B0
:10B60000FCD09B68438000207047C0460000604823
:10B6100000230321026810B583608381837313784C
:10B62000FF2B05D14368043B9B1A8381002010BD8A
:10B63000FE2B0CD103890133038153884468033303
:10B640000B439B185A1C0633A342E8D3EEE7002BAA
:10B6500003D1438901334381EFE70320E7E7F7B5DF
:10B660001D0008AB1E8844682300002E03D001ABE8
:10B670005E80FE261E708668A64201D80420FEBDAC
:10B680001C78FF2CFAD000240327A446047B002C4E
:10B6900017D0644604731C78002CF7D0FE2C1ED102
:10B6A000FF2902D05C788C42F0D1416804311160EE
:10B6B0005A882A80099A002A01D05B7813700020EA
:10B6C000DDE75B88446803333B4301341C192300E6
:10B6D0004460A642D2D92478FF2CDCD1CEE70320E7
:10B6E000CDE7F0B50700150000268C08A400091B63
:10B6F00085B0CBB20193B4420EDC0123019A5B42C8
:10B70000291903A803931EF00CF8039AE1190020ED
:10B71000FBF78EF905B0F0BDA919042203A81EF0AD
:10B7200000F8B9190020039AFBF782F90436E2E722
:10B7300070B5050010006E681A00AB6804249E42C4
:10B7400013D23378FF2B10D02D7B0134002D0CD178
:10B75000FE2B0AD1738801348B4206D90431891932
:10B760001DF028FF431E98414442200070BD000098
:10B77000F8B5002514260127114C3200A379114990
:10B780005A435058002817D1012B15D820688446F9
:10B790005050A0888A186044506020891082584216
:10B7A00030404018FFF734FF002807D16B1C0C34E1
:10B7B0003D00022BE1D1F8BD0120FCE70320FAE7B0
:10B7C0008C520710040900200200012030B582428B
:10B7D0000AD814245443054BE5581B195B6888812B
:10B7E00000204D608B600A7030BDC0460409002007
:10B7F0001422F0B58D4C4243A54400248C4B079095
:10B800009B185B892000A34200D18EE00EAD290079
:10B810000798FFF7D9FF0F9B270003930123049498
:10B8200005938022FF21120112A81DF0D1FEFE22F5
:10B8300006AB1A74059B002B49D000247D4D832351
:10B840001B0106AAE3189B187B4AFF219B1805934E
:10B85000112306AA9B180193049B0EA800930E23A4
:10B860009B180BAAFFF7FBFE061E04D0042800D18C
:10B870009AE0032059E006ABDE89002E5FD02A0053
:10B88000B54200DD32000B9905981DF04AFF0AAB66
:10B890005E8083231B01E31806AA9B18674A04965F
:10B8A0009B180A9A1A600323F21C13430133E4180D
:10B8B000A4B20323F61B013E334301339BB2AB42D8
:10B8C00036D900237F19BFB20026059374E00F9983
:10B8D000049B0D00002B03D00BAD6B80FE232B705F
:10B8E000109B0EAA8B4200D899E02B78FF2B00D139
:10B8F00095E0127B002A17D1FE2B15D16A88BA4237
:10B900001DD94C4BD21B9A4200DD1A00032404318E
:10B91000C91912A81DF005FF6E88464DF31B013BA7
:10B920001C430134A4B2C4E70520454B9D44F0BD3F
:10B93000AB4236D03F4D00272D1BADB27FE706202E
:10B94000F3E7002C4BD00023049301330593042626
:10B950000694630533D000253A4A039B0AA99B1835
:10B96000DB0A0C93069B0BA85A1E374B0B9513430F
:10B970000133DB0A0D93FBF799F88322AB10120118
:10B980009B009B1806AA9B182C4A00209B18039A20
:10B99000A9181A68FBF74CF8069B04359D42ECD3B6
:10B9A00014E0002701238FE780231B019C42C8D1AC
:10B9B0000123059300230493802424010694069A0E
:10B9C000039812A91DF0F6FD0028C4D180221201AF
:10B9D0009446039B63440393002E00D121E7109A01
:10B9E000194B013A1343039A013316499B1A00225B
:10B9F0008C46FF211292039ADB0A6244D20A0A4063
:10BA00000B4012A80BA914931392FBF74FF81420C4
:10BA1000079B5843064BC018FFF7FAFD85E78023C4
:10BA20001B019C4293D10426C6E7C046B4F7FFFF32
:10BA300004090020FC07000004F8FFFF00F8FFFFE6
:10BA40004C0800000000FCEFFF070000F0B51500F7
:10BA50001422047887B0624303930CAB1F88124B07
:10BA60000A249B189B7B002B19D10D9A138002AAE4
:10BA7000A6180193009305AA3300FFF7F0FD041EFA
:10BA80000DD13688B5420DD2721BBA4200DD3A00A4
:10BA90000599039849191DF044FE0D9B1E80200056
:10BAA00007B0F0BD0624FAE704090020F8B5070046
:10BAB00014243D7810006C43134A069E1219927BA1
:10BAC0000A24002A1AD132807D68BA68063C954261
:10BAD00014D22A78FF2A11D03C7B002C10D1FE2AE8
:10BAE0000ED16A8891420DD2521A9A4200DD1A0094
:10BAF000043149191DF015FE6B8833802000F8BD14
:10BB00000524FBE70624F9E704090020F7B5060041
:10BB1000009282680320019308AB1F8875686B1D33
:10BB200093420AD314223178284B4A439B185B89ED
:10BB30000B20002B00D10938FEBD2B78FF2B38D10C
:10BB4000009B521B5C1E044380200134A4B2E31905
:10BB500003334002824200D31D4A9342E2DAFE22BE
:10BB600009023B191B040A431A432900002004352B
:10BB7000FAF75EFF21002800019AFFF7B2FD3900B5
:10BB8000099A6019FFF7ADFD142231780F4B4A4333
:10BB90009B181A89013F01321A81009A0321D71993
:10BBA000052239435242521A9989002052189A812B
:10BBB000C2E7FE2B01D0002B06D16B880135033381
:10BBC00003435D197560A9E70320B5E70409002068
:10BBD000FFFF00004168836810B50400042099420B
:10BBE00015D20B78FF2B12D00130FE2B0FD1084A53
:10BBF0000020FAF71DFF142200202178054B4A434C
:10BC00009B181A89013A1A815A8901325A8110BD4A
:10BC100000FFFFFF0409002030B5154A03009179A9
:10BC200085B0814203D0927C01209A421DD114221A
:10BC30005343104C00251A59E41861680E4B013922
:10BC40000B430E499B1A5218FF210133DB0AD20A1B
:10BC50000A400B4001A86946029203930195FAF746
:10BC600025FF2000FFF7D4FC280005B030BDC046FA
:10BC70008C52071004090020FF0700000000FCEFB1
:10BC8000064A0300917910B5814203D0927C0120CD
:10BC90009A4202D11800FFF7ABFD10BD8C5207107D
:10BCA000F8B5002414261549154D0C57E0B23200A2
:10BCB0004243AA185789431C002F15D09789128A2E
:10BCC000974211D25BB20B70022B08D100230120E6
:10BCD0000B70FFF7D5FF0B481DF07AFB02E043B273
:10BCE000002BF6DA0020F8BDD8B2022800D10020DF
:10BCF000A042DCD100230B70F4E7C046000900200D
:10BD000004090020F6DD06100122024B00201A6013
:10BD10007047C046C4140020EFF3108272B6064B81
:10BD20001968012905D100200231196082F31088B9
:10BD3000704702204042F9E7C4140020EFF310825C
:10BD400072B6064B1968032905D100200239196023
:10BD500082F31088704702204042F9E7C4140020A3
:10BD600010B5034B0A001900FFF79CFB10BDC0463D
:10BD7000A452071070470000F7B50E00140000270A
:10BD80000090019324257D43114BED182800FFF707
:10BD900010FA002803D0009B0130984204D00137EC
:10BDA000052FEFD11220FEBD2A6A33199188122087
:10BDB0008B42F8DC90680199220080191DF0B1FCDB
:10BDC0002B6A1A78920700D55C800020EBE7C0460A
:10BDD000F014002070B5040006480D001600FFF7AF
:10BDE000E8F9013033002A00210080B2FFF7C4FFD8
:10BDF00070BDC046F0140020F7B51E0000231500EA
:10BE00001380089A3380138005330191184202D1C0
:10BE100000242000FEBD124F3800FFF7BEF9041EBB
:10BE2000F7D11048FFF7C5F928800F48FFF7C1F98F
:10BE300030803800FFF7B5F9089B01001C80019B9A
:10BE4000022B05D00821094A0020FFF7C3FFDFE7D6
:10BE5000074B1800FFF7A9F9041EF3D0D9E7C04635
:10BE6000C8140020F01400201415002008530710F7
:10BE70005C15002070B5040006480D001600FFF7A1
:10BE800098F9013033002A00210080B2FFF774FFD7
:10BE900070BDC04614150020F8B50023154C0600EF
:10BEA0000B8020000D00FFF778F9002821D1200039
:10BEB000FFF777F9104F0400F60714D43800FFF7A6
:10BEC00078F9210028800D48FFF76FF9002810D17C
:10BED00021000B48FFF769F900280AD12100094821
:10BEE000FFF763F905E001003800FFF75EF900286D
:10BEF000E4D0F8BDBC1500207C5307105853071040
:10BF000034530710105307101F2070471F2070472D
:10BF100013B52C490B78002841D0002B1ED10122EB
:10BF20008024294B0A70596D6400214359655B6D6B
:10BF300023400193019B8023DB05196B1143196397
:10BF4000596B91435963D96A9143D962996B1143F3
:10BF50009963DA6380221D4B92041A6080221C4B85
:10BF60009200D969114219D1D969490516D4D96904
:10BF70000A43DA61042259691142FCD10F24D969BC
:10BF8000A143002800D00E220A43DA61DA69114980
:10BF90000A40DA61042259691142FCD013BD012B19
:10BFA000DCD1802280240870D205916BA4049943CF
:10BFB00091630949CC67BFF34F8FBFF36F8FD36392
:10BFC000CCE7C046650900200000404800E100E0E1
:10BFD00000005048FFFDFFFF04E100E00E4B1B781E
:10BFE000002B13D08023DB05DB6BDB070ED5A622ED
:10BFF0000A4B920098580221443AC00607D5985837
:10C000000143995080230122DB05DA637047985879
:10C0100088439850F6E7C046650900200014006088
:10C02000064B82B01B685B039B0F0193019B002BA7
:10C0300001D101330193019802B07047900050483C
:10C040008022D20510B5124904005068FF238842AF
:10C0500000D1FC3B0F21237013681B090B40637058
:10C0600013680B40A370536863600A4B1B689BB254
:10C0700001339B00A360FFF7D3FF002805D0FFF733
:10C08000CFFF01308003E06010BDC020C001FAE79F
:10C0900041E0010214100040AC23054A9B00D05837
:10C0A00003231840023843425841C0B27047C0468B
:10C0B0000014006010B5FDF7C7FA10BD10B5FFF70A
:10C0C000EFFD10BD10B5104C104B2188994203D1E3
:10C0D0000F481DF07DF910BD0E481DF009F904212F
:10C0E00003222088FFF77FF8011EF4D00A481DF0D4
:10C0F000FFF80A481DF06CF9208801F0A5FF012324
:10C100005B422380E7E7C04602160020FFFF0000E5
:10C110001ADE061051DE061090DE0610BBDE061099
:10C1200010B5012004F0A8FD05F0F1FA012004F09B
:10C13000A4FD10BD30B51C4D85B06B7C002B2BD001
:10C140001A481DF045F9102302930193FA239B002E
:10C1500028210093502200230120FEF7EAFF011E50
:10C16000134800D013481DF0C3F80120124AA97CDF
:10C17000FEF7EDFF041E11D1012310482B741DF0B2
:10C1800027F9042004F044FE0D4D2988002903D02E
:10C19000200003F06FF82C8005B030BD2100094865
:10C1A0001DF0A6F8F8E7C046840A0020E3DE06107A
:10C1B00002DF061046DF0610970A002089DF06100E
:10C1C000740A0020C1DF061010B504F041F9FFF732
:10C1D0009BFD013001D1F8F7EBFF10BD30B595B0F4
:10C1E0006A46062353740023042153836148624B3B
:10C1F000C8221DF07DF86149342207A81DF091FA8C
:10C2000007A805F069FB011E04D05D481DF070F819
:10C21000F8F7CEFF1F21002005F026F8011E00D1FF
:10C2200087E058481DF064F8122101206944FFF7A7
:10C2300033FE011E00D180E053481DF059F804215F
:10C2400052481DF055F852481DF0C2F80121002057
:10C2500004F01AFE011E00D173E04E481DF048F8AC
:10C2600006AB0093162300216B4405AA0420FFF7B8
:10C27000C3FD1123484C6B4422001900802004F0B8
:10C28000EFFF2578E3782279617902956578434854
:10C290000195A47800941DF02BF80A210020404A53
:10C2A000FFF798FD011E50D03E481DF021F81A23DB
:10C2B0006B4402211A000020FFF7DCFD011E48D06C
:10C2C00039481DF015F839481DF082F80522002084
:10C2D0001100FEF7BAFF011E3FD035481DF008F8E7
:10C2E00034481DF075F80120334C2070FEF73BFFF9
:10C2F000011E36D031481CF0FBFF314B002163801A
:10C300001023617023710193083B0A00029100938E
:10C3100001200B00FEF72BFF011E26D029481CF040
:10C32000E7FF29481DF054F828481DF051F815B0D2
:10C3300030BD27481DF04CF876E726481DF048F838
:10C340007DE725481DF044F88AE724481DF040F8B1
:10C35000ADE723481DF03CF8B5E722481DF038F85A
:10C36000BEE721481DF034F8C7E720481DF030F83B
:10C37000D7E7C046F5DF06105A440000B0B80610F3
:10C3800039E006105CE00610C9E0061034E1061042
:10C3900078E10610AFE10610660A002000E2061000
:10C3A000D853071042E20610B7E206102EE306103B
:10C3B00078E30610E5E30610840A002036E4061050
:10C3C00001080000A1E406101CE506104EE5061069
:10C3D0009BE0061007E10610E0E1061085E206107A
:10C3E000FBE20610A7E3061074E40610E7E406106B
:10C3F000012110B5080004F043FC10BD10B5002168
:10C40000022004F03DFC10BD10B50121042004F011
:10C4100037FC10BD10B5FFF7F1FF10BD10B5FFF7E9
:10C42000EDFF10BD10B512F0F9FEFFF7E7FFFFF7C3
:10C43000EBFF10BD10B5FFF7DBFF10BDF0B58FB0FF
:10C4400005281FD8F3F7F2FE2079031E8B0F002278
:10C450001100100004F0CDFD011E00D07BE0484B20
:10C460001874484866E0464B13219889FEF753FE3E
:10C47000011E454800D06FE044481CF0A9FF012090
:10C4800004F0C6FC0FB0F0BDFA26C825052436011D
:10C49000ED00062200210CA81DF09AF800221100E0
:10C4A000100004F0A6FD011E04D00C2802D038486C
:10C4B0001CF01EFF0123002008930693063302217F
:10C4C000019313222B000A90099007900590049085
:10C4D00003900290009604F053FD011E31D02D48C8
:10C4E0001CF006FF2C492D4C0F782D48E7744E7830
:10C4F00026758D786575CB78A3750A79E2754979CB
:10C5000021760297019600951CF0F2FE032123008C
:10C510001922002004F069FD011E18D021481CF0EA
:10C52000E7FE01210CAA080004F063FD011E1E486D
:10C5300012D11E481CF04CFFA4E70424302620250D
:10C54000A7E70F4B1A481C741CF042FFCAE71948B2
:10C550001CF03EFFE5E718481CF0CAFE92E7084BC6
:10C56000C8229889FA2392009B00110000930023AF
:10C57000FEF749FE011E01D01048EDE71048D9E74B
:10C58000840A00209EE8061006E6061030E6061033
:10C59000B2E60610F3E60610660A00200616002032
:10C5A0006AE70610A4E7061009E8061045E8061039
:10C5B00036E70610DEE7061072E80610C1E806103E
:10C5C00003E9061010B500210120224A04F04CFCBA
:10C5D00000210220204A04F047FC002104201F4AC9
:10C5E00004F042FCFFF7F0FDFFF7F8FD0122002404
:10C5F0001B4B52420A209A811C741CF089FE194878
:10C600001CF0E6FE03F0B8FA02F01FFF01F096FB03
:10C6100001F0D8FB01F0AEFC13481CF0D9FE0A2053
:10C620001CF076FE11481CF0D3FE01F0B1FC012095
:10C63000FFF704FF02F0F8FD802021000C4AC00043
:10C6400004F012FC802021000A4A400104F00CFC96
:10C6500010BDC04621C10410B5C00410BDC00410F7
:10C66000840A002043E906103CE90610E5E30610C1
:10C6700035C10410C5C00410F0B58FB0079314ABDA
:10C6800040CB05001C8816AB1B880F000A9317AB24
:10C690001B8805920B93002808D0290098481CF0AD
:10C6A00027FE0022974B1A740FB0F0BD96481CF07D
:10C6B0001FFE3578F3783279717902957578934851
:10C6C0000195B57800951CF013FE2000F6F7DAF915
:10C6D00000228F4BF5F778FA0D000400F6F796F973
:10C6E0000690F6F7CFF90022089009910023200068
:10C6F0002900F3F765FF002879D0089A099B2000EC
:10C700002900F5F729FD0022824BF5F75DFAF6F7CF
:10C710007DF90A230B99804C4B43020006992000B7
:10C7200000930A9B1CF0E4FD764A7C4D137C2800A4
:10C73000013B59424B4102331374059B97815C1EA8
:10C7400063425C41E4B22C706F8003F0D5F9744809
:10C750000470478002F078FE72480470478001F050
:10C76000DDFA059B012B00D099E002F069F9059BE9
:10C77000079C059A1C40079B0690134207D03F2256
:10C7800073799343C02B37D167481CF021FE0622F2
:10C7900066490CA81CF0C5FF002C09D10622300008
:10C7A0000CA91CF007FF002828D161481CF010FEDE
:10C7B00032000799380001F03DFE380003F0ACFB71
:10C7C00039005C481CF094FD02F028F901260400B1
:10C7D000688028002E7003F08FF95248067044805C
:10C7E00001F09CFA210054481CF082FD3EE022003A
:10C7F000089809992B0084E70024C8E7069B002BC2
:10C8000045D05B79002B42D0069B5A884B4B9A420D
:10C810003DD00699062230000C311CF0CBFE0028DA
:10C8200035D14748C2E70622300006991CF0C2FE07
:10C8300000280DD1069B0B990733180008931CF0B4
:10C84000E3FE002804D008993E481CF051FDAFE7F4
:10C85000069B01342933E4B206930A9B9C42E2D141
:10C8600039481CF0B5FD380001F0EEFB254B1B7C70
:10C87000032B03D10021082004F002FA059B002BB2
:10C8800023D1324B04201F8004F00EFA0CE7304B0A
:10C890001B780A932F4B06932F4B0B93DDE7059BD9
:10C8A000002BE3D12D481CF093FD3200079938008E
:10C8B00001F0C0FD02F0C4F801233900437205986D
:10C8C00002F0D8FC390026488EE7059B012B00D0EA
:10C8D000EAE602F0A9F8194CA04206D121481CF062
:10C8E00077FD0020FFF7AAFDDEE602F097F8A042F0
:10C8F00003D11D481CF06CFDD6E61C48FAE7C04683
:10C9000069E90610840A00209EE90610E1E9061094
:10C910000000F43F0000594025EA0610800A00207C
:10C920007C0A0020780A002092EA061089ED0610A1
:10C93000CCEA0610B2EB0610F0EB0610FFFF000089
:10C9400003EB06104DEB061083EB0610740A002073
:10C950000C0E00200D0E002046EB061030EC0610E9
:10C9600066EC0610ABEC0610F6EC061043ED061074
:10C97000F0B50378040099B0042B03D0822B0CD1BE
:10C98000071D00E0C71C63783E2B00D199E006D854
:10C99000052B21D0102B00D1BCE319B0F0BDFF2B2B
:10C9A000FBD178783B7800021843A24B984200D91B
:10C9B00003E10A3B9842F0D99F4BC0180928ECD8F4
:10C9C000F3F73EFC4203DA02EBFFEBFFEBFFEBFF7A
:10C9D000B802EBFFE802D80221796379E51C974C95
:10C9E0001B02A289964E0B439A423DD101235B4222
:10C9F000A3810023934823741CF0EAFCA9786B7888
:10CA000009021943EA7830001CF072FCAC786B78AC
:10CA100024021C4302F014F80388A34241D18A483F
:10CA20001CF0D6FC01F054FB0224012004F03CF978
:10CA300086486A780470AB781B021343438003F086
:10CA40005BF883486A780470AB781B021343438019
:10CA500002F0FAFC7F486A780470AB781B0213433B
:10CA6000438001F05BF998E77B481CF0B1FCA978A2
:10CA70006B78090219433000EA781CF039FCAE7873
:10CA80006B7836021E4301F0DBFF0388B34208D106
:10CA90006D481CF09DFC01235B42A381002323749D
:10CAA000C0E7AC786B7824021C4301F0C9FF4388CF
:10CAB000A342B9D169481CF08BFCE87801F0D6FD9F
:10CAC000B2E7E07801380C2800D966E7F3F7B8FB45
:10CAD0003B004F0065FF65FF65FF65FF610065FF77
:10CAE00065FF1F0065FF0D005900012004F0DCF810
:10CAF000A57963792D021D4301F096FF854200D090
:10CB00004BE7227AE179207901F056FD45E7651C73
:10CB1000ED7FE67FA17960792D0235430902237A02
:10CB2000E279014320790395A57F667F2D02354385
:10CB30000295E67E257F2D02354309340195009448
:10CB4000FFF79AFD29E7257DE67CA17960792D0222
:10CB500035430902237AE279014320790395A57CC4
:10CB6000667C2D0235430295E67B257CE3E72300B6
:10CB7000627BA079E11D64790E33009401F098FB8B
:10CB80000BE723002100227FE0791D3300240831C8
:10CB9000F3E7657923792D021D4301F045FF8542B6
:10CBA00000D0FAE6E17AA37AE07909021943A37981
:10CBB0000002184301F020FDEFE6294B984200D116
:10CBC00054E216D8274B984256D0274B984200D0B3
:10CBD000E3E6FC78BB7824021C4301F025FF844285
:10CBE00000D0DAE678793B790002184301F020FDA5
:10CBF000D3E61E4B984200D0CFE61D481CF0E8FB60
:10CC0000F979BB79090219431A481CF071FBFA79CA
:10CC1000BB79797912021A433B79F87809021943F2
:10CC2000BB78000218430023019300930833FEF7FA
:10CC3000CDFAB2E60A040000FFFBFFFF840A0020E1
:10CC4000B9ED061090ED0610F6ED0610800A0020F2
:10CC50007C0A0020780A002037EE061017EE061036
:10CC6000070C000002080000030C0000190C000073
:10CC7000DEF2061000F30610DA481CF0A9FBF97882
:10CC8000BB7809021943BE1CD7481CF031FBB079B0
:10CC9000737900021843F5F7F5FE0022D34BF4F741
:10CCA00093FF0D000400F5F7B1FE0690F5F7EAFEDC
:10CCB000002208900991002320002900F3F780FC4E
:10CCC000002800D1D1E0089A099B20002900F5F73F
:10CCD00043FA0022C64BF4F777FFF5F797FE0B9067
:10CCE000307AF37900021843F5F7CCFE0022BF4BEF
:10CCF000F4F76AFF0D000400F5F788FE0600F5F76B
:10CD0000C1FE002208900991002320002900F3F7BA
:10CD100057FC002800D1ADE0089A099B20002900AB
:10CD2000F5F71AFA0022B24BF4F74EFFF5F76EFE54
:10CD3000B04C33000B9A0699009020001CF0D8FAF2
:10CD4000FA213B7AFA791B0213430693BB7A7E7A67
:10CD50001B021E43BB7B7A7B1B0213431A1CC900B8
:10CD60008B4200D20A1C0A2192B20E92A2484A4378
:10CD700059431CF0BDFA0698F5F784FE9B4B002240
:10CD8000F4F722FF0D000400F5F740FE0B90F5F7D5
:10CD900079FE069B08900991172B01D9172E78D898
:10CDA0000022002320002900F3F70AFC002866D0A7
:10CDB000089A099B20002900F5F7CEF900228C4B38
:10CDC000F4F702FFF5F722FE08903000F5F75AFE5F
:10CDD0000022864BF4F7F8FE0D000400F5F716FE6E
:10CDE0000600F5F74FFE0022069007910023200071
:10CDF0002900F3F7E5FB002846D0069A079B2000A0
:10CE00002900F5F7A9F90022794BF4F7DDFE1E237E
:10CE10000193F5F7FBFD794C33000090089A200050
:10CE20000B991CF065FA18232826002406933B7BF7
:10CE3000FA7AF8781B021343BA780002049410437C
:10CE40003A79069903921022029201920E9A009268
:10CE50003200FEF7DFF9011E694803D1002C65D1CD
:10CE60001E2168481CF044FA97E5220008980999A9
:10CE70002B002CE72200089809992B0050E722008C
:10CE8000089809992B0097E72200069807992B002C
:10CE9000B7E70022002320002900F3F791FB0028C8
:10CEA0003AD0089A099B20002900F5F755F900228D
:10CEB0004F4BF4F789FEF5F7A9FD0F903000F5F719
:10CEC000E1FD0022494BF4F77FFE0D000400F5F769
:10CED0009DFD0890F5F7D6FD00220C900D910023E2
:10CEE00020002900F3F76CFB00281AD00C9A0D9B48
:10CEF00020002900F5F730F900223D4BF4F764FEDD
:10CF0000F5F784FD404C0090089B20000F9A0B9988
:10CF10001CF0EEF901248AE72200089809992B00F9
:10CF2000C3E722000C980D992B00E3E737481CF06B
:10CF30004FFA32E536481CF04BFABA78012A00D095
:10CF40002BE5FD78002D00D027E5324C2678012E08
:10CF500007D101F005FC80203100800003F090FE35
:10CF600025702D481CF034FA80200021C00003F009
:10CF700087FE12E52948DAE729481CF029FA294BEF
:10CF800029499889FEF701F9011E284800D069E770
:10CF90002748CCE727481CF01BFA7A793B79120224
:10CFA0001A43BB79F9791B04134309061943224834
:10CFB0001CF09EF97A793B7912021A43BB79F97910
:10CFC0001B041343090619431C481CF091F9154B27
:10CFD00001219889FEF7DDF8011E194800D041E7CC
:10CFE0001848A4E76EEE06109EEE06100000F43F0F
:10CFF00000005940BEEE0610F0EE061029EF0610B4
:10D00000B8EF061007F0061080EF061041F006108A
:10D0100066F00610760A00208CF00610CAF00610A2
:10D02000F8F00610840A002007B201001CF1061077
:10D030004EF1061072F10610A3F10610BEF10610B3
:10D04000D5F1061021F2061039481CF0C1F93979E2
:10D05000002907D07A7937481CF04AF90A201CF0D9
:10D0600057F99AE434481CF0B3F9F7E7334CFB78EE
:10D07000B97822881B020B439A4200D08DE420220B
:10D08000002110A81CF0A4FAFB79BA791B02134303
:10D090001D1CDBB21F2B00D91F253900EDB2083152
:10D0A0002A0010A81CF03DFB182200260AAB9B1892
:10D0B00023485E551CF08CF9218822481CF018F991
:10D0C00010A921481CF014F9204910A81CF09CFA62
:10D0D000B0421AD01E481CF07BF901F0B1FC238845
:10D0E000028805009A4206D11A481CF071F9012302
:10D0F0005B422E712B80184B184A1978208801F05A
:10D1000099F901235B42238047E410A914481CF0DD
:10D11000EFF8F6E7E378032B00D93EE4BFF34F8F37
:10D12000104B114ADA60BFF34F8FC046FDE7C0468F
:10D130005FF2061088F20610C7F2061004160020EF
:10D140000FF306104AF306106CF3061046EB0610B8
:10D1500086F30610C6F306106C0A00206D0A002044
:10D16000F5F3061000ED00E00400FA0537B5041EE3
:10D1700002D001281FD037BD9023019310330093B4
:10D180009F3B1A000100FDF7CAFF051E1BD11F4877
:10D190001CF01EF91E481CF01BF901212B00080091
:10D1A000C822FDF7D8FF011E26D01A481CF0A0F8AF
:10D1B000194B1D700DE0FDF7D2FF011E21D1174B59
:10D1C0001874174815E0290016481CF091F8124B06
:10D1D0001C70012000F000FF01F032FC002803D198
:10D1E0000120FFF72BF9C6E745300378002BF7D075
:10D1F0000D481CF0EDF8BEE70622084B0B481A74E8
:10D20000F7E70B481CF074F8B5E7C0469FF406102A
:10D21000CDF4061000F50610760A0020840A0020DE
:10D220008EF5061026F4061061F4061034F506108B
:10D230005BF5061070B5437801783A4A1B02060088
:10D2400086B00B43934202D0002006B070BDC37875
:10D2500082781B0201AC1343A381C37982791B023C
:10D260001343E381027A3049227202000A3262607B
:10D270004A88851C901C83420ED12B7A002B03D048
:10D28000012B07D00120E0E703232370200000F0EA
:10D29000B5F9F7E70223F8E7898802318B4208D114
:10D2A0002B7A002B03D0012BECD10523EDE70623CD
:10D2B000EBE701329342C7D101231C4823701CF0D5
:10D2C00087F86978B3780902194319481CF010F8F7
:10D2D00069792B790902194316481CF009F8E97994
:10D2E000AB790902194314481CF002F8EB79AA79CA
:10D2F0001B021343CAD011481BF0FAFF0026EB793A
:10D30000AA791B021343B34203D80A201CF000F889
:10D31000BCE7AB19197A0A4801361BF0E9FFB6B22F
:10D32000EDE7C046010C0000A20B0020B8F5061086
:10D33000DBF50610F9F5061011F606102BF60610AF
:10D3400035F6061070B51248FDF734FD114D280072
:10D35000FDF723FF041E16D021000F481BF0C8FF65
:10D360002800FDF71EFF0D4D28800D48FDF721FF19
:10D3700068800C48FDF71DFFA880002C02D00A48E9
:10D380001CF026F870BD09481CF022F8E8E7C046FA
:10D3900035D20410E45307103DF60610A20B00200E
:10D3A0000C54071030540710D2F6061091F60610F0
:10D3B00010B5012806D107480A7909681CF0B1F9AF
:10D3C000002010BD0028FBD10A790348531E9A4162
:10D3D000F3E7C0469E0A00209D0B002037B50300EE
:10D3E0000D001000002B16D01224012B11D1164B6A
:10D3F0009A880B68013201930B7992B20093042151
:10D400000023FDF7DAFE041E1AD0104821001BF09D
:10D410006FFF20003EBD09680B4A528801912979AF
:10D420000132009192B20421FDF7C7FE041E0848A4
:10D43000ECD12B68074819781BF05AFF0024E8E765
:10D4400005481BF0C5FFF9E7A20B002091F7061075
:10D4500001F706104DF70610D7F706100023F0B5B8
:10D46000454F85B0454802AD2B7102971BF0B0FFC8
:10D47000434B444819781BF03BFF434C4348217809
:10D480001BF036FF424E434831781BF031FF2178C4
:10D49000414839701BF02CFF317840481BF028FFC1
:10D4A000012332783E499A424BDC21783D482A716B
:10D4B0001BF01EFF3C4E3D4831781BF019FF718870
:10D4C0003B481BF015FF33780193012B3DD13948C0
:10D4D0001BF07EFF7288384B9A423DD0290001989C
:10D4E000FFF77CFF0400354821001BF001FF0C2CE6
:10D4F00021D133481BF06CFF3220F9F709F92900DC
:10D5000072880198FFF76AFF04002E4821001BF083
:10D51000EFFE0C2C0FD12C481BF05AFF6420F9F7BA
:10D52000F7F8290072880198FFF758FF0400274890
:10D5300021001BF0DDFE002C18D125481BF048FF10
:10D540000AE0C85CF8540133ADE722481BF040FF05
:10D5500029000120FFF72CFF522329003B700020F7
:10D56000513B2B71FFF724FF05B0F0BD21001A4895
:10D570001BF0BEFEF0E7C046A80B002009F806101D
:10D580000C0E002021F80610650A002036F806105F
:10D59000001600204FF8061062F8061093F80610E7
:10D5A00066090020BDF80610A00C00200CF906103A
:10D5B00040F9061079F90610FFFF0000BEF90610C9
:10D5C000F3F906101AFA06104FFA061077FA061049
:10D5D000ACFA06109AF90610DCFA06100022014B8C
:10D5E0001A707047AC0C0020034B18780138434286
:10D5F0005841C0B27047C046A00C0020F0B50500ED
:10D60000017893B0AF481BF073FE2C78601E05289C
:10D6100000D9D7E0F2F71EFE0600A802C102D6002C
:10D62000C302F302A8481BF0D3FEE989A7481BF008
:10D630005FFE297AA6481BF05BFE6B68A5481F7841
:10D6400039001BF055FE642F00D141E212D80A2F99
:10D6500071D9632F00D18DE13B00203B5E2B00D9B7
:10D660007FE2297A9C481BF043FE297A686801F022
:10D67000B9F9A7E0732F00D159E2762FECD12B7ABC
:10D68000012B00D86BE26B685C78022C00D963E256
:10D69000200002F005FC914A002C03D0904A012C96
:10D6A00000D1904A210090481BF022FE8AE00A2A0D
:10D6B00001D10133DBB20134E4B26246125DBB42F8
:10D6C000F5D3002322008948894D03706646B65C75
:10D6D000111BC9B20A2E32D1002B00D001700022DA
:10D6E000037839008348EA541BF002FE82481BF09D
:10D6F000FFFD01356B1E1C78002C27D10A201BF082
:10D7000007FE00F063FC7D4E0500022822D13000A8
:10D710001BF05EFE7A481BF05BFE30001BF058FEEB
:10D72000290078481BF0E4FD77481BF051FE77484C
:10D730001BF04EFE80E0764A00239446BDE7002EA3
:10D74000CAD0013201236E54D2B2BFE720001BF0D1
:10D75000DFFDCEE76F4B300005931B78002B10D117
:10D760001BF036FE6C481BF033FE30001BF030FE21
:10D7700039006A481BF0BCFD69481BF029FE694866
:10D78000D6E71BF025FE68481BF022FE0AAD3000EC
:10D790001BF01EFE0622210028001BF019FF02AB21
:10D7A000290038001C7608AA01F0B2F8049000287D
:10D7B0000AD039005D481BF09BFD059B5C48197839
:10D7C0001BF096FD13B0F0BD02AC247EEB782A79F5
:10D7D000697903942C78574802946C780194AC785A
:10D7E00000941BF085FD01F02BF904005248210044
:10D7F0001BF07EFD5148002C29D06379002B1DD0F1
:10D8000061884F4B994219D023000C33049A985CDD
:10D81000AA5C904200D0FBE1049A01320492062AED
:10D82000F4D148481BF064FD343447481BF0D0FD68
:10D83000217846481BF05CFD300008E023003433BB
:10D840001B78042B06D142481BF0C2FD41481BF057
:10D85000BFFDB7E7230026004633049345361A7808
:10D8600031783D481BF044FD2000290006220C3091
:10D870001BF057FF02AB1B7E2200A3740123E3724F
:10D880003370049B3C321F70002349341370042012
:10D89000237000F0A1FB049B31781A782F481BF00D
:10D8A00027FD01F0BBF8264B02002D49984200D01D
:10D8B0002C492D481BF01CFD2C481BF089FD2C48E1
:10D8C000C5E7C04630FB061068FB0610B7FB061024
:10D8D000CCFB0610E3FB0610D503071029FB06104E
:10D8E00025FB06102DFB061053030710AD0C00207E
:10D8F000AE0C002009FC06102CFC0610BA0C071018
:10D900003AFC061074FC061097FC0610CEFC0610BC
:10D91000660900200C0E00200BFD06103DFD0610D0
:10D9200052FD06107BFD0610ACFD0610DCFD061056
:10D930000BFE06108CD506102AFE061085FF061079
:10D94000FFFF0000E705071029060710550607101E
:10D950003EFE06107DFE0610B4FE0610EAFE06101E
:10D96000D50E07104ED30610BED506101FFF0610A9
:10D9700054FF0610B5481BF02BFDB5481BF028FDE1
:10D9800001F058F8002865D0B2481BF021FD08AC22
:10D99000202200210AA81BF01BFE062200212000E5
:10D9A0001BF016FE002302AAD37517339B18210023
:10D9B0001A000AA800F0D2FF011E49D10125A64F86
:10D9C000A64BFD2238001D701BF002FEA44E0AA8D3
:10D9D0003570F2F723FC0AA9C5B202003800757051
:10D9E0001BF09FFE2A002100AB1C0832DBB2D2B232
:10D9F00008780131F0540133DBB29342F8D1172794
:10DA000002AABF1897493A7809350D70803A0AA9D9
:10DA10009548F2541BF06CFC6579A3786278217804
:10DA20000295257991480195E47800941BF060FCFB
:10DA3000002179568E480A00803AD2B21BF058FC79
:10DA400001218C4B19708020800003F019F9B9E690
:10DA50008948FCE600F0F4FF00280DD0343001784E
:10DA6000062904D185481BF0B3FC8548EFE60B1F5F
:10DA7000012B01D88348A3E6834B84481D78002DF1
:10DA800000D0E4E600F0DCFF041E1BD0836B002B0B
:10DA900018D0F8F731FEA16B7D4B411A994211D88D
:10DAA0007C481BF025FC7C4C2378002B00D189E6B8
:10DAB0008020704B012180001D7003F0E1F8217877
:10DAC00076487DE600206B4B187000F083FB79E60A
:10DAD000734D28001BF07CFC72481BF079FC280079
:10DAE0001BF076FC00F0A6FF00281CD000F09CFF85
:10DAF00004006D4821001BF0FBFB6C481BF068FC28
:10DB0000132000F0B3FD6A481BF062FC13212000D3
:10DB1000FDF701FB674A011E00D1674A67481BF009
:10DB2000E7FB280093E666481BF052FCF9E76548DE
:10DB30001BF04EFC00F04AFA2421012302AA08AC93
:10DB4000521820700A9413700AA90020AA89FFF7BE
:10DB500045FC21785C4833E621005C4830E65C48AF
:10DB600075E639005B482BE65B481BF031FC00F0A2
:10DB70002DFA2421012302AA521808AC20700A941D
:10DB800013700AA90020AA89FFF728FC011E534838
:10DB900000D015E62178524812E6524857E6012493
:10DBA000514B52481C701BF013FCF8F7A5FD030005
:10DBB0004F4A50491068181A88420CD8F2F762FF91
:10DBC0004D49F2F749FEF4F7AFFF02000B004B4856
:10DBD0001BF08EFBF6E51360204B264D19782B7851
:10DBE000002907D0002B05D145481BF081FB2100FF
:10DBF0002C7028E74348012B00D0E3E527E60024FA
:10DC0000394B41481C701BF0E3FB1A4B1C70D9E5E3
:10DC10003E481BF0DDFB277BE37B227C617C029787
:10DC2000677B3B480197A47B00941BF061FB2C7839
:10DC3000EB782A79697902946C7836480194AC784B
:10DC400000941BF055FB344872E5C0469AFF06105D
:10DC5000D0FF0610EEFF061068090020650A0020BC
:10DC600066090020001600203B0007105400071032
:10DC70007B000710AC0C00209C000710C2000710AE
:10DC80000501071034010710760A00207001071003
:10DC900087130000AC0107100C0E0020E9010710EB
:10DCA000BA0C07102A020710510207107902071058
:10DCB000A30207101CFB061012FB0610C902071076
:10DCC000F3020710240307103C0307106F0307102B
:10DCD000A3030710FC030710150407107F040710A7
:10DCE0005A040710B3040710A00C0020D704071033
:10DCF000A80C0020B70B000000007A44FC040710B9
:10DD00003F05071089050710C10507109906071080
:10DD1000D706071007070710330707100378012BF2
:10DD200002D1024B42885A807047C046A00C0020A6
:10DD30000022014B1A707047A00C002010B5FFF7AD
:10DD400001FB80200021024A800003F08DF810BD05
:10DD50005DD40410030010B55A78007817491202F8
:10DD600086B002438A4202D0002006B010BDDA78A5
:10DD70009C78120201A822438281DA799C791202EE
:10DD80002243C2811C7A991C04720A330C4C4360F2
:10DD9000A38802339A420BD10B7A002B03D0012BBC
:10DDA00002D00120E1E70223037000F05FF8F8E7FA
:10DDB000638801339A42D7D10023F5E7010C0000B4
:10DDC000780D002070B50F48FCF7F4FF0E4C2000D2
:10DDD000FDF7E3F905002000FDF7E3F90B4C208087
:10DDE0000B48FDF7E6F960800A48FDF7E2F902000A
:10DDF00061882B00A0800132013107481BF078FABE
:10DE000070BDC04655DD04106C540710780D00201D
:10DE100094540710B854071073070710024B588822
:10DE2000013080B27047C046780D0020024B9888C0
:10DE3000013080B27047C046780D002013B5122320
:10DE400004001000012C0CD1074B9A880B6801329A
:10DE500001930B7992B2009304210023FDF7ADF9F1
:10DE60000300180016BDC046780D0020F0B50378F9
:10DE7000050085B0012B5AD0022B5DD0002B4CD170
:10DE8000027A322A49D82E4F416838001BF049FCEB
:10DE90002C4E2B7A337000F0D3FDA989041E44D098
:10DEA00042888A421FD10379002B1CD0264B1D7853
:10DEB000012D06D025481BF08BFA25481BF088FA67
:10DEC0002BE00288317823481BF012FA337802A93C
:10DED0000B71029728002288FFF7B0FF011E1E4831
:10DEE00019D11E48EAE723888B421AD160790028AD
:10DEF00017D0FFF793FF05006288317818481BF0B0
:10DF0000F7F90421337860882A000097FDF76FF94C
:10DF1000011E04D013481BF0EBF905B0F0BD124808
:10DF2000CCE712481BF0E4F9F7E71148C6E7064AC8
:10DF3000137083895380F0E70022034B1A70ECE7DB
:10DF40007F0D00207E0D0020B20D0020CC070710B1
:10DF50000E0807105108071093080710BB08071098
:10DF6000DF08071021090710480907106B0907107F
:10DF7000BC090710002210B5034B04481A705A80E0
:10DF80001BF026FA10BDC046B20D0020F4090710A0
:10DF900010B5502200210A481BF01AFB094B012240
:10DFA0001900524246311A600A701A0001214832A3
:10DFB00011700322503304481A701BF009FA10BD87
:10DFC000BC0D0020B80D0020100A0710014B187876
:10DFD0007047C046EC0D00207FB50400144E154D6F
:10DFE0002200317814481BF083F934702B79002B10
:10DFF0000AD0FFF7F9FA002806D02A880F4B9A4278
:10E0000003D10F481BF0E4F97FBD6B46DC71073389
:10E0100069460293012300200B7302A9FFF7DEF982
:10E02000011EF1D08828EFD006481BF061F9EBE71C
:10E03000EC0D0020B80D00202E0A0710FFFF000095
:10E040004A0A0710860A071073B51A4C050023798F
:10E05000002B09D02188814206D02A0016481BF0E7
:10E0600047F916481BF0B4F9012601A8067045804F
:10E070002580267101F040FD290011481BF038F978
:10E0800063793000002B07D061880E481BF030F90F
:10E090000D481BF09DF90620FFF79EFF29000B4855
:10E0A0001BF026F92300002244331A70F8F724FBF2
:10E0B000206473BDB80D0020CA0A07100D0B0710AD
:10E0C000470B07107B0B0710B90B0710DE0B07106F
:10E0D000F8B50123314C5B422380230000254433F3
:10E0E0001D70230026003C3328001D70257101F0AF
:10E0F000D7FE2B481BF06CF901F030FDFFF718FE3E
:10E1000028481BF065F94536FFF768FA26481BF0EA
:10E110005FF93378AB421CD0244F463438001BF0F3
:10E1200057F923481BF054F922481BF051F93800E5
:10E130001BF04EF90120FEF781F92800FFF74CFF94
:10E140001D481BF045F9227831781C481BF0D0F8A7
:10E15000F8BD60791A4D002810D0618819481BF06D
:10E16000C7F819481BF034F90520FFF735FF2800E0
:10E170001BF02EF90120FEF761F9E9E7FFF72CFF0C
:10E1800012481BF025F928001BF022F90120FEF7A8
:10E1900055F90F481BF01CF9DAE7C046B80D00200E
:10E1A000FE0B0710350C07107C0C0710B10C071084
:10E1B0004B0D0710830D0710B90D0710F70D071051
:10E1C000990E0710290E07106C0E0710CF0E0710BE
:10E1D000E20E0710F8B5274D01002B79002B06D170
:10E1E00025481BF0F5F8FF20FFF7F6FEF8BD0028E4
:10E1F00027D01F2221481BF0F3F92B0000223233D5
:10E200001A70002401260220EC72FFF7E5FE1C4F75
:10E210001C483E701BF0DCF81B481BF0D9F80220AC
:10E22000FEF70CF919481BF0D3F834352000FEF73F
:10E230009DFF2B78022B06D015483C701BF0C8F8C8
:10E24000D4E7E874DDE7CD22124B21001C70124B9D
:10E2500052001C70114B12481E701BF0B9F9FF22BE
:10E26000210010481BF0B4F9FFF7B8F90E4B0F4826
:10E270001E70E3E7B80D0020120F0710CB0D002031
:10E280006C100020330F0710680F0710980F07104D
:10E29000D50F07100C0E0020650A00200016002084
:10E2A0000D0E002066090020760A002017100710C6
:10E2B000F0B595B00993494B0B901B780E001700F1
:10E2C000022B00D087E0464B1B780893092B00D91E
:10E2D00081E0202200210CA81BF07AF900230A9388
:10E2E0009F4202D0099BDB5D0A9300240794BC4245
:10E2F00021D2099B1D5D002D1DD01B195B78083BA9
:10E30000012B13D82B1C202D00D92023013BDBB27D
:10E310000793099BA11C5918079A0CA81BF001FA36
:10E3200018200023079906AA1218535401346419BF
:10E33000E4B2A742DBD8079B002B4CD00024292550
:10E34000284F089AE3B29A423BD828226B469B1882
:10E350001B7831005BB20993089B223A5D437C191C
:10E3600020001BF0DEF907350B9B079A0CA97819E2
:10E37000A3711BF0D6F90022079B1B48E318DA7142
:10E380002300079A0833DA77089A099B511C28342E
:10E39000099A237073790592327804927278039205
:10E3A000B2780292F2780192327900920CAA1AF0B5
:10E3B0009FFF0B4A13780133DBB213700B4A1370C3
:10E3C00009E0280060430622310038181BF0F2F8FB
:10E3D00001340028B5D115B0F0BDC046EC0D0020C9
:10E3E0000C0E00200D0E002058100710650A0020AA
:10E3F00010B5002401220A4B21001C70094B0A4869
:10E400001C700A4B1A70CC3252001BF0E1F8FF224C
:10E41000210007481BF0DCF8FFF7E0F810BDC0460C
:10E420000C0E0020650A00200D0E002000160020B2
:10E4300066090020F0B5504C060023790D00170046
:10E4400089B0002B03D022884C4B9A4202D14C4811
:10E450001AF0BEFF0123637100236680E3802381ED
:10E46000A3729F4206D02000062239000C301BF018
:10E4700058F9A574E57C002D3FD1002F3DD0414BCC
:10E480001B780593404B0493059AEBB29A422BD923
:10E490000A2D29D029236B430193019A049B9446AA
:10E4A000634406223900180002931BF083F803909E
:10E4B000002854D10199354D049B073159181F226A
:10E4C00028001BF08DF82300039A32331A7028229B
:10E4D000029B29009A562B002D4820331A701AF0FF
:10E4E00007FFE37C002B08D1284D2A4928001BF0A8
:10E4F000FCF8290028481AF0FBFE06ABDD1D7F233F
:10E50000290030002B70FCF79CFE011E29D1002150
:10E51000230069563333214819701AF0E9FE0520AB
:10E52000FFF75AFD144B1D79002D20D01C481AF01E
:10E530004FFF0220FDF782FF300001F0EDFC3100BB
:10E5400018481AF0D5FE00234934174823701AF0F2
:10E550003FFF310015481AF0CBFE09B0F0BD013580
:10E5600092E723008022333311481A70D5E711480F
:10E570001AF02EFF2800DDE7B80D0020FFFF000095
:10E58000951007100C0E00200D0E0020CB0D002062
:10E59000E3100710201107102B1107105811071056
:10E5A000A71107104112071074120710A5120710C7
:10E5B00070110710EE11071010B5002808D00A4B93
:10E5C000010018001AF094FE0122084B9A7110BD48
:10E5D000032905D1032A03D105481AF0F9FEF3E710
:10E5E00004481AF085FEEFE7F3120710B80D00207B
:10E5F000391307107A1307100A00012110B5094CCE
:10E6000003002172E179002904D0190006481AF0AC
:10E610006FFE10BD190005481AF06AFE6088FCF70D
:10E62000DEFDF6E7B80D0020B4130710F81307104D
:10E6300070B50B4C0100E379012B10D00125094B7B
:10E64000E57118001AF054FE0620FFF7C5FC4734A8
:10E6500005481AF0BDFE2378002B00D1257070BD4F
:10E66000B80D00203014071048140710F8B5012326
:10E670000026324C05005B423148677A6380667140
:10E68000E680A66001F048FC2E481AF0A1FE132D8A
:10E6900001D0162D27D129002B481AF029FE22007F
:10E6A00000234932137022004532137023002500E5
:10E6B0005033493519782B788B4204D323481AF00C
:10E6C00017FE00232B702079002832D00120FFF79D
:10E6D00083FC1F481AF07CFE0120FDF7AFFE1D48A9
:10E6E0001AF076FE24E0002FE0D0230048331B7898
:10E6F000002BDBD02379002BD8D02500270049350B
:10E7000050372B783A789A42D0D901332B70F7F7EB
:10E71000F3FF230001224533E0641A703A78297828
:10E720000D481AF0E5FD3C3404202670FFF754FC38
:10E73000F8BDFFF751FC0948CCE7C046B80D0020F2
:10E74000FFFF000069140710971407102515071024
:10E750006B150710E6150710E5140710B215071022
:10E76000F0B50125554F564B3978564E564C85B06D
:10E7700056481970217035701AF0BAFD00218C4688
:10E780003B785348039333780193039A62454ED103
:10E79000002902D04B4A019313700024019A039977
:10E7A0004C481AF0A5FD4C4B4C481C701AF010FE5A
:10E7B0004B4B4C481C701AF00BFEFEF70FFF4A48FB
:10E7C0001AF006FE494F4A4C3D784A4829001AF093
:10E7D0008FFD207900286AD02300667934331978B8
:10E7E000002E02D10B1F022B44D843481AF080FDA3
:10E7F00005B0F0BD317801333970DBB22900013644
:10E80000013723E0029901324979D2B23970029975
:10E810000137013902912900B24222D1FE2A22D0C9
:10E8200007334778DAB2284B803F9F551BE062469A
:10E830000A2AADD00278FD2B03D8591CE254CBB282
:10E84000290006009A18203EE718D2B2934201D060
:10E85000FD2BCFD90200273A02921A009E1DE7181D
:10E86000F6B2FD2ACED963460133DBB29C4629308D
:10E8700013008AE70120FFF7AFFB20481AF0A8FD3C
:10E880003D70270029001E481AF032FD3C37002D4C
:10E8900008D11C481AF09CFDF7F72EFF0123A06356
:10E8A0003B70A5E718481AF093FD3E70A0E7FFF70C
:10E8B00093FB16481AF08CFD9AE7C0460C0E002018
:10E8C000650A00200016002066090020F8150710D0
:10E8D000340E0020251607106C1000205316071068
:10E8E000760A002087160710AB160710FD0D0020D2
:10E8F000B80D0020E5160710181707107717071036
:10E900009F170710D0170710131807105E1807106D
:10E9100070B5104B04001B7808001500A34202D804
:10E9200015D3013CE4B2002806D0292363430A49E9
:10E93000062259181AF0F5FE002D01D1002070BDF5
:10E9400029226243044B9B189B792B70F6E7012028
:10E950004042F4E70C0E00200D0E002073B51D4E52
:10E960000C0073791500002B31D0002805D0F37C02
:10E97000002B10D018491AF0B8FE002C07D0330035
:10E98000A21D587C013B207001349442F9D1002D26
:10E9900003D1002076BD0370EFE76B46DC1D7F23BB
:10E9A000237021007088FCF74CFC3336011E07D120
:10E9B000002161560948317029701AF099FCE8E786
:10E9C0000022B25606482A701AF092FCE1E70120B4
:10E9D0004042DFE7B80D0020CB0D00207B18071068
:10E9E0009818071010B5094B5A79002A03D1084826
:10E9F0001AF0EEFC10BD34331B780648062B01D00C
:10EA0000190005481AF074FCF4E7C046B80D002060
:10EA1000D018071020190710F1180710014B18889B
:10EA20007047C046B80D0020014B58887047C0465B
:10EA3000B80D0020014B58797047C046B80D002032
:10EA400000487047B80D002070B5134D134C2B785B
:10EA5000002B07D0260034363378043B022B02D833
:10EA600000232B7070BDF7F747FEA36BC01A0C4B49
:10EA70009842F7D90B481AF0ABFC00232B7023798E
:10EA8000002BEFD03478012CECD107481AF0A0FC11
:10EA90002000FDF7D3FCE5E7F40D0020B80D0020C1
:10EAA0000F27000062190710A81907107FB501F0A1
:10EAB00073FA0123050003AE3380364C2378052B0F
:10EAC00002D9217934485DE00133D8B22070023890
:10EAD000042804D8F1F7AAFB1C29364354002B78EC
:10EAE000002B11D12D481AF073FC022313226088E9
:10EAF00000960421FCF781FB011E3BD101236371C9
:10EB00002379013323717FBD25481AF061FCD4E7D6
:10EB10006B78002B07D123481AF05AFC6088022337
:10EB200016220096E5E72048EFE7AB78002B07D1E7
:10EB30001E481AF04DFC6088022319220096D8E77F
:10EB40001B48E2E7EB78002B07D11A481AF040FC8B
:10EB5000608802231C220096CBE71748D5E72B7963
:10EB6000002B0BD115481AF033FC608802231F22BA
:10EB70000096BEE712481AF0BBFB9EE71148C4E7B7
:10EB8000217911481AF0B4FB00232370013B638004
:10EB9000B9E7C046A4160020A91B0710D719071013
:10EBA000201A0710461A07106D1A0710901A07103E
:10EBB000B71A0710DA1A0710041B07102A1B0710D0
:10EBC000011A07104D1B07106C1B071041780378C2
:10EBD000F0B509021943B44B0400C8188DB01328CE
:10EBE00000D999E2F1F736FB92028601B200D1001A
:10EBF00098029802980214009802980298029802CB
:10EC000028027F02980298029802980298024D000A
:10EC1000E178A37809021943A448A71C1AF068FBFD
:10EC20007B78A2781B021343A14A002551889942A0
:10EC300004D0558BED1A691E8D41013518216943A9
:10EC4000521852889A4200D07CE0B8797B793E799C
:10EC5000000218433100F1F791FB6B4607901B7FD0
:10EC6000099300230893062E01D00C330893012347
:10EC7000059303330493059B099A013BDBB29A4247
:10EC800002D800200DB0F0BD049AA31C9A18117987
:10EC9000D77809020F43917956790902089A0E43F1
:10ECA000049984485218FF219B181A7ADB791202C2
:10ECB0001343079A01960A400097059906931AF0A4
:10ECC00017FB18226A437A4B9A189288002A01D0BF
:10ECD000974203D218226A439B189F8018226A43E6
:10ECE000734B9A18D288002A01D0964203D9182271
:10ECF0006A439B18DE80C023069A5B019A4211D1B9
:10ED000018226A436A4B6C489B181F815E811AF077
:10ED10005FFBA379049AD318DBB20493059B0133FC
:10ED20000593A8E7654B069A9A4207D118226A43D1
:10ED30005F4B63489B189F81DE81E8E70A201AF049
:10ED4000E7FAE6E75F481AF043FB9AE7E178A37831
:10ED50000902A2795C4819431AF0CAFA0025A61CD8
:10ED60003379AB4200D88CE7A90061188B7A4A7AD4
:10ED70001B0213430A7AC8791202290002430135A3
:10ED800052481AF0B5FAEDB2EAE7E178A378090241
:10ED900019434F481AF0ACFA0020E378A2781B021E
:10EDA0001343434AA61C51880690994205D0518BC3
:10EDB000C91A481E81410131069118210698414324
:10EDC000521857889F426CD1B57973792D023679E4
:10EDD0001D4331002800F1F7D1FAC3B20993002393
:10EDE0000893072E01D00C330893013DABB21B0AE8
:10EDF0002372C3B21A0039003648E57107931AF03E
:10EE000077FA0123059304330493059B099A013B88
:10EE1000DBB29A4200D834E70499089AA31C52182E
:10EE20009A18117AD57909020D432DD0049A9B18AE
:10EE30001979002928D0DA789F781202174323D055
:10EE40009A795E79120216431ED02B000091224857
:10EE5000079A0599029601971AF04AFAA8231F48C3
:10EE60009B019D420ED01E4B1E489D420AD01E4B58
:10EE70009D4212D1182206990D4B4A431B489B18FC
:10EE80001F825E821AF0A4FAA379049AD318DBB227
:10EE90000493059B01330593B7E70A201AF038FA6B
:10EEA000F2E713484FE7C046FDF3FFFFD61B0710FC
:10EEB000AC0F0020131C0710471C0710011800009E
:10EEC000601C0710871C0710DE1C0710321D07107E
:10EED000A11D0710D81D0710051E0710521E071090
:10EEE000012A0000711E0710052A00008F1E07105E
:10EEF000C71E0710E178A3780902194387481AF062
:10EF0000F7F90020E378A2781B021343844AA51C7A
:10EF100051880490994205D0518BC91A481E8141ED
:10EF200001310491182104984143521852889A42A1
:10EF300000D07FE02B79022B32D0042305930023ED
:10EF40000893A8796B79000218430599F1F716FA2E
:10EF5000C3B20993002302270693099B069A9342A2
:10EF600000D18EE6A31CD9198A794E791202164374
:10EF7000089AD2199B181A7ADD79A0231202154338
:10EF80009B019D4210D13200190066481AF0B0F979
:10EF9000059BDF19069BFFB20133DBB20693DCE76A
:10EFA00012230593063BCBE75F4B9D4208D100221D
:10EFB0005E4B29001A805E4B32005E481E80E5E7FA
:10EFC0005A4BA422022107932B0092018B439342B8
:10EFD0001BD1079B564A1B88128829005648009669
:10EFE0001AF086F9182204994D4B4A439B18079A48
:10EFF000598A1288914204D150489E821AF0E8F949
:10F00000C6E70A201AF084F9C2E7079B32002900FC
:10F010004B481E801AF06CF9A8234A489B019D4278
:10F02000ECD0494B49489D42E8D0494B9D42E8D13C
:10F030004848E3E7484886E6FEF7F8FEE179A37919
:10F040000902A51C194388421DD1FFF7F9FC0028CD
:10F0500000D116E60379002B00D112E602883F4B5F
:10F060009A4200D10DE60A340A94AB790AA90B71D1
:10F0700002880120FEF7E2FE011E394800D100E6B9
:10F080001AF036F9FDE5080012380C2823D8F1F7FC
:10F09000CDF80722220C22221122221622221C0045
:10F0A00020000A3000F07CFFEBE520000A3000F081
:10F0B000C1FFE6E520000A3001F006F8E1E5200096
:10F0C000A9790A3001F04CF8DBE52000A9790A3073
:10F0D00001F08EF8D5E5EA79AB7912021A4321489E
:10F0E0001AF006F9CDE5204A5379002B0AD0E378CF
:10F0F000A07851881B020343994203D10023537126
:10F10000FFF7D4FC022001F0CFFDBAE56179237945
:10F11000090216481943B3E71548B1E71B1F07104A
:10F12000AC0F00204F1F071003280000A80F00207D
:10F13000AA0F00207A1F0710C51F0710F91F07101C
:10F14000112007102E200710012A00004B20071065
:10F15000052A00006720071098200710FFFF000015
:10F16000E92007101F210710A41600205A210710BC
:10F170007521071070B5234D2B78012B03D1224840
:10F180001AF026F970BDFEF721FF04001F48210088
:10F190001AF0AEF8062C0AD11D481AF019F9FFF73B
:10F1A00043FC1C4B010018001AF0A2F8EAE7FF2C00
:10F1B0001CD119481AF00CF90120FEF70DFFFFF7DA
:10F1C00017F916481AF004F90220FDF737F9642000
:10F1D000F7F79EFA0220FEF7FFFE11481AF0F8F842
:10F1E0000020FDF7C3FF01232B70CBE7022CE6D1F3
:10F1F0000C481AF0EDF80120FDF7B8FF6420F7F78E
:10F2000087FADCE7760A0020700107108B210710CF
:10F21000C2000710AF210710E9210710680F07107F
:10F220004B2207100C22071000220D4B10B50D4881
:10F230005A705A76FBF7BEFD002801D0F5F7B8FFEB
:10F2400000210820084A01F00FFE80200021074A13
:10F25000400001F009FE06481AF0BAF810BDC04699
:10F26000AC0F0020CDEB0410CDF2041075F10410AA
:10F270006722071002000120824205D8173042435E
:10F280000020024B9B1859807047C046AC0F0020ED
:10F290000B4B10B51978002907D05A88824204D147
:10F2A00008481AF025F8002010BD002258800648B2
:10F2B0001A709A801AF08CF8FFF7F8FBF3E7C04653
:10F2C000A416002079220710C522071010B5084B9C
:10F2D0005C88084B9C4203D107481AF079F810BDAE
:10F2E000210006481AF004F82000FFF7D1FFF6E7E6
:10F2F000AC0F0020FFFF0000FB2207102A2307109D
:10F30000030010B55A7800781149120286B0024302
:10F310008A4202D0002006B010BDDA789978120235
:10F3200001A80A438281DA79997912020A43C281DB
:10F33000197A0A334360074B01725B8801339A42A2
:10F34000E8D10124047000F037F82000E3E7C0465C
:10F35000010C0000DE0F002070B51048FBF72AFDFD
:10F360000F4D2800FBF719FF041E12D021000D4895
:10F3700019F0BEFF2800FBF714FF0B4D28800B4847
:10F38000FBF717FF6880002C02D009481AF020F81C
:10F3900070BD08481AF01CF8ECE7C04601F30410F1
:10F3A000E854071072230710DE0F002010550710D5
:10F3B000FB230710C0230710037870B50500012B4D
:10F3C00018D1037A012B2FD9436800241A78762AA2
:10F3D0001DD15C78022C0ED8200000F061FD134A8C
:10F3E000002C03D0124A012C00D1124A21001248ED
:10F3F00019F07EFF70BD2100104819F079FFF9E780
:10F40000042C0CD90E4819F073FF0134E4B22B7AA6
:10F41000A342F5D80021102001F032FCEAE76B6826
:10F420001A5D084B1A55F0E70024F0E729FB061097
:10F4300025FB06102DFB061024240710422407107C
:10F440006B240710A5050020704710B5FFF784FF57
:10F4500010BD000010B543780178414A1B0286B008
:10F460000B43934202D0002006B010BDC3788178D0
:10F470001B0201AC0B43A381C37981791B020B43AF
:10F48000E381017A821C21720A3036496060488823
:10F49000023083420CD1137A002B03D0012B02D00F
:10F4A0000120E1E702232370200000F09DFAF7E736
:10F4B00088880230834208D1137A002B03D0012BB5
:10F4C000EED10423EFE70523EDE7C888023083423D
:10F4D00008D1137A002B03D0012BE1D10723E2E7F7
:10F4E0000823E0E708890230834208D1137A002B11
:10F4F00003D0012BD4D10A23D5E70B23D3E74889C6
:10F500000230834209D1137A0D211748DB0700D45A
:10F510000E21217019F0ECFEC6E788890230834283
:10F5200006D1137A10211048DB07F2D41121F0E73D
:10F53000C8890230834206D1137A13210A48DB07B7
:10F54000E7D41421E5E7098A02318B4200D08AE72B
:10F55000137A16210448DB07DBD41721D9E7C0460C
:10F56000010C00002A1000207E24071070B52948E5
:10F57000FBF720FC284C2000FBF70FFE051E45D0B2
:10F580002900264819F0B4FE2000FBF70AFE244C9F
:10F5900020802448FBF70DFE60802348FBF709FE1E
:10F5A000A0802248FBF705FEE0802148FBF701FE22
:10F5B00020812048FBF7FDFD60811F48FBF7F9FD26
:10F5C000A0811E48FBF7F5FDE0811D48FBF7F1FD2A
:10F5D00020821C4819F0FCFE61891B488A1C19F026
:10F5E00087FEA18919488A1C19F082FEE189184812
:10F5F0008A1C19F07DFE218A16488A1C19F078FEB3
:10F60000002D02D0144819F0E3FE70BD134819F024
:10F61000DFFEB9E755F404103455071095240710A0
:10F620002A1000205C55071080550710A4550710BC
:10F63000C8550710EC550710105607103456071020
:10F64000585607102025071041250710612507107F
:10F6500081250710A1250710C1250710E4240710F4
:10F6600010B501280FD002280FD0002809D10A4870
:10F670000B791A1C022B00D902220968D2B21AF0A7
:10F6800050F8002010BD0548F2E70B7904481A1C19
:10F69000032BF2D90322F0E71810002016100020E7
:10F6A0001310002037B515001224072815D8494A31
:10F6B0000C680B79F0F7BAFD041A2A3A4A5A6A7BA9
:10F6C000528804210132019400932800002392B251
:10F6D000FBF773FD041E02D1002420003EBD3E480E
:10F6E000882CFAD0210019F003FEF6E79288042155
:10F6F0000132019400932800002392B2FBF75DFDD4
:10F70000041EE9D03548882CECD1E6E7D2880421E4
:10F710000132019400932800002392B2FBF74DFDC3
:10F72000041ED9D02E48882CDCD1D6E712890421BA
:10F730000132019400932800002392B2FBF73DFDB3
:10F74000041EC9D02748882CCCD1C6E75289042191
:10F750000132019400932800002392B2FBF72DFDA3
:10F76000041EB9D02048882CBCD1B6E79289042168
:10F770000132019400932800002392B2FBF71DFD93
:10F78000041EA9D01948882CACD1A6E7D28904213F
:10F790000132019400932800002392B2FBF70DFD83
:10F7A000041E00D198E71248882C9BD195E7128A55
:10F7B00004210132019400932800002392B2FBF748
:10F7C000FCFC041E00D187E7882800D185E70948A2
:10F7D00088E7C0462A100020EB25071030260710C6
:10F7E00074260710B8260710FC26071041270710BB
:10F7F00087270710CC270710F7B500236D462B711C
:10F80000344B354C1B780094002B22D1334E344AB4
:10F810003389934216D1334F3B68002B05D0F6F75E
:10F820006BFF3B68C01AC72813D92F4B19782F4B91
:10F83000C9B29B78002B0DD12D4B1B78002B2AD001
:10F840002C4B08E0F6F758FF2B4B1B68C01AC72853
:10F85000E1D8F7BD294B1A7822705A7862709B78EC
:10F86000A3702B7903332B71B378052B1ED132890A
:10F870001B4B9A421FD17289194B9A42E9D0290039
:10F880000220FFF70FFF011EE3D08828E1D01C48BB
:10F8900019F02EFDDDE7194B1F7858783A009B7858
:10F8A00002431A43D5D027706070D9E7290002209F
:10F8B000FFF7D6FECDE70129DDD029000220FFF7B2
:10F8C000F1FE011ED7D08828D5D00E4819F010FDC2
:10F8D000D1E7C0466C100020781000207011002085
:10F8E000FFFF0000701000206B1000206610002049
:10F8F0003D1000205F10002074100020F401002053
:10F90000452807101028071073B52B4B1B78002BC8
:10F9100028D12A4C2A4D2389AB421CD1294E336869
:10F92000002B05D0F6F7E8FE3368C01AC72819D9AE
:10F93000254B1978254BC9B21B79002B13D1244BC9
:10F940001B78002B36D1234AD05C00280CD1013320
:10F95000142BF9D106E0F6F7CFFE1F4B1B68C01A37
:10F96000C728DBD873BD1B4A009214236A46137163
:10F970002289AA420FD001290DD0237B0F2B0AD157
:10F9800069460420FFF78EFE011E04D0882802D0AD
:10F99000124819F0ADFC6289AA42E3D069460420FE
:10F9A000FFF780FE011EDDD08828DBD00C4819F05F
:10F9B0009FFCD7E70B4AD7E76C100020701100209E
:10F9C000FFFF0000701000206B1000206610002068
:10F9D0003C100020850500207410002079280710B5
:10F9E000AF28071040100020007810B50138162805
:10F9F00013D8F0F71BFC0C1312181D122227122C1F
:10FA00003112363B124045124A4F1254590001221E
:10FA1000284B29481A7019F06BFC10BD0022254BA9
:10FA200026481A70F7E70322224B25485A70F2E75E
:10FA30000222204B23485A70EDE705221D4B224835
:10FA40009A70E8E704221B4B20489A70E3E70722EC
:10FA5000184B1F48DA70DEE70622164B1D48DA7095
:10FA6000D9E70F22134B1C481A73D4E70E22114B0F
:10FA70001A481A73CFE709220E4B19481A71CAE7C0
:10FA800008220C4B17481A71C5E70B22094B164880
:10FA90005A71C0E70A22074B14485A71BBE70D227E
:10FAA000044B13489A71B6E70C22024B11489A7125
:10FAB000B1E7C04670110020E42807101329071091
:10FAC0004329071071290710A0290710CE29071014
:10FAD000FD2907102B2A07105A2A0710892A071018
:10FAE000B92A0710E92A07101A2B0710492B07100B
:10FAF000792B0710A72B0710037810B5012B02D024
:10FB0000022B0CD010BD104B42881A81F6F7F4FD81
:10FB10000E4BC82118600E4819F0EAFBF2E70A4BB9
:10FB200042881989914206D101220A4852421A811B
:10FB300019F04EFCE6E759899142E3D10122524285
:10FB400005485A81F4E7C046701100207410002067
:10FB5000D62B0710312C0710822C07108022044B63
:10FB600092001A80034A5A800E221A737047C046C8
:10FB7000701100200406000010B5FFF7F7FC012209
:10FB8000094B52421A815A8100212020074A01F074
:10FB90006BF900214020064A01F066F9002180201F
:10FBA000044A01F061F910BD70110020BDFD041080
:10FBB000F9F7041009F9041073B500236C46314EAF
:10FBC000314D237133680095002B33D12F4E3368AC
:10FBD000002B05D0F6F790FD3368C01AC7282FD93F
:10FBE0002B4B1B78002B2BD12A4B19782A4BC9B2EF
:10FBF0001B78002B25D0294B1A782A705B786B7004
:10FC00002379274D023323712B78012B27D12A89A1
:10FC1000244EB24228D16A89B24211D0210000207C
:10FC2000FFF740FD011E0BD0882809D01E4819F0AF
:10FC30005FFB05E0F6F760FD3368C01AC728C5D83A
:10FC400073BD1A4B1B78002B01D0194BD4E7134B13
:10FC50001A785B7810001843F2D02A70CFE72100A1
:10FC60000020FFF7FDFCEBE70129D4D021000020A4
:10FC7000FFF718FD011ECED08828CCD00D4819F012
:10FC800037FBC8E7741000207810002070100020A7
:10FC90006C1000206B10002066100020F90100207D
:10FCA00070110020FFFF0000DB2C07103F10002028
:10FCB00064100020C02C0710F7B500236C46237198
:10FCC000314B324D1B780095002B22D1304E314AFA
:10FCD0003389934216D1304F3B68002B05D0F6F79D
:10FCE0000BFD3B68C01AC72813D92C4B19782C4B35
:10FCF000C9B25B78002B0DD12A4B1B78002B28D082
:10FD0000294B08E0F6F7F8FC284B1B68C01AC728F7
:10FD1000E1D8F7BD264B1A782A705B786B7023798F
:10FD2000023323717378032B1BD13289194B9A420A
:10FD30001CD17289174B9A42EBD021000120FFF7AA
:10FD4000B1FC011EE5D08828E3D01A4819F0D0FA9A
:10FD5000DFE7174B1A785B7810001843D9D02A7068
:10FD6000DCE721000120FFF77BFCD2E70129E0D08E
:10FD700021000120FFF796FC011EDAD08828D8D098
:10FD80000D4819F0B5FAD4E76C1000207810002067
:10FD900070110020FFFF0000701000206B10002089
:10FDA000661000203E100020621000207410002019
:10FDB000F70100202A2D0710F52C071010B5FFF7CA
:10FDC000FBFEFFF779FF10BD0023F0B585B002AA56
:10FDD0001371294B294E1B780296002B29D1284CF0
:10FDE000284D2389AB421DD1274F3B68002B05D0FE
:10FDF000F6F782FC3B68C01AC7281AD90B27234B99
:10FE00003A001B783000DBB22149019319F089FCDC
:10FE100002AB1F71E378072B0DD002A90320FFF777
:10FE20001FFC06E0F6F768FC1A4B1B68C01AC728CF
:10FE3000DAD805B0F0BD2289AA420ED16289AA4261
:10FE4000F7D002A90320FFF72DFC011EF1D088286E
:10FE5000EFD0114819F04CFAEBE7019B012BEDD0E4
:10FE600002A90320FFF71EFC011EE7D08828E5D079
:10FE70000A4819F03DFAE1E76C10002078100020E4
:10FE800070110020FFFF0000701000206B10002098
:10FE90009A05002074100020932D07105E2D071086
:10FEA00070B50500144E2A0034781448E4B22100DD
:10FEB00019F01EFA3570012D17D1012C0FD0104A00
:10FEC0001048517813780B439178D2780B43134341
:10FED00003D00D48FAF72EFB0C4819F079FA2A00E6
:10FEE00021000B4819F004FA70BD012CF7D1064827
:10FEF000FAF740FB0748F0E76B100020C72D07100A
:10FF0000661000202F2E0710BC050020042E0710BD
:10FF1000992E07106E2E071010B50400084B210013
:10FF20005881084819F0E4F9074B9C4207D0F6F7CE
:10FF3000E3FB064BC8211860054819F0D9F910BD3C
:10FF400070110020CD2E0710FFFF00007010002060
:10FF5000FB2E071037B50E4C042805D8F0F766F9CC
:10FF6000030F1113150021702579A3786278217889
:10FF70000195E4780748009419F0BAF937BD61702B
:10FF8000F2E7A170F0E7E170EEE72171ECE7C0461F
:10FF900066100020552F071000487047661000209B
:10FFA00073B51C4B027804001A7042785A70012213
:10FFB000194B1A70194B1B78002B29D1184D194B6E
:10FFC0002A899A4224D0F6F797FB174B1B68C01A70
:10FFD000C7281DD9154E3368002B13D12B78012B60
:10FFE00016D102236A4600941371694600202A89BB
:10FFF000FFF758FB011E0BD00C2809D00C4819F054
:020000041005E5
:1000000077F905E0F6F778FB3368C01AC728E5D81A
:1000100073BDC046641000203F1000206610002011
:1000200070110020FFFF00007410002070100020ED
:100030009D2F071073B51C4B027804001A7042788C
:100040005A700122194B1A70194B5B78002B29D179
:10005000184D194B2A899A4224D0F6F74DFB174BBD
:100060001B68C01AC7281DD9154E3368002B13D141
:100070006B78032B16D102236A46009413716946EC
:1000800001202A89FFF70EFB011E0BD00C2809D096
:100090000C4819F02DF905E0F6F72EFB3368C01A6D
:1000A000C728E5D873BDC046621000203E1000206E
:1000B0006610002070110020FFFF00007410002067
:1000C00070100020BF2F071073B51D4B027804007D
:1000D0001A7042785A7082789A700122194B1A70FD
:1000E000194B9B78002B29D1184D194B2A899A421C
:1000F00024D0F6F701FB174B1B68C01AC7281DD97F
:10010000154E3368002B13D1AB78052B16D1032382
:100110006A4600941371694602202A89FFF7C2FAE1
:10012000011E0BD00C2809D00C4819F0E1F805E0AD
:10013000F6F7E2FA3368C01AC728E5D873BDC0469F
:100140005F1000203D10002066100020701100207C
:10015000FFFF00007410002070100020E02F071037
:1001600073B50A1C1B4C0B2900D90B220100D2B21B
:10017000200019F0D6FA184BDB78002B29D1174D47
:10018000174B2A899A4224D0F6F7B6FA154B1B680A
:10019000C01AC7281DD9144E3368002B13D1EB7831
:1001A000072B16D10B236A4600941371694603206E
:1001B0002A89FFF777FA011E0BD00C2809D00B48CB
:1001C00019F096F805E0F6F797FA3368C01AC728D1
:1001D000E5D873BD54100020661000207011002077
:1001E000FFFF000074100020701000200130071085
:1001F00073B50A1C1D4C142900D914220100D2B277
:10020000200019F08EFA0122194B1A70194B1B7934
:10021000002B29D1184D194B2A899A4224D0F6F780
:100220006BFA174B1B68C01AC7281DD9154E3368C7
:10023000002B13D12B7B0F2B16D114236A4600946D
:100240001371694604202A89FFF72CFA011E0BD08E
:100250000C2809D00C4819F04BF805E0F6F74CFAD9
:100260003368C01AC728E5D873BDC04640100020C7
:100270003C1000206610002070110020FFFF0000DD
:1002800074100020701000202230071073B5194C34
:10029000194B228905009A422AD0F6F72DFA174BFE
:1002A0001B68C01AC72823D9154E3368002B19D1F3
:1002B0002379092B1CD1134B1B78002B18D0062354
:1002C0006A4600951371694605202289FFF7EAF90D
:1002D000011E0DD00C280BD0882809D00A4819F02F
:1002E00007F805E0F6F708FA3368C01AC728DFD820
:1002F00073BDC04670110020FFFF00007410002085
:10030000701000206B1000204430071073B5184C9B
:10031000184B228905009A4229D0F6F7EDF9164BC1
:100320001B68C01AC72822D9144E3368002B18D175
:1003300063790B2B1BD1124B1B78002B17D0062097
:100340006B460095187169462289FFF7ABF9011ECB
:100350000DD00C280BD0882809D00A4818F0C8FF07
:1003600005E0F6F7C9F93368C01AC728E0D873BDAD
:1003700070110020FFFF000074100020701000209A
:100380006B1000206730071073B5194C194B228988
:1003900005009A422AD0F6F7AFF9174B1B68C01A2E
:1003A000C72823D9154E3368002B19D1A3790D2BFB
:1003B0001CD1134B1B78002B18D006236A460095DE
:1003C0001371694607202289FFF76CF9011E0DD0D1
:1003D0000C280BD0882809D00A4818F089FF05E0BE
:1003E000F6F78AF93368C01AC728DFD873BDC0464C
:1003F00070110020FFFF000074100020701000201A
:100400006B1000208930071010B50C4C2368002BAE
:100410000DD10B4B1B78002B0FD10A48FFF736FF8D
:100420000948FFF773FF0948FFF7AEFF05E0F6F74D
:1004300063F92368C01AC728EBD810BD74100020D8
:100440006C100020B6050020B0050020AA05002091
:1004500010B5FBF78DF9064C00202100FBF7B4F92D
:1004600004490120FBF7B0F9034B1C6010BDC046E6
:1004700094110020841100208011002073B5040025
:1004800006A805880948022C00D10948094E3060A9
:10049000019300950B002100FBF738FB031E03D0EE
:1004A000023B5A425341981E76BDC046941100202B
:1004B0008411002080110020F0B587B003930CABAD
:1004C00084460C001D880292022917D1012314488A
:1004D0000E2702AABF186246124E3060022A10D1BF
:1004E0002B00039A02990097FBF7E0FA031E03D052
:1004F000043B5A1E9341D81E07B0F0BD00230A48A2
:10050000E6E7002A03D101001800FBF75DF9019727
:1005100000952100039B029A3068FBF797FAE5E704
:1005200084110020801100209411002070B5084D26
:10053000140013000A0001002868FBF7F9F80028EE
:1005400001D001DA200070BD03204042FBE7C04625
:100550008011002010B5022807D1074B1868074BFF
:10056000984201D0FBF736FB10BD0328FCD10020D8
:10057000FBF752FBF8E7C0468011002084110020F1
:1005800010B5EFF7BFFD10BD10B519F021F810BD83
:1005900010B519F00FF810BDF0B585B06C46070026
:1005A0000E0068461500FBF74BFD23783B7063781F
:1005B0003370A3782B7005B0F0BD10B5FBF7D0FBFE
:1005C00010BD10B5FAF76EFF10BD10B5FAF796FE24
:1005D00010BD10B51BF0D4F810BD10B51AF066FFB1
:1005E00010BD10B51BF096F810BD10B5FAF7F2FF6C
:1005F00010BD10B5FAF7FAFF10BD10B5FBF784FC7B
:1006000010BD10B5FBF782FC10BD10B5FBF780FCE8
:1006100010BD10B5F8F74EF910BD10B5FBF73CFD55
:1006200010BD10B5F8F7B6FF10BD10B5F8F7BCFF58
:1006300010BD10B5F8F7CCFF10BD10B5F9F764F98F
:10064000C0B210BD10B5F8F747FEC0B210BD10B56E
:10065000F8F71AFE10BD10B5F8F78EFE10BD10B5F4
:10066000012909D000290FD00624022905D0002431
:10067000032906D1412301E008244323012A00D1A4
:1006800072331B19C01A10BD0624F3E7C0224F2194
:10069000D205536888430B40034353607047C02220
:1006A0000823D20591690B4393617047C02201234F
:1006B000D20591690B439361704700008021024A83
:1006C00053688B4353607047C00000208023024A68
:1006D00051680B4353607047C00000207F21034ADC
:1006E000084053688B43034353607047C0000020A9
:1006F000014B18407047C04630DFCB008023DB033E
:1007000018407047002070478023DB051840704771
:1007100080239B041840704780239B01184070473A
:100720008023DB021840704780235B02184070472B
:1007300080239B031840704780239B00184070471C
:1007400080231B0118407047C00FC00770478023EB
:10075000DB041840704740231840704780235B0437
:100760001840704770478022436893434360704746
:10077000012243689343436070478068704710B517
:100780001422002118F024FF10BD202342681343D7
:1007900043607047102342681343436070477047BB
:1007A00083688160704780234268134343607047C9
:1007B0008023C268DB051343C36070478023C2688F
:1007C0009B041343C36070478023C2681B06134316
:1007D000C36070478023C268DB041343C360704763
:1007E0008023C2685B041343C360704704234268DC
:1007F0001343436070470368016070474368024ACF
:10080000134043607047C046FFFEFFFF70478023E0
:1008100042685B00134343607047402342681343C0
:10082000436070470123426813434360704780234D
:1008300042689B00134343607047C36809031B0D64
:10084000090B1B050B43C36070478023C2685B0321
:100850001343C36070478023C2681B041343C36003
:1008600070478023C268DB031343C3607047802353
:100870004268DB0013434360802342689B001343BC
:1008800043607047044A054809021369014004485F
:100890000340194311617047C000002000FFFF0FA3
:1008A000FF0000F07047000050235843054B064AF4
:1008B000C018036813400360036A044A13400362CC
:1008C0007047C046DC000020FFFFDFFFFFFFFFDFB7
:1008D00050235843064BC018802302689B031343E0
:1008E00003608023026A9B05134303627047C0467E
:1008F000DC00002050234343014A9B18586A70478C
:10090000DC00002050235843094BC018C36A1B0C5D
:100910000B70C36A1B0E4B70036B8B70036B9B02D7
:100920009B0CCB70036B9B029B0E0B717047C046F8
:10093000DC00002050235843014BC0187047C046CC
:100940001401002050235843014BC0187047C04683
:100950001C01002050234343024A9B18D86A80049C
:10096000800E7047DC00002050234343024A9B184E
:1009700018680006C00F7047DC0000205023434376
:10098000024A9B1818688004800E7047DC00002023
:1009900050235843064BC018C269120A0A60036A02
:1009A0001B0613430B60036A1B0ADBB24B607047E4
:1009B000DC00002050234343024A9B181868400083
:1009C000400F7047DC00002050234343024A9B182D
:1009D00018684001400F7047DC000020502343435B
:1009E000024A9B18D86A1F2318407047DC00002079
:1009F00050225043054B10B5C4180021200018F0B8
:100A0000E7FD402322681343236010BDDC00002073
:100A100050235843024BC018436A41627047C04696
:100A2000DC000020502310B558430D4B0C78C01843
:100A30004B78C26A1B02234392B21B041343C36266
:100A4000CB780C791B0289782404026B23430B4377
:100A50009B02920D92059B0A1343036310BDC0468F
:100A6000DC00002050235843044B0902C018836A5D
:100A7000090A1B0E1B060B4383627047DC00002033
:100A800050235843044B0906C018836A1B021B0AF3
:100A90000B4383627047C046DC0000205023FC22D9
:100AA0005843054B9201C0180902C36A1140034A1A
:100AB00013401943C1627047DC000020FFC0FFFFF4
:100AC0005023FC225843054B9201C01809020368C9
:100AD0001140034A1340194301607047DC000020B5
:100AE000FFC0FFFF50235843094BC018C2690B6871
:100AF000D2B21B021343C3614B680968026A090E34
:100B00001B020B43120C12049BB213430362704787
:100B1000DC00002050235843064BC018026A036AC9
:100B200092B21B0C1B041343802212021343036274
:100B30007047C046DC000020502380225843034BFE
:100B4000C0180368934303607047C046DC00002070
:100B500050235843024BC018836881607047C046D9
:100B6000DC0000205023E0225843054BD205C0187A
:100B7000090703681140034A134019430160704795
:100B8000DC000020FFFFFF8F50235843064B0A680C
:100B9000C018836982614B68FF21C2690B408A4398
:100BA0001343C3617047C046DC0000205023FF217F
:100BB0005843054BC018C269C3690A408B431343AD
:100BC00080221343C3617047DC0000205023584348
:100BD000034BC01880230268134303607047C0466C
:100BE000DC00002050235843024BC018436841608A
:100BF0007047C046DC0000205023E0225843054BDC
:100C0000D204C018090603681140034A134019436F
:100C100001607047DC000020FFFFFFF850231F2217
:100C20005843044B1140C018C36A93430B43C3623B
:100C30007047C046DC00002050233F225843044B3D
:100C40001140C018036893430B4303607047C046CC
:100C5000DC00002050235843034BC0188023026857
:100C60001B02534003607047DC000020122304285D
:100C700000D18B33180070477047704770470000F1
:100C800010B5EFF3108472B6054AC9001368034328
:100C90001360044BCA580243CA5084F3108810BD35
:100CA00040120020A41100200300EFF3108172B65F
:100CB000034A10681843106081F310887047C046DB
:100CC0003C12002070470000802200235202904214
:100CD00001D20004103380225204904202D2083321
:100CE000DBB2000280225205904202D20433DBB212
:100CF00000011F22D31A034A000F105C181AC0B259
:100D00007047C046DC560710F7B5364E364F33688D
:100D1000184001933060354B354A3C6835491B68B3
:100D200012680D681100306801400C4237D02C0069
:100D30001C401D4233D1304D2B6803401A4201D173
:100D40000124AB68E40028592B195A680840104266
:100D500002D1012252425A602C1963681840FFF7F1
:100D6000B3FF012181406368244A8B4310606360B4
:100D7000EFF3108072B60121136899403B688B43F2
:100D80003B60AB688B43AB602B688B432B6080F37D
:100D9000108812681A4B9200D3589847BBE701217C
:100DA000164A144C494211602268134216D1F2F7D8
:100DB000A0F8EFF3108572B60C4B39681A680C4B2B
:100DC0001B680B403168194204D123681A4201D1D3
:100DD000F2F790F885F31088FFF774FF019B3360FA
:100DE000F7BDC046F8170020401200203C1200203A
:100DF000FC17002038120020A4110020341200201B
:100E0000B411002010B5C043FFF77EFF10BD0000F5
:100E1000F7B5124F04003B6800250093013302D060
:100E2000009B01359D400E4E3368346001930D4B9D
:100E30001A6814420CD0009A3A60EFF3108172B62F
:100E40001A68A2431A6081F31088019B3360F7BDD2
:100E500021002800FFF7D6FFE9E7C0463412002042
:100E6000381200203C12002070B51400EFF31085FA
:100E700072B6FFF729FF034B8000C45085F310883A
:100E800070BDC046B411002080B5022801D91220DF
:100E900080BD01F091FF80BD80B502F089F980BD71
:100EA000BFB502AC2371099B6380089B23806B460E
:100EB00000259D70597018701846214601F026FBD8
:100EC00004B0B0BDBFB504466846012505730A9D50
:100ED0004581099D0581089DC580838042800180F0
:100EE000214601F03DFB04B0B0BD80B513460A4673
:100EF0000146402001F0A6FB80BD0000E0B56A4637
:100F0000002393800093052807D840B204A2105C08
:100F100000226B4601F096FB8CBD12208CBDC046B2
:100F2000010204081020000080B5072805D840B24F
:100F300003A1085CF9F780FF80BD122080BDC04688
:100F400001020408102040801FB51C4608460A997B
:100F50000391099902910899019107990091069BC3
:100F60001146224602F0ECF904B010BD80B51946D6
:100F7000104602F059FB80BD80B502F051FA80BDE9
:100F8000F0B593B01F4615460E4612901C9C0846BD
:100F90001146224602F0A6F9002824D122980D908D
:100FA0001FAB0DCB11901E980F901D980E901B98A3
:100FB0000C901A9919981097189F089209930D9AF6
:100FC0000A920097019002910C98039004940E9855
:100FD00005900F98069011980790129831462A466E
:100FE000109BFFF7B1FF13B0F0BD80B5FFF7BEFF58
:100FF00080BD80B5FFF7C0FF80BD80B5042801D952
:10100000122080BD12F08AF980BD0000F0B589B0D1
:101010000546084628431224012836D80E9F072F7C
:1010200033D3102F31D80F9810282ED8B8422CD394
:101030000E461099022928D8019102900393049238
:10104000F9F762FF012806D1049902291DD8039AF5
:10105000012A07D919E0039A10460499084301D0E0
:10106000112412E005AC019820730948E080029831
:1010700060712771E270A1706670257002F078F8D7
:101080006073204612F080F90446204609B0F0BD96
:101090000707000080B5044A914201D9122080BDA3
:1010A00012F09CF980BDC0463F420F0080B5012977
:1010B00002D812F0B1F980BD122080BD80B504F0D5
:1010C000DDFD80BD80B505F09FF880BD80B504F0E2
:1010D00085FE80BD80B505F0A1F880BDBFB51C467A
:1010E00002AB089D5D801A80099A03920093012348
:1010F000224604F0F9FF04B0B0BD1CB5059C019474
:10110000049C009405F078F800201CBD80B503F025
:1011100050FE80BD80B5002A02D003F057FE80BD8E
:10112000122080BDBCB51224002A08D0069D002BD9
:1011300001D0002D03D0009503F069FE044620463F
:10114000BCBDBCB51224002A08D0069D002B01D0DE
:10115000002D03D0009503F06AFE04462046BCBD76
:1011600000207047F0B58BB015460C463A490B6825
:101170000646283E062212210B2E10D900281CD02C
:10118000FF2835D0082817D0182815D080283CD043
:10119000812847D0FE284BD006280BD013E0C0464C
:1011A0007E4436797600B744050E050E110E080E02
:1011B0000E0E0E18022200E0102222701918284686
:1011C000FFF7DEF9002108460BB0F0BD01202070CA
:1011D0002C21595C01402970F4E702F07BF801A949
:1011E0000870012628463246FFF7CAF92670E9E75B
:1011F00001A8FFF7B5FF002826D001A9042628463C
:101200003246FFF7BDF9002120E00620207001A83A
:1012100012F045FD00281BD02278FF212846FFF759
:10122000B3F9CFE7062222700C4801686631C6E7A1
:1012300001AE304600F086FB0527284631463A4687
:10124000FFF79EF92770BDE7122100262670BAE746
:10125000227801A92031B2E7481200205012002064
:1012600080B5FFF77FFF80BD80B500F001F880BD3D
:10127000F8B50E4605461224FFF7BFF9B04217D362
:10128000012D15D80B480068817A00918572477A44
:1012900046722846FFF7B9F90024B74202D10098F8
:1012A000A84205D0FF207F2201210B460BF098FFBA
:1012B0002046F8BD9C12002080B5044800686030CC
:1012C00000210422FFF760F980BDC0469C12002077
:1012D00070B503460A480468EFF3108072B6207DAB
:1012E00000252575257C0F262E401E70237C1B09AA
:1012F0000B70E1681160411E884162B670BDC04646
:101300009C1200200348006800210175418201748D
:101310007047C0469C12002010B586B0154804687E
:1013200002A801A96A46FFF7D3FF00281FD002A830
:101330000178608AC840C00719D0019A009B03A8B1
:10134000082484701C0EC4721C0C84721C0A447223
:101350000372C2718171FF214170822101700021ED
:10136000417104220271C1700C21F9F733FD06B0FE
:1013700010BDC0469C120020BFB501AC089D258160
:10138000E380A28061802080204605F0CDFA04B081
:10139000B0BDBFB56C460A9DA581099D6581089DBC
:1013A0002581E380A280618020800B990C9A2046E1
:1013B00005F034FB04B0B0BD034800688821034A3F
:1013C000425000207047C0469C12002000000303DA
:1013D000054800688821415C88308078814201D8C6
:1013E00000207047012070479C12002005480068CB
:1013F0008921415C89308078814201D80020704782
:10140000012070479C12002010B504460A4800686D
:10141000006990210122134600F09AFA002804D0B6
:1014200001464460902000F030FB044800688821A9
:10143000425C521C425410BD4C1200209C120020F1
:1014400010B50446007AF721014021720A4800686D
:10145000006990210022012300F07AFA002804D0CC
:1014600001464460902000F010FB04480068892188
:10147000425C521C425410BD4C1200209C120020B1
:1014800010B50024C46107F0B3FB842800D0812488
:10149000204610BDB0B5096883240022002912D06F
:1014A000CD690024CC61087AC00603D4002005F081
:1014B000B9FD02E0084604F0EFFE012200282946AB
:1014C000ECD083240CE0D0070AD0EFF3108072B682
:1014D000044800688921425C521E425462B60024CE
:1014E000E0B2B0BD9C12002010B50C68207BC00794
:1014F00008D000210122204600F0F6F8207BFE21D2
:10150000014021730E4800682C21405CC00703D1C4
:10151000204605F0F9FC02E0204604F089FE002890
:1015200001D0832010BDEFF3108072B6054800682B
:101530008821425C521E425462B6002010BDC04653
:10154000481200209C12002070B50B4C012504228B
:10155000204629460EF02AFF084E3060062220461B
:1015600029460EF023FF31680860306801680020CA
:1015700088804880087070BDAC12002044120020A2
:10158000B0B50D460446411E8841511E1F220A4334
:10159000213291B20EF0E8FD002806D08580016866
:1015A0008160002C03D1402103E00020B0BD7F21E9
:1015B000C9430173001DB0BD80B5411E88410EF0C6
:1015C0003BFE80BD80B5017A8A0901219143001F4D
:1015D0000EF004FE80BD80B50A46017A8B09012118
:1015E000994340680EF03CFE80BD10B514460A4693
:1015F0004068194623460FF00DF810BD10B514468B
:101600000A464068194623460EF0CBFF10BDE0B5F0
:10161000022201ABFFF7F2FF002801D0002004E016
:1016200001A8017840780002401880B28CBDE0B576
:1016300001AB1A70120A5A70022200F001F88CBD38
:1016400010B514460A464068194623460EF06FFF4F
:1016500010BD011F00220A6040687047F8B50F48AE
:10166000006805682878411C29700D4F398A25319A
:101670004E09741C002809D1002021460EF02CFED2
:10168000388A25304009401C6880B41C012021465E
:101690000EF022FEA8880019A880F8BD4412002090
:1016A000B0120020F8B50E48006806683078401E79
:1016B00030700C49098A25314F097C1C000606D17F
:1016C0000025284621460EF05BFE7580BC1C0120DB
:1016D00021460EF055FEB088001BB080F8BDC04614
:1016E00044120020B012002070B591420ED215466F
:1016F0000E46044640680FF004F8751B60680EF053
:10170000D5FE281881B22046FFF765FF70BD80B571
:10171000002012F0E7FA80BDF0B58FB009930B926C
:101720000A9108900EF03CFE0124382120460EF06C
:101730004FFE3349C97A34228154324E306000273B
:10174000077030684770306887703068E121C17079
:101750000520C00131688880302008850EAD0DA9B4
:101760000CAA2846FEF718FF0C98000229780901F8
:1017700001430D9800030843001D31684885182176
:1017800020460EF025FE20490860077512F0A0FAE9
:101790001C9806901B9C05941A9804901998039025
:1017A0001898029017980190159D009508980A992D
:1017B0000B9A099BF9F71AFCF9F7A2FB1D9F012C64
:1017C00001D1F9F775FB00F089F9012F01D100F083
:1017D000BAF830682C21405CC0070ED1012C06D12C
:1017E0001698F9F79DFBF9F77AFCF9F77CFC0A9853
:1017F0000B992A46234601F043FA0FB0F0BDC046CC
:10180000B012002048120020EC120020F0B595B074
:101810000120810414912E480160BFF34F8FBFF364
:101820006F8FFEF74BFFFEF70DFF00201290C043B5
:10183000FEF72CFFF9F72CFB1390F9F72DFB119015
:101840000DF0E9FC109008F037FB0F90F9F75CFB06
:10185000F9F726FB0E9005F0A9FA0D9008F018FB99
:101860000C9008F019FB0B9004F0BFFE044605F045
:1018700009F80546F9F718FB064609F069FF07461F
:1018800000F064F8C0B2F9B208910990F0B2E9B280
:10189000E2B20B9BDBB20C9CE4B20D9DEDB20E9E4E
:1018A000F6B2129F00970196029503940493059255
:1018B000069107901398C0B21199C9B20F9AD3B28A
:1018C000109AFFF729FF03481499016015B0F0BD85
:1018D00080E100E000E100E0B0B50546C07A1224E6
:1018E000802829D8298C172926D31448821D914293
:1018F00022D8298A17291FD381421DD8A87E002803
:101900001AD008F0C9FA002808D0E87E002813D0C1
:10191000802811D8287F401E0E280DD80848342270
:101920002946FEF72DFE0EF077FF002803D4FFF7BF
:101930006DFF002400E087242046B0BDFA030000BC
:10194000B012002070477047704770470020704702
:10195000FEB515460C460646080614D402AA01AF89
:10196000304619463B4600F053F8002821D0600667
:1019700038D402988178FC220A4082700199018053
:10198000718001272FE0EFF3108072B602AA01AF39
:10199000304619463B4600F03BF800280BD0029930
:1019A0008A78FC2313408B70019A0A807280012789
:1019B00002E0002703E0002762B6002813D1EFF30E
:1019C000108072B6A0060AD4104800680168082288
:1019D0000A430260002012F0CBF9FAF72BFD62B641
:1019E00000260AE00027029EF570A0006021014059
:1019F000B078032202405018B070002F04D00020AD
:101A000012F0B6F9FAF716FD3046FEBD4C12002072
:101A1000F8B500924588AC081C80491C8AB2A6180B
:101A20008788BE4200D9091B0A199200BE4200D91C
:101A30006D1C0326354052191A80A3001B18083369
:101A4000009C236092B20588521B17463740848859
:101A50006743354052199208D21995B2C688B542EB
:101A600000D9C280A5420AD809B2002907D59978C1
:101A7000FC220A40511C9970083000990860A54268
:101A800001D90020F8BD0120F8BD80B5400605D47D
:101A90008878FC220240901C887080BD084600F0C7
:101AA00001F880BD80B5011DC278142A04D84268AF
:101AB00080788008904780BD3D2A03D8002000F040
:101AC000E9F880BD3F2A03D8002000F0F5F880BD7A
:101AD000602A02D8002000F0E4F880BDF8B50120AB
:101AE0001C21294A9047294F3860294DA88D401E56
:101AF00003263043401C8008C01C04242146224A8F
:101B0000904739684860E88D401E3043401C80088B
:101B1000C01C21461C4DA8472A46396888601C4DC8
:101B2000288E401E3043401C8008C01C2146904730
:101B30003968C860FFF7E6FB386842680021118009
:101B4000518083681980D180AF8D7F1E37437F1C01
:101B5000BF0897805980D980EF8D7F1E37437F1C47
:101B6000BF089F80C768398002614361F9802A8E6F
:101B7000521E3243521C9208BA80798087612246F5
:101B8000FEF702FDF8BDC046D10306104C1200203E
:101B9000B0120020FEB53D4D286810300021062906
:101BA00005D004C8528801AB5A52891CF7E7EFF3FD
:101BB000108072B6286804680027076062B6E007E4
:101BC00002D0002000F094FCA00702D5012000F014
:101BD0008FFC600702D5022000F08AFC200702D5A6
:101BE000032000F085FCE0064AD5042000F080FCCC
:101BF00046E0780001A90E5A0097BF002868C01976
